:020000040806ec
:100000000000060896a3140800008c0c20000401d0
:100010000200f0030000000000500010210006085c
:100020000d490e4a0e4b9b1a03dd043bc858d050b5
:10003000fbdc0b490b4a0020521a02dd043a8850bf
:10004000fcdc0949094a0a4b9b1a03dd043bc858ea
:10005000d050fbdc074880477c2f1408105100105b
:10006000c0c30010f8ba01108000060800000002aa
:10007000fc2e0e0271000002c809fa79010000008e
:1000800048740c0208020c0264020c0208790c028b
:10009000e0770c023c770c02307a0c0280760c027e
:1000a000d4790c02907a0c0290030c0240030c02eb
:1000b000ec750c02d87a0c02bc790c02e4750c02c7
:1000c0002c770c024c2f0c02e4030c02c0780c02bb
:1000d000f0780c023c780c02a0790c02387b0c0200
:1000e000b8740c0230790c02807a0c02ffffffff1b
:1000f00041f050fb18f044ff1bf0c8fe18f0caff97
:1001000081f0004102e000bf83f0004330b54feac8
:1001100041044fea430594ea050f08bf90ea020f35
:100120001fbf54ea000c55ea020c7fea645c7feac8
:10013000655c00f0e2804fea5454d4eb5555b8bfeb
:100140006d420cdd2c4480ea020281ea030382ea5c
:10015000000083ea010180ea020281ea0303362dee
:1001600088bf30bd11f0004f4fea01314ff4801cc1
:100170004cea113102d0404261eb410113f0004fd3
:100180004fea03334cea133302d0524263eb43038a
:1001900094ea050f00f0a780a4f10104d5f1200e28
:1001a0000ddb02fa0efc22fa05f2801841f1000183
:1001b00003fa0ef2801843fa05f359410ee0a5f157
:1001c00020050ef1200e012a03fa0efc28bf4cf088
:1001d000020c43fa05f3c01851ebe37101f000453e
:1001e00007d54ff0000edcf1000c7eeb00006eeb4b
:1001f0000101b1f5801f1bd3b1f5001f0cd34908d5
:100200005fea30004fea3c0c04f101044fea44522b
:1002100012f5800f80f09a80bcf1004f08bf5feab2
:10022000500c50f1000041eb045141ea050130bd92
:100230005fea4c0c404141eb0101013c28bfb1f5a4
:10024000801fe9d291f0000f04bf01460020b1faef
:1002500081f308bf2033a3f10b03b3f120020cdac2
:100260000c3208dd02f1140cc2f10c0201fa0cf0a0
:1002700021fa02f10ce002f11402d8bfc2f1200c05
:1002800001fa02f120fa0cfcdcbf41ea0c019040bb
:10029000e41aa2bf01eb0451294330bd6fea040404
:1002a0001f3c1cda0c340edc04f11404c4f12002ef
:1002b00020fa04f001fa02f340ea030021fa04f301
:1002c00045ea030130bdc4f10c04c4f1200220fa58
:1002d00002f001fa04f340ea0300294630bd21fa96
:1002e00004f0294630bd94f0000f83f4801306bf5c
:1002f00081f480110134013d4ee77fea645c18bf50
:100300007fea655c29d094ea050f08bf90ea020fe6
:1003100005d054ea000c04bf1946104630bd91eade
:10032000030f1ebf0021002030bd5fea545c05d1e1
:100330004000494128bf41f0004130bd14f5800420
:100340003cbf01f5801130bd01f0004545f0fe4194
:1003500041f470014ff0000030bd7fea645c1abfc9
:10036000194610467fea655c1cbf0b46024650ea00
:10037000013406bf52ea033591ea030f41f400212c
:1003800030bd00bf90f0000f04bf0021704730b5b2
:100390004ff4806404f132044ff000054ff0000187
:1003a00050e700bf90f0000f04bf0021704730b548
:1003b0004ff4806404f1320410f0004548bf40421d
:1003c0004ff000013ee700bf42004feae2014fea72
:1003d00031014fea02701fbf12f07f4393f07f4f4d
:1003e00081f06051704732f07f4208bf704793f050
:1003f0007f4f04bf41f40021704730b54ff4607463
:1004000001f0004521f000411ce700bf50ea010265
:1004100008bf704730b54ff000050ae050ea01020e
:1004200008bf704730b511f0004502d5404261eb7e
:1004300041014ff4806404f132045fea915c3ff4bf
:10044000d8ae4ff003025feadc0c18bf03325fea5c
:10045000dc0c18bf033202ebdc02c2f1200300fa0d
:1004600003fc20fa02f001fa03fe40ea0e0021fa32
:1004700002f11444bde600bf70b54ff0ff0c4cf420
:10048000e06c1cea11541dbf1cea135594ea0c0fd2
:1004900095ea0c0f00f0def82c4481ea030621ea0d
:1004a0004c5123ea4c5350ea013518bf52ea033548
:1004b00041f4801143f4801338d0a0fb02ce4ff0fa
:1004c0000005e1fb02e506f00042e0fb03e54ff02a
:1004d0000006e1fb03569cf0000f18bf4ef0010e22
:1004e000a4f1ff04b6f5007f64f5407404d25fea1e
:1004f0004e0e6d4146eb060642eac62141ea5551d1
:100500004feac52040ea5e504feace2eb4f1fd0c12
:1005100088bfbcf5e06f1ed8bef1004f08bf5fea90
:10052000500e50f1000041eb045170bd06f0004642
:1005300046ea010140ea020081ea0301b4eb5c04ef
:10054000c2bfd4eb0c0541ea045170bd41f48011e7
:100550004ff0000e013c00f3ab8014f1360fdebf0c
:10056000002001f0004170bdc4f10004203c35dae8
:100570000c341bdc04f11404c4f1200500fa05f36b
:1005800020fa04f001fa05f240ea020001f000420c
:1005900021f0004110ebd37021fa04f642eb060182
:1005a0005eea430e08bf20ead37070bdc4f10c04ac
:1005b000c4f1200500fa04f320fa05f001fa04f270
:1005c00040ea020001f0004110ebd37041f100015c
:1005d0005eea430e08bf20ead37070bdc4f1200567
:1005e00000fa05f24eea020e20fa04f301fa05f2cf
:1005f00043ea020321fa04f001f0004121fa04f277
:1006000020ea020000ebd3705eea430e08bf20ea46
:10061000d37070bd94f0000f0fd101f00046400080
:1006200041eb010111f4801f08bf013cf7d041ea02
:10063000060195f0000f18bf704703f00046520006
:1006400043eb030313f4801f08bf013df7d043ead7
:100650000603704794ea0c0f0cea135518bf95ea8d
:100660000c0f0cd050ea410618bf52ea4306d1d114
:1006700081ea030101f000414ff0000070bd50ea33
:10068000410606bf1046194652ea430619d094eabd
:100690000c0f02d150ea013613d195ea0c0f05d1a7
:1006a00052ea03361cbf104619460ad181ea0301fb
:1006b00001f0004141f0fe4141f470014ff00000b3
:1006c00070bd41f0fe4141f4780170bd70b54ff04e
:1006d000ff0c4cf4e06c1cea11541dbf1cea1355ce
:1006e00094ea0c0f95ea0c0f00f0a7f8a4eb0504b0
:1006f00081ea030e52ea03354fea013100f08880a7
:100700004fea03334ff0805545ea131343ea12636f
:100710004fea022245ea111545ea10654fea002624
:100720000ef000419d4208bf964244f1fd0404f5dd
:10073000407402d25b084fea3202b61a65eb030539
:100740005b084fea32024ff480104ff4002cb6ebf6
:10075000020e75eb030e22bfb61a754640ea0c0076
:100760005b084fea3202b6eb020e75eb030e22bfb6
:10077000b61a754640ea5c005b084fea3202b6ebf7
:10078000020e75eb030e22bfb61a754640ea9c00b6
:100790005b084fea3202b6eb020e75eb030e22bf86
:1007a000b61a754640eadc0055ea060e18d04fea44
:1007b000051545ea16754fea06164feac30343eae4
:1007c00052734feac2025fea1c1cc0d111f4801fb1
:1007d0000bd141ea00014ff000004ff0004cb6e7aa
:1007e00011f4801f04bf01430020b4f1fd0c88bf49
:1007f000bcf5e06f3ff6afaeb5eb030c04bfb6eb54
:10080000020c5fea500c50f1000041eb045170bd46
:100810000ef0004e4eea113114eb5c04c2bfd4eb73
:100820000c0541ea045170bd41f480114ff0000ef7
:10083000013c90e645ea060e8de60cea135594ea73
:100840000c0f08bf95ea0c0f3ff43baf94ea0c0f76
:100850000ad150ea01347ff434af95ea0c0f7ff4eb
:1008600025af104619462ce795ea0c0f06d152ea3f
:1008700003353ff4fdae1046194622e750ea410623
:1008800018bf52ea43067ff4c5ae50ea41047ff434
:100890000daf52ea43057ff4ebae12e74ff0ff3c99
:1008a00006e000bf4ff0010c02e000bf4ff0010c6a
:1008b0004df804cd4fea410c7fea6c5c4fea430ce3
:1008c00018bf7fea6c5c1bd001b050ea410c0cbf32
:1008d00052ea430c91ea030f02bf90ea020f002094
:1008e000704710f1000f91ea030f58bf994208bffb
:1008f00090422cbfd8176feae37040f001007047b8
:100900004fea410c7fea6c5c02d150ea013c07d10e
:100910004fea430c7fea6c5cd6d152ea033cd3d059
:100920005df8040b704700bf8446104662468c4653
:100930001946634600e000bf01b5fff7b7ff002886
:1009400048bf10f1000f01bd4df808edfff7f4ffaf
:100950000cbf012000205df808fb00bf4df808ed3a
:10096000fff7eaff34bf012000205df808fb00bf5d
:100970004df808edfff7e0ff94bf012000205df87f
:1009800008fb00bf4df808edfff7ceff94bf012034
:1009900000205df808fb00bf4df808edfff7c4ff2d
:1009a00034bf012000205df808fb00bf4fea410c76
:1009b0007fea6c5c02d150ea013c0ad14fea430c59
:1009c0007fea6c5c02d152ea033c02d14ff0000096
:1009d00070474ff0010070474fea410212f50012d4
:1009e00015d211d56ff47873b3eb625212d94fea76
:1009f000c12343f0004343ea505311f0004f23fa60
:100a000002f018bf404270474ff00000704750eab4
:100a1000013005d111f0004008bf6ff00040704771
:100a20004ff00000704700bf4a0011d212f50012cb
:100a300011d20dd56ff47873b3eb62520ed44fea36
:100a4000c12343f0004343ea505323fa02f07047b6
:100a50004ff00000704750ea013002d14ff0ff30f4
:100a600070474ff00000704753b94ab9002908bfda
:100a700000281cbf4ff0ff314ff0ff3000f096b957
:100a8000adf1080c6de904ce00f01af8ddf804e0d1
:100a9000dde9022304b07047430803f05533c01a60
:100aa000830800f0333003f03333184400eb1010a8
:100ab00000f00f3000eb002000eb0040000e70470c
:100ac0002de9f04f099d04460f46002b48d18a427c
:100ad000944661d9b2fa82f343b1c3f120019f4039
:100ae00002fa03fc9c4020fa01f10f434fea1c413b
:100af0001ffa8cfe220cb7fbf1f601fb167706fb02
:100b00000ef042ea0742904208d91ceb020206f1bd
:100b1000ff3702d2904200f237813e46121aa4b249
:100b2000b2fbf1f001fb102200fb0efe44ea02448e
:100b3000a64508d91ceb040400f1ff3202d2a645f9
:100b400000f21c81104640ea0640a4eb0e04002689
:100b50001db1dc400023c5e900433146bde8f08ffc
:100b60008b4209d9002d00f0fd800026c5e9000167
:100b700030463146bde8f08fb3fa83f6002e4bd1f4
:100b80008b42c0f0f280824240f2ef803046002d6e
:100b9000e3d0c5e90047e0e702b9ffdeb2fa82f32d
:100ba000002b40f09d80891a4fea124e97b2012621
:100bb000200cb1fbfef20efb121140ea014107fbd3
:100bc00002f088420fd91ceb010102f1ff382cbf63
:100bd0004ff001094ff00009884203d9b9f1000f25
:100be00000f0cf804246091aa4b2b1fbfef00efb22
:100bf000101100fb07f744ea0144a74208d91ceb97
:100c0000040400f1ff3102d2a74200f2b48008468a
:100c1000e41b40ea02409be7c6f12007b34001fa1b
:100c200006f422fa07fcf940b2404cea030c20fa21
:100c300007f34fea1c491c431ffa8cfe00fa06f327
:100c4000200cb1fbf9f809fb181140ea014108fb3f
:100c50000ef088420fd91ceb010108f1ff3a2cbfbe
:100c60004ff0010b4ff0000b884203d9bbf1000f8e
:100c700000f08d80d046091aa4b2b1fbf9f009fb4f
:100c8000101100fb0efe44ea01418e4507d91ceb12
:100c9000010100f1ff3401d28e457fd8204640eaa1
:100ca0000840a1eb0e01a0fb029841454c46c64608
:100cb00002d306d14b4504d20138b9eb020468ebec
:100cc0000c0e002d70d01a1b61eb0e0122fa06f3f8
:100cd00001fa07f7f14000261f43c5e900713ce720
:100ce00002fa03fcc3f1200001fa03f221fa00f634
:100cf0004fea1c4e24fa00f11ffa8cf79c40114376
:100d0000b6fbfef00a0c0efb106642ea064200fb40
:100d100007f696420ed91ceb020200f1ff382cbff9
:100d20004ff001094ff00009964202d9b9f1000fc6
:100d300031d04046921b89b2b2fbfef60efb162262
:100d400041ea024106fb07f28a4207d91ceb010186
:100d500006f1ff3801d28a4223d84646891a46ea6c
:100d6000004625e72e462846f7e6841a61eb030382
:100d700001201f460be76444023849e76444023807
:100d8000e1e6023a61442ee7023e6244c6e6a8f17b
:100d9000020861446fe702386244cbe702386144dd
:100da0007de7023e6144d9e72e46d6e6704700bf94
:100db00010f8012b11f8013b012a28bf9a42f7d005
:100dc000d01a7047034613f8012b002afbd1181ada
:100dd000013870477bb972b90029bebf00204ff0bf
:100de000004106e008bf00281cbf6ff000414ff033
:100df000ff30fff7dbbfadf1080c6de904ce002931
:100e000009db002b1adbfff75bfeddf804e0dde910
:100e1000022304b07047404261eb4101002b1bdb11
:100e2000fff74efeddf804e0dde9022304b04042a6
:100e300061eb4101524263eb43037047524263eb63
:100e40004303fff73dfeddf804e0dde9022304b0d3
:100e5000404261eb41017047524263eb4303fff7ad
:100e60002ffeddf804e0dde9022304b0524263eb1b
:100e70004303704709b504480068044b03441b68ea
:100e80001b68029309bd0000e8c3001004000000c5
:100e900009b504480068044b03441b685b6802936f
:100ea00009bd0000e8c300100400000009b50448b3
:100eb0000068044b03441b689b68029309bd000053
:100ec000e8c300100400000000b1807b704708b147
:100ed000c07b7047ff20704708b1408970474ff6cc
:100ee000ff70704708b1808970474ff6ff707047f8
:100ef00042680068101a704709b504480068044b3e
:100f000003441b681b68029309bd0000e8c300107e
:100f1000000000007047000010b50021012017f00c
:100f20006dfe044617f0ecfe24b9bde81040042025
:100f30000af0f4bc0028f8d1024823f003fa002894
:100f4000f3d110bdc0c3001008b50af005fd043888
:100f500018bf012008bd000010b5fff7f5ff20b154
:100f6000bde81040014bdb69184710bdc0c300103d
:100f700010b5fff7e9ff20b1bde81040014b5b6af7
:100f8000184710bdc0c3001010b5fff7ddff20b13a
:100f9000bde81040014b1b6a184710bdc0c30010cc
:100fa000f8b504460e4617461d4624b92846bde846
:100fb000f8401cf075bae72000f042f930461cf00a
:100fc0006ffae72000f060f938461cf069fa013c3e
:100fd000ebe70000014b1860704700bfecc3001046
:100fe0002de9ff4104460020039118f0b7f8234b88
:100ff0001b6813b12046039998474ff47f0000f017
:101000007ff8602000f09ef800f090f80023009335
:1010100001231b4a18461b4900f070ffe72000f02f
:1010200033f94ff47f0000f06bf80226164ddff81d
:101030006880164f2b4641460320134afff7b0ff46
:101040002b4639460320104afff7aaff2a4641469d
:1010500003200f4bfff7a4ff3a4620460d4b0b49e8
:10106000fff79eff012e07d100222146822004b007
:10107000bde8f04117f016be0126dbe7ecc3001017
:10108000dd6c0c02dc030c02a0860100e09304007e
:10109000a0bb0d0000350c00f049020037b500255b
:1010a0000195069d079c009500f074fa04b120603c
:1010b0007f28a8bf7f2040b203b030bd10b5054bdc
:1010c0001b7800fb03f4044b0020db689847604367
:1010d000000c10bd2a5100101051001038b5054603
:1010e000c0f307400c46fff7e9ff2080c5f3072057
:1010f000fff7e4ff6080e8b2fff7e0ffa08038bdb3
:10110000014b1860704700bff4c30010014b18601a
:10111000704700bff8c3001010b9024b1868704741
:10112000014bfbe7f4c30010f8c30010044b1a781e
:1011300022b100210120197000f0fcbf704700bff0
:10114000f0c30010014b1870704700bf2a51001007
:10115000014b1878704700bf2a510010024b1860ed
:10116000024b1960704700bffcc3001000c40010a0
:1011700010b5054b0446db68002098472402b4fbf9
:10118000f0f0c0b210bd00bf105100102de9f341c6
:10119000dff83480044600216846d8f808309847c4
:1011a0006e46671e02340020d8f80c3036f8025b19
:1011b00098472d02b5fbf0f507f8015fa742f2d181
:1011c00002b0bde8f08100bf1051001010b4054b13
:1011d00082885c684188a446002300885df8044b3f
:1011e000604700bf1051001030b50e4d85b0044669
:1011f000fff7ecff2b689bb12088fff7b9ff039046
:101200006088fff7b5ff0290a088fff7b1ffdde926
:10121000022103460020009003482c680068a04784
:1012200005b030bdfcc3001000c4001007b569460e
:10123000fff754ff6846fff7d7ff03b05df804fbe4
:1012400008b510b1e72805d008bd0120bde8084069
:101250001bf0cbbb074b1b7853b1074b1868fff74c
:10126000e5ff6322054b1a70ff22054b1a70ebe76e
:10127000044bf3e7f0c30010f8c30010295100102d
:1012800028510010f4c3001008b510b1e72804d0ad
:1012900008bdbde808401bf0a8bb0020fff7c6ff53
:1012a0000022034b1a700122024b1a70f0e700bfb4
:1012b000295100102851001013b518b1e72807d0a4
:1012c00002b010bd104b5b6902b0bde8104018477a
:1012d0000e4b1b78a3b10e4b1c680b4b00219b6877
:1012e00068469847bdf80220bdf800301343bdf8aa
:1012f000042013439bb22bb10020fff797ffdfe7d9
:10130000044be9e72046f8e710510010f0c3001045
:10131000f8c30010f4c3001038b5094b1a7802f076
:10132000ff0462b90125214620461d7000f002ff2e
:101330002046fff77bff034b1c70034b1d7038bd2d
:10134000f0c30010295100102851001013b50446b5
:1013500008466946fff7c2fe6322bdf800306343ca
:10136000b3fbf2f3adf80030bdf802306343b3fbda
:10137000f2f3adf80230bdf8043004fb03f0b0fb2b
:10138000f2f0adf804006846fff72eff02b010bd82
:1013900010b40f4c024623780e4983b9012008701f
:1013a0000878e72a0344d8b220700ed10a4b1b7884
:1013b0004bb10a4b19685df8044bfff7c7bf632bad
:1013c000eed1ff20ebe7064bf4e75df8044b7047e6
:1013d0002951001028510010f0c30010f8c300106c
:1013e000f4c30010024b1878003818bf0120704772
:1013f000f0c3001084b030b503ac84e80f00064c95
:1014000003ad0fcd0fc495e8030084e80300bde8e9
:10141000304004b0704700bf1051001070b5054651
:1014200000200e46144627f005f940b12346324607
:101430006968403045f00cff231a5842584170bd8e
:1014400070b5054600200e46144627f0f3f840b16b
:10145000234632466968403046f0b5f8231a5842b0
:10146000584170bd01211020a8f068bc08b510b12a
:10147000a8f05afe012008bd01210c20a8f05ebc96
:1014800008b510b1a8f050fe012008bd30b50446e3
:1014900085b078b168462bf06df96a46234604adf5
:1014a000144603ccac4218605960224603f108038d
:1014b000f6d1012005b030bd1fb5044648b101a8e2
:1014c0002bf004fd01ab03cb206018686160a060c5
:1014d000012004b010bd000038b50d46044608b91f
:1014e000002038bd0029fbd0002027f0a3f80028f9
:1014f000f6d00023e360044b0120c4e900354ff02f
:10150000ff33a360ede700bf9d130002f8b50e4660
:10151000054608b90020f8bd0029fbd0002027f0bf
:1015200089f804460028f5d040343146204645f07d
:1015300094fc07463146204645f091fc002fe9db3c
:101540000028e7db034bc01ba860c5e9003601207b
:10155000e1e700bfc1130002002908bf3221024b9e
:101560001970024b186070472b51001008c400100e
:1015700070470cb402b07047034b1860034b1960fe
:10158000034b1a60704700bf0cc4001010c4001059
:1015900004c400102de9f04f4ff0010c00244ff06f
:1015a000ff36d0f804e0964504d211f80e80b8f169
:1015b000000f09d18268511e03eb0213002980f24b
:1015c000a8812046bde8f08fb8f13a0f7dd033d81e
:1015d000b8f1220f00f0a58010d8a8f109085ffa31
:1015e00088f8b8f1170f0dd8ac4d0cfa08f818eac6
:1015f000050f07d0456801354560d2e7b8f12c0fdb
:1016000000f02981d0f8048042450ed911f8085025
:101610005db13a2d00f25e811f2d00f246810a2d48
:1016200000f25581082d40f24b81002b40f057818c
:1016300008f1ff354560a4e0b8f17b0f1dd00ad852
:10164000b8f15b0f19d0b8f15d0fdbd1002bd1d011
:101650004ff0020906e0b8f17d0fd3d1002bc9d0bd
:101660004ff001098568013d03eb0518002d2fdac5
:101670000135bfd16ff00104a3e70134002bb9d0cd
:101680008568099faf4265d905f1010ec0f808e0f1
:101690004fea051a03eb051e0025cee90166cef8d8
:1016a0000c50c5686f1c1fbf03eb0519d9f80c500f
:1016b0000135c9f80c50b8f17b0f0cbf012502258c
:1016c00003f80a504568cef804508568013d1ce0d7
:1016d000d8f8047001371ad0d8f808a0baf1ff3f43
:1016e00015d198f800b0cb45c4d10ef1010ec0f869
:1016f0000ca0c8f808e003eb051edef80470013703
:1017000009d0def80870013705d1c56072e7013de8
:10171000a8f11008aae7013d6f1caef1100eecd144
:1017200068e70ef10109c0f80490d0f80480424542
:1017300002d911f8085025b9c0f804e06ff002048e
:101740003fe7222d2dd1e3b18568099faf4204d830
:10175000c0f804e04ff0ff3433e700274ff0030aee
:1017600005f1010e4fea051803eb0515c0f808e076
:10177000c5e90166ef60d0f804e003f808a0c5e908
:10178000019ec56801346f1c3ff434af002b3ff459
:1017900031af03eb051edef80c500135cef80c50ce
:1017a00028e75c2d11d108f1010595420dd2456065
:1017b0004d5d752d2cd86d2d0bd8662d28d85b2d41
:1017c0001ed8222d01d02f2d22d14568013545602c
:1017d000abe76e3d072d1bd801a757f825f000bfda
:1017e0004b17000291170002911700029117000297
:1017f0004b170002911700024b17000297170002c7
:1018000040f241475c3dedb20cfa05f53d42dcd1ba
:10181000c0f804e02ee74ff0040a08f10205456025
:10182000d0f80480424512d911f808507db1a5f1d5
:10183000300bbbf1090f04d925f02005413d052de2
:10184000e6d808f10105baf1010a4560e8d145681a
:10185000013d4560b9e7002b3ff4ccaec5682d01d2
:101860005d5d013d012d7ff6c5ae856805f1ff3850
:1018700003eb051eb8f1000ffff6bcae1ef8105cbe
:10188000013d012d0cd85ef80c5c013508d05ef8e6
:10189000085c013504d1c0f80c80abe61300800071
:1018a00008f1ff38aef1100ee4e7a5f120091f4f53
:1018b0005ffa89f90cfa09f919ea070f7ff4b5ae56
:1018c000203d5e2da4d808f1010545609ae60d2d56
:1018d000f6d1aae605f0df09b9f15d0ff8e78568f2
:1018e000099faf427ff634af002705f101084feaa8
:1018f000051903eb0515c0f80880c5e90166ef601e
:10190000d0f8048003f80970c5e901e84568013d95
:1019100090e653f80c2c013204d053f8082c013215
:101920003ff40caf0139103b48e600bf0110000442
:101930000023c0e901334ff0ff33c360704700005c
:101940002de9f0418046c2b000200d46174626f032
:1019500071fe044618b34ff4847200216846403487
:10196000a8f02ffc6a462946204645f081fa50b37c
:101970002f212846aaf0b1fab8b1854215d0411bf3
:101980002846aaf07bfa0646c8b10146204646f032
:10199000cdfa38b1113005d03046a8f0c5fb6ff054
:1019a000e0000de03046a8f0bffb47f480773b46ef
:1019b0002a464146204646f0b7fb08b1efe7044807
:1019c00042b0bde8f0819df80030112befd0e6e782
:1019d000fcfefffff8b5074600200d461646fff750
:1019e0004bfd0446a0b100223946fff78ffd28b118
:1019f0003246294620462bf099fd38b96ff0e005b4
:101a000000212046fff73cfd2846f8bd0025f7e7fa
:101a1000004df9e7fcfefffff8b5074600200d4634
:101a20001646fff71ffd0446a0b100223946fff716
:101a300053fd28b13246294620462bf07bf838b9b1
:101a40006ff0e00500212046fff710fd2846f8bda5
:101a50000025f7e7004df9e7fcfeffff0fb413b5d3
:101a60000a4b586a23f023fa58b1094c05ab802180
:101a70002046049a0193aaf0d9fd0028bcbf002398
:101a8000237002b0bde8104004b07047fcc50010e0
:101a900014c4001008b5044b586a23f008fa10b1ba
:101aa0000022024b1a7008bdfcc5001014c40010bf
:101ab000021e80f2ed8012f5877f00f0eb8000f3cc
:101ac000918012f5a56f00f0e78059dc894b9a42ae
:101ad00000f0e48001339a4240da1e3b9a4200f063
:101ae000df8001339a422eda12f5af6f00f0da8010
:101af0008149824b82488a4218bf18467047c932d2
:101b00000b2a00f2db80dfe812f0b900b700d90041
:101b1000d900d900d900d900d900d900d900b50021
:101b2000cf00e6320b2a00f2c980dfe812f0af00e6
:101b3000c700c700c700c700ad00c700c700c70087
:101b4000ab00a900bf006f4b9a4200f0b1806b4818
:101b50006d4b12f5aa6f08bf184670476b498a4251
:101b600000f0a88001318a4206da9a4200f0a4808f
:101b7000624b67480a39bee740f0a080654870476d
:101b8000654b9a4200f09c8001339a4217da6f3b12
:101b90009a4200f097806ff497639a4207da653ba8
:101ba0009a4200f091805d49544b5d48a3e712f5dd
:101bb000966f00f08b805b49504b5b489be712f5ba
:101bc000917f00f0858008dc12f57a7f00f082803a
:101bd0004a48564b12f5967fbde74848544b12f5dc
:101be0008c7fb8e712f1bd0f1ada12f1c90f86da4d
:101bf00012f1da0f0dda12f1e60f92da12f1fa0fa2
:101c00006ad012f1f00f69d03c484a4b12f5827f3e
:101c1000a1e73a4b484812f1d20f18bf1846704757
:101c200012f18c0f5cd012f18b0f16da12f1a00fab
:101c300058d012f19f0f09da12f1b40f54d02f4b84
:101c40003e4812f1aa0f18bf184670472b4b3c486c
:101c500012f1960f18bf1846704712f1780f45d051
:101c600012f16e0f44d0254b364812f1820f18bf87
:101c700018467047344870473448704734487047b6
:101c80003448704734487047344870473448704788
:101c90003448704734487047344870473448704778
:101ca0003448704734487047344870473448704768
:101cb0003448704734487047344870470f4870477d
:101cc000334870473348704733487047334870474c
:101cd000334870473348704733487047334870473c
:101ce000334870473348704733487047334870472c
:101cf00033487047b9faffff92faffffbc040c02a9
:101d000066070c02a6faffff65050c02cdfaffff7d
:101d10007d050c020a060c02b4fbffffecfaffff84
:101d2000e6050c0294fbffff40060c024a060c027b
:101d300064060c02bb060c024a070c0240070c02a8
:101d40009c040c027c070c02f0060c02e1060c025b
:101d5000d3060c02b2060c02a0060c0295060c0279
:101d600087060c021bda0c029c050c021f050c02f4
:101d7000f5040c02ca040c02e8040c0200070c0271
:101d8000ac060c0209050c0238050c024e050c02cb
:101d9000dc050c02ad050c02c9050c02f7050c02ae
:101da00028060c0235060c0278060c0255060c02b9
:101db0002c070c020f070c021d070c02ae040c02cc
:101dc00058070c0210b5084b0446586a23f06ff808
:101dd00010b1064803782bb92046bde81040002119
:101de000fff766be10bd00bffcc5001014c4001094
:101df000a0f13003dab2092a01d818467047a0f1e1
:101e00006103052b01d857387047a0f14103052b1a
:101e100094bf37384ff0ff307047102af8b50646a8
:101e20000c461bd900252078fff7e2ff071e15dbc3
:101e30006078fff7ddff031e10db43ea0713052d73
:101e4000735505d102340135062decd1012006e091
:101e5000a278e31c3a2a01d11c46f4e70020f8bd21
:101e6000034b1860034b1960034b1a60704700bfa7
:101e700094c4001098c400109cc40010f0b5164b18
:101e800005461e680f461446abb036b9134b1b68a7
:101e900003b3134b1b7883421cdc23791b0706d446
:101ea0001ef097f82379606143f0080323718eb127
:101eb000dde93023a02102a8aaf0b8fb9f28c4bf07
:101ec0007e238df8a63000233a4600932946234608
:101ed00002a8b0472bb0f0bd94c4001008c4001095
:101ee0002b51001030b585b008ac54f8045bcde937
:101ef00000540394fff7c2ff05b030bd70b4044630
:101f00000d46104619464bb1054b1e6836b10023ed
:101f100022460393b4462b4670bc604770bc7047a2
:101f200098c4001070b51a46134b04461d680e463f
:101f3000aab035b9114b1b68bbb1114b1b7883425a
:101f400013dc2e9ba02102a8aaf070fb9f28c8bf1b
:101f50007e230146c4bf8df8a6309f213db10023ea
:101f60002246009302a83346a8472ab070bd034b0f
:101f700002a81b689847f8e798c4001008c400102e
:101f80002b51001008b410b585b007ac54f8043bd1
:101f900000940394fff7c6ff05b0bde8104001b000
:101fa000704700002de9f04f8846294907460d6823
:101fb000adb0002b3ad035b926490968b1b32649ee
:101fc0000978814232dc00211446dff89090dff876
:101fd00084b08df8ac10d61814f8013b2ca84fea49
:101fe000131c19f80cc0084403f00f034a1c00f836
:101ff000a4cc19f8033002312ca80244a02902f81d
:10200000a43c09d1adb14ff0000a43463a46cdf8a1
:1020100000a003a8a8475146a642ddd131b175b151
:1020200000233a46009303a84346a8472db0bde8d5
:10203000f08fdbf8003003a898472946ece72cab7b
:102040001944044b01f8a45c1b6803a89847ede70a
:1020500098c4001008c400102b510010c0070c02d7
:10206000074b02461b680bb100221847054b186846
:1020700028b1054b1b789a42b4bf0020012070475d
:102080009cc4001008c400102b5100104528dabf72
:102090000a2390fbf3f00620034bd8bf20eae07040
:1020a00053f82000704700bfa4070c0270b50d461e
:1020b000044620b90a201c4a1c49fef791ff16f07d
:1020c00097fca37bdb070bd563680bb1a2689a6012
:1020d000d4e9013282b15360a37b03f0fe03a37302
:1020e00013490b686db1002283b11e7b257bae4284
:1020f0000bd91a465b68f7e70d4a1360ece70c60f2
:1021000007e063b901238b7409e09c60002af6d0d4
:102110005460c4e90132a37b43f00103a373bde81b
:10212000704016f069bc00bf21d40102d1070c0237
:10213000a0c4001010b5044616f05afc094b1a8ac8
:102140005cb1013a92b21a821a8a92b20ab9012299
:102150009a74bde8104016f04fbc013292b21a8258
:10216000f7e700bfa0c4001010b516f041fc044b07
:102170001c8a16f041fca4b2b4fa84f0400910bde8
:10218000a0c400102de9f04f85b04ff000090546be
:1021900016f02efcca4683464b46012049464f4660
:1021a0004e464a46614cd4f8008010b3b8f1000f97
:1021b0001fd098f80d300f2b5ffa83fa15d1d8e9ac
:1021c0000531284698470022d8f8106098f80e107c
:1021d000238a94f812909bb2b3fa83f30020c9b219
:1021e0005b095ffa89f9a274dde7b8f81470bfb231
:1021f000eae75846cde9021316f0fefbdde90213cb
:10220000a27a524502d1a289ba4261d0002284f852
:102210000aa0a781e281002b57d011f0020067d1fc
:10222000434bc6f307481f78424bffb2db68984721
:102230007843f5b2c6f3072700fb08f84743454348
:10224000b4f80cc04fea18413a0c280c88461746df
:102250000546bcf1000f05d0a67ae389022e44d0d2
:10226000032e49d0b9f1000f08d1a388434505d109
:10227000e388bb4202d12389ab4226d0dff8b49079
:102280000023d9f804602a4639464046b0472a4e12
:102290003368b3b1d9f80c30002098474fea0821d1
:1022a0002b023a02b3fbf0f3b2fbf0f2b1fbf0f019
:1022b00000210091c1b2214836680068dbb2d2b279
:1022c000b047a4f80480e780258105b0bde8f08f11
:1022d000002fa0d0e0890544adb2bd4224bfb5fbbc
:1022e000f7f207fb1255e58195e7b3eb5c0fb9d325
:1022f00000252f46a846b5e74fea5c06b3eb5c0f16
:1023000034bff31a9b1b9bb203fb01f803fb02f7dc
:1023100003fb00f5b8fbf6f8b7fbf6f7b5fbf6f5ef
:102320001ffa88f8bfb2adb29ce700bfa0c400108e
:102330002a51001010510010fcc3001000c40010fe
:10234000064b0022194641f8042b5a601a828a80f3
:102350005a81da6001229a74704700bfa0c400104d
:1023600070b5d0e90043204643f31d03002b0ddd7b
:102370005a1050f8226000eb8205b6888e4203d2d4
:102380009b1a281d013bf1e71346efe7001b801065
:1023900070bd000070b51048d0e88f5f15f00105e2
:1023a0000e4e16d11cf0f2f898b110201af0b4f9c4
:1023b000044650b1c0e90055856005738020a7f040
:1023c000abfe10b120232060a360034834601cf0f2
:1023d00017f9306870bd00bfb4c40010b8c4001055
:1023e000f8b50746fff7d6ff037b044673bbb988f1
:1023f000fff7b6ff0546d4e90006b54204da50f807
:1024000025309b888b4224d0a3689e420ddb013689
:10241000002e05ddb100a8f055fe20b90e4814e0ed
:10242000a7f082fe00202060a6602668626806eba6
:1024300085019200a2eb8502081da7f0a8fe0020ee
:1024400046f82570636801336360f8bd6ff0d10012
:10245000fbe76ff0b300f8e7fcfeffff2de9f84360
:1024600007460e469046fff795ff037b0546a3b14e
:1024700077b1d0e9004304eb83094c45234607d0ec
:10248000414618680434b8470028f6d0bde8f88300
:1024900036b16b6800203360f8e76ff0d100f5e7e4
:1024a0003046f3e770b506460c46fff773ff037b33
:1024b00005467bb13146fff753ff6b6898420cda53
:1024c0002b6853f820309a88b24206d144b10020dc
:1024d000236070bd6ff0d100fbe76ff0a900f8e753
:1024e0002046f6e710b50446fff754ff022c05bf5f
:1024f000012303736ff07700002010bd38b5382238
:102500000d4600210446a7f05cfe4ff0ff32002389
:102510002046c4e90f23a56338bd000030b5054649
:102520008db0002026f086f8044618b325f0b8ffd9
:102530002b6c990706d40025204625f0d5ff2846a8
:102540000db030bd294604f1400045f001fb0028e4
:10255000f1da202200230290cde90423aa6b322075
:102560000192064a0649009204aafff7bbfc6ff0ed
:10257000e005e1e76ff0e005e1e700bff1070c02dd
:10258000e9070c02002370b501f14006044601463c
:102590001a4630468eb045f07af800284ff0000514
:1025a00011da2023cde90635a36b029001930f4b7e
:1025b000322000930e492b4606aafff793fc6ff0da
:1025c000e0000eb070bd04232146304605aa0595f3
:1025d00044f0f9ff042807d02023cde90635a36b8a
:1025e00002900193034be3e70598eae710080c0219
:1025f000e9070c022f080c0210b50446236c0846ac
:102600008cb0abb12146403045f0eafa00280dda33
:1026100020220023cde90423a26b02900192054af7
:1026200032200092044904aafff75cfc00232364d3
:102630000cb010bd4e080c02e9070c0238b5054677
:10264000002025f0f7ff044650b125f029ff284669
:102650002146fff7d1ff2046bde8384025f044bfb2
:1026600038bd000030b505468db0002025f0e2fff2
:10267000044610b325f014ff21462846fff7bcff9f
:10268000a96b04f1400045f057fd00280fda811cca
:102690000dd020220023cde90423aa6b02900192e1
:1026a000074a32200092074904aafff71bfc204684
:1026b0000db0bde8304025f017bf0db030bd00bff4
:1026c0006e080c02e9070c02002a70b540f60315eb
:1026d00018bf0125036c044635ea03030e468cb08f
:1026e0001fd0fff789ff2b462146a26b06f1400061
:1026f00045f01afd002813da811c14d02022002393
:10270000cde90423a26b02900192084a3220009284
:10271000074904aafff7e6fb6ff0e0000cb070bdbc
:1027200025640020fae76ff0a900f7e78a080c0299
:10273000e9070c022de9f04705468cb000208946d8
:10274000904625f077ff0746002863d025f0a8fec5
:10275000012239462846fff7b7ff041e1bdb07f1ad
:10276000400a2946504644f07afb061e10da202023
:102770000023aa6bcde904030192284a0296009235
:102780003220274904aafff7adfb6ff0e00402e016
:10279000032e07dc234c384625f0a6fe20460cb05d
:1027a000bde8f087eb6b002b09da39462846fff7c6
:1027b000e9fe041eefdb17d1042eebd1ec63ea6bcc
:1027c00000239045a8bf904629465046b21a44f0cf
:1027d0005eff00280cda20210023aa6bcde9041348
:1027e00001920290104acae7f31ea342e6dcd1e749
:1027f00043464a462946504644f0e5fe8045044695
:10280000c9d020220023cde90423aa6b02900192b3
:10281000064ab4e76ff0e004c0e700bfa9080c0265
:10282000e9070c02e8feffff10080c022f080c025b
:102830002de9f04705468eb000208946164625f062
:10284000f9fe804600287fd025f02afe002241466e
:102850002846fff739ff041e18db08f1400a294615
:10286000504644f0fcfa071e17da4ff0200c002304
:10287000aa6bcde906c30192354a02970092322035
:10288000344906aafff72efb6ff0e004404625f01e
:102890002bfe20460eb0bde8f087032f0fdc002290
:1028a0002946504644f00cff002828da2026002351
:1028b000aa6bcde9066301920290274adee7eb6b33
:1028c000002b06da41462846fff75cfe041edddbde
:1028d000ec63eb6bb342e2d13744b7f5805fdedceb
:1028e00033464a462946504644f0b2fc86420446e6
:1028f000ccd0202200230290cde906231ee0002345
:1029000029461a46504644f0c2fe002808da202420
:102910000023aa6bcde90643019202900f4aade76e
:1029200004232946504605aa059644f091fc042844
:1029300008d020210023cde906130290aa6b019252
:10294000074a9be7ee63cbe76ff0e004a1e700bf27
:10295000a9080c02e9070c02c8080c0210080c02b6
:10296000eb080c027047704770470000074b1a785d
:1029700012b10021064a11705a7812b10121054a9c
:1029800011709b780bb108f099bf7047bcc4001060
:1029900002c9001000c90010fff7e8bf10b5c368f6
:1029a00004460bb9a6f066fe03690430984700217f
:1029b000a0616069bde8104022f0b2bb10b508f01c
:1029c000a5ff124b124c1b780246b3fa83f35b0946
:1029d000a070237080b10120002205216070104694
:1029e00004f0bcf908f08cffbde8104000231a4643
:1029f0001946184604f04eba014604f089f802461a
:102a00000028e8d1014604f0d2f8e5e702c9001039
:102a1000bcc40010012af8b5064603d10b68036058
:102a20000020f8bd022a08d0032af9d10068002846
:102a3000f6d01c2119f078fef2e71c200c6819f082
:102a40006bfe074630b105460fcc0fc594e8070072
:102a500085e807003760e3e7012a70b5054603d132
:102a60000b680360002070bd022a08d0032af9d148
:102a700000680028f6d0102119f056fef2e7102069
:102a80000e6819f049fe044618b196e80f0084e874
:102a90000f002c60e6e7000070b5037d04460e468b
:102aa000154683b10368db6873b19a88012a06d0a2
:102ab0009b68f9e79b683bb19a88012afad19a8909
:102ac000b242f7d19d7370bd002110200bf090fd34
:102ad00008b92075f7e7054b03600123838023695c
:102ae0008681836085732061ede700bf10000300dd
:102af00038b5037d04460d466bb10368db6823b12e
:102b00009a88042a11d09b68f9e7002110200bf065
:102b10006ffd08b9207538bd054b03600423838021
:102b20002369c0e902352061f5e7dd60f3e700bf06
:102b30001000030010b58368044613b10322014658
:102b40009847204610bd000010b50446034b40f8de
:102b5000043bfff7efff204610bd00bf740e0c02d0
:102b600010b50446fff7f0ff2046142119f0dcfdf4
:102b7000204610bd10b5074b04460360406918b1ec
:102b800022f0a9fa002363612046fff7ddff20460b
:102b900010bd00bf880e0c0210b50446fff7eaff17
:102ba0002046182119f0c0fd204610bd10b504467e
:102bb000024b0360fff7deff204610bd9c0e0c02a7
:102bc00010b50446fff7f2ff20461c2119f0acfdba
:102bd000204610bd38b50446006928b1856800213b
:102be0000bf018fd2846f8e7204638bd002330b525
:102bf00087b0cde90233049301238df814301023fc
:102c0000adf80430032301ad00280c460095adf863
:102c100006308df8083005dd4ff47a71414368467f
:102c2000fff766ffa30704d401220a216846fff7d5
:102c300033ff0120fff797fe00222846114619f0c6
:102c400017fa04466846fff7c5ff204607b030bdb7
:102c50002de9f0470e4698461021002388b0cde9b3
:102c600004330693adf80c10012303211746109a84
:102c70000df10c09002a0546cdf808908df81c309e
:102c8000adf80e108df8103005dd4ff47a7102a802
:102c90005143fff72dffb5b1beb1002f3cd0b8f1c5
:102ca000000f39d0002407eb080ab4420dd0444588
:102cb00035f8141034bf3a5d1af8012c02a8fff75a
:102cc000ebfe0134f1e72c46ede700270120fff78a
:102cd0004afe3a46484601a9019719f0c9f9041e6f
:102ce00011dbfff741fe0198c0b183883c46012b00
:102cf00007d1b4420ed035f81430828901349a429b
:102d0000f7d1a7f011fa02a8fff764ff204608b038
:102d1000bde8f0870024f4e7014cf4e70446f2e74d
:102d2000f2feffff73b506461c200d4619f0f4fcb9
:102d3000044628b3144b03600023c360ab683bb167
:102d40000222294604309847eb682361ab68e360b0
:102d5000002220460d4b0121236040f8142f22f061
:102d6000aff90b4b30462360336801945b6801a9cf
:102d70009847054620b9236820469b6898472c460b
:102d8000204602b070bd00bf740e0c02880e0c020b
:102d90009c0e0c02f0b51f463c4b164693f82c20b7
:102da00005460c4689b0f2b1586a22f080f8d0b9d5
:102db0000690102019f0b0fc18b1c0e9014605706a
:102dc000c760334b04900793324b304804a90693f5
:102dd000fff7a8ff0546b8b9044604a8fff7aafe06
:102de000204609b0f0bd02f01dfbc8b9f34313f053
:102df000010300d195bbfff7e1fd012d3ed0022d6f
:102e00003cd0bdb10024ebe700224ff0ff31406918
:102e100022f066f92b6828469b68ac699847dce786
:102e200016f00403e2d11a460621012000940bf0ab
:102e30006bf9dbe7002cd3d0e317cde90443012184
:102e40002b46154a009504a8cde906551df010fa49
:102e500004460028c4d0fff789fdc1e7012d0dd03d
:102e6000022dcfd11a4618460521039303f076ffb1
:102e7000039b1a461946184604f00cf831462046c2
:102e800009b0bde8f040fff7b1be00bffcc50010bf
:102e90001d2e0002d929000219290002006841688c
:102ea000d0e902230078fff775bf2de9f0411f46f6
:102eb000002304460d46164601211a46184603f023
:102ec00094fe3b46324629462046bde8f041fff7d6
:102ed00061bf00002de9f04f9846504b174693f81c
:102ee0002c2087b00546dde910940e4622b3586abf
:102ef00021f0ddff00bb04901c2019f00dfc38b15f
:102f0000129bc0e90056c0e90278c0e904948361cd
:102f1000434b02900593434b404802a90493fff7ab
:102f200001ff0446002853d1054602a8fff702fe20
:102f3000284607b0bde8f08f02f074fa82460028f8
:102f400052d1e44314f0010403d0fff737fd4ff0f2
:102f5000000a00210846fff7edf8e720fef794f994
:102f600043463a4631462846cdf80090fff770feba
:102f7000002105460120fff7ddf8e720fef760f9a4
:102f80000cb1fff7f3fc08f0e7fc0446002008f062
:102f9000effc0646b8bb013ce4b2012c33d808f084
:102fa000b5fc80b330461df007f84ef660260446a7
:102fb00000201df001f8001b61f10001b04271f129
:102fc00000031ed202f02efad8b902f03bfaefe766
:102fd00000224ff0ff31406922f082f8236820463a
:102fe0009b68a5699847a0e714f0040ba9d15b463c
:102ff0005a4606210120cdf800900bf085f8da46fc
:103000009fe702f00ffabaf1000f91d006f070fbc3
:10301000002304211a4610f0fcf889e7fcc50010d3
:10302000a92f0002952900021fb500688369029349
:103030004369019303690093d0e90223d0e90001b9
:10304000fff748ff05b05df804fb2de9f0471f4688
:10305000dde90889002304460d461646ddf828a060
:103060001a460121184603f0c0fd3b463246294668
:103070002046cde9099acdf82080bde8f047fff75a
:1030800029bf70b51d46002388b00e461446adf822
:1030900016001a460121184603f0a7fd0c9b009468
:1030a000cde9015301230df11f0219460df1160060
:1030b0008df81f60fff7c9ff08b070bd38b5154621
:1030c000d0e902239342044607d2d21a4068aa42aa
:1030d00028bf2a461844a7f04df8e26801202a4488
:1030e000e26038bd13b5044608460191fdf76afe5b
:1030f00002462046236801991b6802b0bde81040d3
:103100001847000004281fb5034614460cd14ff69b
:10311000ff7345f61b210920002a08bf194604b099
:10312000bde8104016f048b801280ed100233c221b
:103130000093112312481349002c18bf014612486e
:10314000006802f031fd04b010bd09280ad1002347
:103150000b480c490093002c18bf014611233c2258
:103160000a48ede70028eed1002aecd00246cde96e
:103170000100009000214ff4007003f04df9e2e7e8
:10318000a80e0c0211350c022c5100103051001009
:1031900009280a4608b50dd8084b195c914203d19d
:1031a000042801d0082803d1195c1a54fff7aaff9c
:1031b000002001e04ff0ff3008bd00bf3d5100107e
:1031c000092838b50c4613d8a9b104280b4d0cd1e9
:1031d000092015f0fbff45f61b2380b2c31a5842a5
:1031e000584120702871002038bd2b5c0b70fae725
:1031f0004ff0ff30f8e70846f6e700bf3d510010fa
:1032000037b500220df107010546fff7d9ff044647
:1032100028b99df8072028461146fff773ff20467e
:1032200003b030bd014b1860704700bfc8c4001028
:1032300038b50b4b45681c6864b100f108010022e9
:103240002846a047044618b1064928460ff0c8fa98
:10325000204638bd044928460ff0c2fa0349f4e776
:10326000c8c40010ad0e0c02db0e0c02110f0c02d4
:103270000c4a0d4b00b51a601c2389b00021adf833
:1032800004301423029001a8cde90311cde9051102
:10329000adf806100791adf80c30fff7c9ff09b083
:1032a0005df804fbfd4b0002c8c4001010b50f4bc5
:1032b00004461b68834208d1002301211a461846a0
:1032c00003f093fc00200ff039fc00221146104659
:1032d00003f0dbfc024640b9054b1b68a34204d156
:1032e000bde81040014603f027be10bd3451001068
:1032f0003851001030b50d4b05469b7885b003f072
:10330000ff0483b9224601210220fff741ff084b49
:1033100022461d704ff4806023460021cde9014410
:10332000009403f079f805b030bd00bf3d510010a6
:103330003c51001013b50024022022460df1070174
:103340008df80740fff73cff9df8070060b122466b
:1033500003200df107018df80740fff731ff9df8bd
:103360000700001b18bf012002b010bd07b5fff712
:10337000e1ffa0b10b4b1a7802f0ff0342b100232a
:1033800002201a46194603b05df804ebfff78dbd25
:10339000054900931a460120097808f0effa03b0b6
:1033a0005df804fb45cc00103c510010f0b585b031
:1033b000fff7c0ff48b3164d2b7833bb01222a70ac
:1033c000144a4ff400600021cde9013300921a46ff
:1033d00003f022f81cf0fdfd47f22f5704460e4e75
:1033e000fff7a8ff30b90020287005b0bde8f04015
:1033f000fff7bcbf1cf0edfd001bb842f3d802f094
:1034000021f8304603f01affeae705b0f0bd00bf2f
:10341000ccc40010ed320002fcc5001037b5837a31
:1034200004460d46ebb91df0a9fb636818442389d7
:10343000206113b91df0aefb2081e36813b91df0c4
:10344000a3fbe06015f0010f0cbf0025042504f07c
:103450000ffc0023e1681a46009504f017ff03b043
:1034600030bd0148fbe700bfe2faffff2de9f04164
:103470001646ca0788b038d511f0020f0cbf0024d9
:10348000042404f0f5fb214604f078fd14f008054f
:10349000074626d106b34ff0ff082946424630467c
:1034a000a6f08ffe124b134904a8cde90436cde9ee
:1034b0000685fff717fe3b460c210f4a01a8cde910
:1034c00001550395a7f0b4fe01a904a8fff70afe71
:1034d0000a4904a8fff706fe630702d44620fff757
:1034e00009ff384608b0bde8f0810824c9e700bfed
:1034f000600f0c024e0f0c028c1b0c02540f0c02be
:1035000030b50446002585b0039104f0b1fb626834
:1035100023690399d31a0095228904f06ffd05b041
:1035200030bdc1684a69506803681b6818470000cd
:1035300038b50c461546c8683ab11146a7f0c2fd29
:1035400038b1e0600020256138bda6f0edfde560f2
:10355000f8e70148f8e700bffcfeffff10b591f85f
:1035600043300c46db0748680cd500210bf052f8bd
:1035700094f8433023f0010384f843300023c4e976
:10358000013310bda6f0d0fdf8e708b508b108f08a
:10359000b7f9002301211a46184603f026fbbde8bf
:1035a000084001f017b910b5c468a068a6f0b4fdd2
:1035b000606015f01dfa94f842202ab963687bb167
:1035c000022384f84230144615f016fa6cb1606894
:1035d000a6f0aafd2046bde8104000210bf01ab865
:1035e000012284f842201c46eee710bd136810b596
:1035f000032b17d90b685c1c0c6018700b685c1ce3
:103600000c60040a1c700b685c1c0c60040c1c70c1
:103610000b68000e5c1c0c60187001201368043be2
:10362000136010bd0020fce773b58b6804460d469f
:1036300000931bb90026304602b070bdcb880068ed
:10364000694601aa0193fff7d1ff06460028f1d091
:10365000019b012beed9009aa389511c0091137094
:10366000009a1b0a511c00911370019b2268023bb7
:10367000910701930ed5012bdcd9009ae389511ce7
:1036800000911370009a1b0a511c00911370019b4a
:10369000023b019323685a070ed423681b0706d503
:1036a0006946606801aafff7a1ff0028c2d0aa6896
:1036b000009b9b1aeb80bee76946a06801aafff752
:1036c00095ff0028e9d1b5e738b50c4b41600360a0
:1036d0000023c0e902330361044615f089f9054669
:1036e0002146074820f0fafc2146064820f002fd5a
:1036f000284615f081f9204638bd00bfb80f0c02ee
:10370000f33a0002153b00022de9ff41cb88064643
:103710003f2b0f4640f29380886860b1338a032bb9
:103720000cd9002301220293cde900230323039344
:103730006846fff779ff04b0bde8f081002144201e
:103740000af056ff044638b90123cde900300423be
:10375000029003933946ebe718230380bb884ff0b0
:10376000000843807b88c0e9038883606ff06303af
:10377000c0e90c8846614062c0f83880c363738a30
:1037800001339bb273828568a0f8403080f8438093
:10379000002d35d12b4b00f11801c3612a4803f0ed
:1037a00079fd032384f8423063886560462b0ed090
:1037b00010d8322b07d004d8283b012b03d9002581
:1037c00008e03c2bfbd10120fff7dffef7e728469e
:1037d000fff7dbfe0023a362b368e36203b19c62e0
:1037e000338ab460013333820023cde90133b4f866
:1037f0004030adf80c50adf80e3003230093a9e72c
:10380000402d0fd8414628460af0f2fe606048b1cc
:1038100094f8433043f0010384f84330022384f8e2
:103820004230cce7094b0848e36104f1180103f08a
:1038300031fd00230225636084f84230cae700208e
:1038400079e700bfa334000274d0001027350002ce
:1038500070b58b8884685cb1b4f840209a4209d076
:10386000e46af8e7d8b9636833448b60012070bd1f
:103870000020fce794f84230022bf9d1cd88a66bea
:10388000a36872199a42f3d8402d8868ead80028b4
:10389000edd0636801462a469819a6f06bfca26b2e
:1038a000a36815449d42a563e0d1064b0648e36139
:1038b00004f1180103f0eefc0023a363032384f852
:1038c0004230d3e7a334000274d00010f8b50646a6
:1038d0008b8884684cb1b4f840209a4207d0e46adf
:1038e000f8e7e3683b448b6016e0002019e094f8a9
:1038f0004230042bf9d1cd88002df6d0a76b236977
:103900007a199a42f1d8402debd8886848b1e1681d
:103910002a463944a6f02efca06b2844a06301205f
:10392000f460f8bdf0b54b780c46502b85b00cd147
:1039300091f90030002b42dacb8833b1886880b32c
:103940008a88142a03d01e2a2dd0002029e01021b5
:10395000684618f0d5fb1028f7d8e3884500b3eb8c
:10396000400ff2d36b46a2685619b24217d01f46d9
:1039700019780133090901f13000392888bf01f1b4
:10398000370002f8020b397801f00f0101f1300025
:10399000392888bf01f1370002f8010ce5e7e5801e
:1039a000012005b0f0bd092bcfd90d4b1a6802607c
:1039b0005a681b89426003810a23cb80f0e78b8819
:1039c000282b06d0b3f5977fbfd10120fff7ddfd8f
:1039d000e6e700228c20114615f064f9e0e700bf0d
:1039e000a30f0c0210b5cb6a0c460bb18a6a9a621f
:1039f000d4e90a2362b1d362038a013b038294f8bb
:103a000042300bb1032b05d1042384f8423010bda2
:103a10008360f1e7606840b194f84330db070dd56f
:103a200000210af0f7fd00236360e36833b9216bde
:103a300021b92046bde810400af0ecbd044b04f16a
:103a40001801e3610348bde8104003f023bc00bf48
:103a5000d53b000274d000101fb5cb880c463f2b1d
:103a600038d98b68002b37d08b88816829b1b1f8a1
:103a700040209a4201d0c96af8e700230122cde92b
:103a80000233cde9002319b391f84230042b0dd84d
:103a9000dfe803f003070c0312000223adf80c303b
:103aa00004e00423adf80c30fff79cff2146684684
:103ab000fff7bafd04b010bdcb6b0193092300934f
:103ac0000b691bb102930d230093efe7c160ede793
:103ad0000523e3e70020ede71846ebe77fb5cb8849
:103ae00004463f2b0d4615d98868a0b18b884bb989
:103af0006ff08b06a368e3b1de632046a168fff791
:103b000071fff7e7a16841b1b1f840209a420ad0ad
:103b1000c96af8e7002004b070bd01230291cde925
:103b2000003105230ae06ff08b032046cb63fff7db
:103b300059ff00230122cde900230293294668465c
:103b40000393fff771fde6e74b78013b042b0ed89a
:103b5000dfe803f0030507090b00fff7d5bdfff70a
:103b60007bbffff775befff7b1befff7b7bf002001
:103b7000704708b503465a780846013a0e2a194696
:103b800005d8fff7e1ff80f00100c0b208bdfff7e4
:103b9000c9fef8e7012838b50c460bd0022815d12c
:103ba0006ff09505a3689bb1dd632046a168fff720
:103bb00019fff7e7c96849b18a6b0b699a4205d1c9
:103bc00000252046cd63fff70dffe560002038bdde
:103bd000e360fbe738b54b6805460c4613b1036854
:103be0005b689847e3682bb12b6800222146284682
:103bf0001b689847236b13b1616be06b98472046b5
:103c0000bde8384000210af005bd2de9f0411f460e
:103c10004b6805460c461646ddf8188013b103685c
:103c20005b689847c4e90c7814f0e2fe94f84230df
:103c3000032b01bf0423e66384f84230002414f010
:103c4000dbfe2cb121462846bde8f041fff7c2bf9c
:103c5000bde8f081c1684869fff7bcbf03681b6815
:103c60001847000007b50022044bcde900021146b9
:103c7000104604f0fffe03b05df804fbdd3b0002dc
:103c800008b54ff47a7019f008fcbde808400ef052
:103c90006dbf08b54ff47a7019f0fffbbde808401e
:103ca00000200ef04bbf10b5c36804460bb9a5f059
:103cb000e1fc03690430984723682046bde81040c2
:103cc0009b68184708b54ff47a7019f0e6fbbde819
:103cd000084000200ef04dbf08b54ff47a7019f07f
:103ce000dcfbbde8084000200ef012bf37b5446988
:103cf00025680093ad6813460a4601462046a8474a
:103d000003b030bd012a38b5044602d10b682360e8
:103d100003e0022a03d0032a0dd0002038bd0c2076
:103d20000d6818f0f9fc03460028f0d095e807006c
:103d300083e80700ebe700680028eed00c2118f0bc
:103d4000f3fceae7012a034602d101600020704734
:103d5000022a04bfd1e90001c3e90001f6e700002f
:103d600010b50446034b40f8043bfef7e3fe204643
:103d700010bd00bfec0f0c0210b50446fff7f0ffba
:103d80002046142118f0d0fc204610bd10b5044682
:103d9000024b0360fff7e4ff204610bd00100c0249
:103da00010b50446fff7f2ff2046142118f0bcfcc2
:103db000204610bd10b50446074b214640f8043b91
:103dc000fff782fc214604f118000bf05bfa002398
:103dd0002046c4f8f43010bd14100c0210b504468f
:103de00007f0bafd042805d104f11800bde8104021
:103df0000bf02abc092015f097f80028f4d0002019
:103e000010bd18300cf02ebc00487047d0c4001014
:103e1000024bc3f8f4000020704700bfd0c400106c
:103e200010b443690a4619680c68014618462346cf
:103e30005df8044b18470146406903685b68184702
:103e4000fff754bff0b5354e074696f82c300d46b7
:103e5000144687b0002b51d0706a21f028f8002852
:103e60004cd104900c2018f057fc10b1c0e901545b
:103e700007702b4b029005932a4b1c20049318f0db
:103e80004bfc0446002832d0274b03600023c3605c
:103e9000049b3bb1022202a904309847059b236191
:103ea000049be36000252046204b2a462360012125
:103eb00040f8145f21f004f91d4b01a92360f26959
:103ec0002b46306b019421f050f8014650b9706ace
:103ed00008b121f019f800224ff0ff31606921f09c
:103ee000fff8a569236820469b68984700e00546cf
:103ef00002a8fef71ffe284607b0f0bd0d4c84f85f
:103f0000fc70d4f8f80028b18368c4f8f830a6f043
:103f10000bf9f6e7c4f8f8500546ece7fcc50010cd
:103f2000b93e0002853c0002740e0c02880e0c02a1
:103f30009c0e0c02d0c4001003681878d3e901125b
:103f4000fff780bf73b5064614200d4618f0e4fb5a
:103f50000446d0b10e4b03600023c360ab683bb195
:103f60000222294604309847eb682361ab68e3607e
:103f7000084b30462360336801945b6801a9984779
:103f800018b9236820469b68984702b070bd00bfef
:103f9000ec0f0c0200100c027fb5144e044696f88c
:103fa0002c300d4693b1706a20f081ff70b9104b30
:103fb000694603930f4b30460293cde90054fff757
:103fc000c1ff6846fef7b6fd04b070bdd4f8f4300a
:103fd00023b90a20084a0949fdf702f82846d4f80f
:103fe000f43004b0bde87040184700bfc4cb0010e7
:103ff000ed430002c53c000221d40102c40f0c02b3
:10400000f0b50c46d0f8f83085b0002b00f02082d7
:1040100099886288914200f00d829b68f5e7638879
:10402000d32b00f2bf80c72b25d8322b00f055814f
:1040300000f2a280012b00f06e81143b9ab2152a87
:1040400068d9d0f8f430002b00f0a780214605b0e5
:10405000bde8f040fff7a0bf6ff4fa7213442046aa
:10406000052b00f2d281dfe813f0d301d601d9018c
:10407000dc01df01e201c83b0b2be2d801a252f8c0
:1040800023f000bff7420002ff420002c33f0002dc
:10409000c33f0002c33f0002c33f0002c33f000210
:1040a000c33f0002c33f0002c33f000207430002b8
:1040b0000f430002463b142bc3d801a252f823f051
:1040c0006142000271420002774200027f42000218
:1040d000874200028f420002c33f0002c33f00023a
:1040e000c33f0002c33f0002c33f0002c33f0002c0
:1040f000c33f0002c33f0002c33f0002c33f0002b0
:10410000c33f0002c33f0002c33f0002c33f00029f
:104110009f420002152b94d801a252f823f000bf51
:104120000f4200021d420002c33f0002c33f0002d3
:10413000c33f0002c33f0002c33f0002c33f00026f
:10414000c33f0002c33f0002254200022d4200028d
:10415000354200023d42000245420002c33f0002d8
:10416000c33f0002c33f0002c33f0002c33f00023f
:104170004d420002554200025a2b07d8452b99d8d0
:104180003c2b7ff45eaf0023b34aa1e0642b7ff4a5
:1041900058afa368002b00f0c68000236ff07701b2
:1041a0001a464fe1b3f5967f00f023814cd8e72bf8
:1041b00022d8db2b7ff645afdc3b0b2b3ff641af24
:1041c00001a252f823f000bf174300021f43000270
:1041d000274300022f430002c33f0002c33f0002f7
:1041e000c33f0002c33f0002c33f0002c33f0002bf
:1041f000374300023f430002f03b9ab20d2a3ff6dc
:1042000020af0d2b3ff61daf01a252f823f000bfe7
:1042100047430002c33f0002c33f0002c33f000206
:10422000c33f0002c33f0002c33f0002c33f00027e
:10423000c33f0002c33f00024f4300025743000246
:10424000634300026b430002b3f5fd7f3ff6f9ae16
:10425000b3f5fa7fbff400afb3f5c87f00f0d180ab
:104260000cd840f22d12934200f0c780b3f5977f2f
:104270007ff4e7ae20460cf006fd0be040f2911211
:1042800093427ff4deae20460cf026fc02e020468e
:104290000cf060fd002301461a46d3e020460cf0e6
:1042a00091fdf7e720460cf0a5fdf3e720460cf062
:1042b000b7fdefe720460cf009feebe720460cf0d7
:1042c0007dfee7e720460cf097fee3e70023634a14
:1042d0001946b7e00023624afae70023614af7e78c
:1042e00000221146104602f027fe00231a46efe78f
:1042f00000220121f6e720460cf02efecae72046f8
:104300000cf03cfec6e720460cf03bfec2e7204620
:104310000cf03afebee720460cf094febae72046c9
:104320000df066fdb6e780264f4f606932460368a0
:1043300021461b689847054640b100221146204699
:10434000fff76efd002329461a467be0e36801462d
:1043500003906846cde900730296fff783fc0022c4
:1043600005460028ead1039b9e4202d203eb1316b6
:10437000dbe72361e6e720460cf0b6fd8ae720463e
:104380000cf0c8fd86e720460cf06bfe82e7204665
:104390000cf06afe7ee720460cf069fe7ae72046c4
:1043a0000cf068fe76e720460cf067fe72e72046c8
:1043b0000cf066fe6ee720460cf0befd6ae7204674
:1043c0000cf0c2fd66e720460cf05dfe62e7204679
:1043d0000df026fc5ee7204605b0bde8f0400df08c
:1043e00099bc20460df0c6fc54e720460df0c8fcf1
:1043f00050e720460cf012fc4ce720460cf03efc47
:1044000048e720460cf048fb44e70df077f841e719
:104410000cf03aff3ee70cf0a1ff3be70cf0d4ffb5
:1044200038e70cf0f5ff35e70cf0feff32e70df052
:10443000cff92fe79b79022b7ff4f1ad00236ff0ca
:1044400081011a46204605b0bde8f040fff74ebc9a
:1044500090f8fc30efe700bf453c0002013c000251
:10446000593c0002133c0002600f0c02d0e900101e
:10447000fff792bd0148fff79dbc00bfd0c40010fc
:104480000023202200b58bb0cde90223054a01208c
:104490000092054902aafdf725fd4ff0ff300bb051
:1044a0005df804fb1f100c0218100c02f0b500247c
:1044b00020274ff4837605460e4bc5b0009302aa21
:1044c00023461e200c49cde90274fdf70bfd324650
:1044d000214602a8a5f075fe3a4621462846a5f0d9
:1044e00070fe23462246314602a804f0b5fb45b0d3
:1044f000f0bd00bf7b100c0218100c022de9f0413a
:10450000ceb04ff4837204460e460ca80021a5f0ed
:1045100058fe00234ff483711a460ca804f0befb2a
:10452000b0f5837f2dd1bdf83030b3f5837f28d12e
:1045300080213046149d14f053fc854234d0002570
:10454000202780213046ddf85080cde9047514f035
:1045500047fc214bcde90180009304aa2b46322071
:104560001e49fdf7bffc9df83530322001931c4bee
:104570001a49009304aa2b46cde90475fdf7b2fc55
:104580000ae020210023174acde9041300922820d5
:10459000124904aafdf7a6fc2046fff787ff4ff05b
:1045a000ff304eb0bde8f0819df83530002bc6d00d
:1045b0000dad0fcd0fc495e80700002384e8070078
:1045c0002022cde90423084a1e200092034904aab0
:1045d000fdf788fce3e700bfc7100c0218100c02bf
:1045e000ec100c0293100c02ff100c0210b50446e4
:1045f0000846802114f0f4fbe061002010bd0000ab
:10460000f0b50020b3b003f09bfa032014f08cfc4b
:104610000446002837d05f4b1d888022002112a855
:10462000a5f0cffd12a81cf0e3fb9df84830012b4c
:1046300016d920220023cde90a23574a28200092c8
:1046400056490aaafdf74efc2cb1554b55491a683c
:1046500012a8a5f08ffd544a136843f004031360b9
:104660009df8482020218ab1012a4ff0000360d034
:1046700001924e4acde90a130092282047490aaa1e
:10468000fdf730fc1fe041f23365c6e7ddf84a3044
:10469000cde90a12bdf88a101e200791d9b2069101
:1046a000c3f307210591c3f307411b0e03930df1db
:1046b0004a03cde901233e4b049100933749134649
:1046c0000aaafdf70ffc4ff6fd71bdf88a20531eb4
:1046d0009bb28b4202d81cb1aa4201d0adf88a50dd
:1046e00012a93448fff70aff002c14bf112006203e
:1046f000304a12a902f0a6ff0646002842d14ff424
:10470000a06512a92b48fff771ff09a8099625f0ab
:104710009dfa099cdcb1606848b10aa90a9625f0a7
:10472000cbfe20b90a9b13b19d4228bf1d462468c9
:10473000f0e7cde90a130df14a01cde901211e4a46
:104740001e20009215490aaafdf7ccfbbbe7099889
:1047500025f0a8fab5f5a06f184f16d02023cde9a3
:104760000a34174b803d00930aaa23461e200b49aa
:104770000195fdf7b7fb23462a46009407213868c8
:104780000ef0e7fc304633b0f0bd234622460094dd
:10479000f4e700bf5051001036110c0218100c0243
:1047a00024090c020b090c0290ca0010cc110c0257
:1047b00062110c02d4c50010a4110c0298ca00109a
:1047c00008120c0203f0bcb908b5002003f0faf996
:1047d000c0b208bd0122014b1a707047d0c500104d
:1047e00013b50f4b04461b7823b102b0bde810404f
:1047f000fff746be0b4b01911b78002bf5d1fff75d
:10480000e3ff0028f1d1084b1b7803f0ff02002bd7
:10481000ebd12046019902b0bde8104003f02cb95d
:1048200001c9001002c90010d0c50010fff7d8bfa1
:1048300013b50f4b04461b7823b102b0bde81040fe
:10484000fff71ebe0b4b01911b78002bf5d1fff734
:10485000bbff0028f1d1084b1b7803f0ff02002baf
:10486000ebd12046019902b0bde8104003f030b909
:1048700001c9001002c90010d0c50010fff7d8bf51
:1048800008b5002003f088f910f1780f08bf002068
:1048900008bd002003f092b9f0b5022806460d4687
:1048a00014468db005d00a2834d01f4c20460db0d8
:1048b000f0bd202000231d4fcde904033a68cde967
:1048c00001211b4a009201201a4904aafdf70afba4
:1048d0003d6000f0a7fd10b914f00104e6d0164bbe
:1048e00000245b78b342e1d12023cde90434134b9b
:1048f00004aa0093012023460e49fdf7f3fa08228b
:1049000002232946cde904232046234604aa00f0c9
:104910007ffecbe720210023094fcde904133a683d
:10492000cde90125074acde7f2feffff485100100f
:1049300030120c0218100c02d4c5001093120c0295
:104940004c51001061120c0219b1022803d00a2840
:1049500006d004487047044b1b6800200b6070476a
:10496000024bf9e7f2feffff485100104c510010d6
:1049700003689b6818470eb403b503ab53f8042bc8
:10498000002101930df054ff02b05df804eb03b079
:1049900070472de9f04106460d4690461bf019fb85
:1049a00007461bf016fbc01b40450ed83468236831
:1049b00020461b6998470028f3d0236820465b698e
:1049c000984728700020bde8f0814ff0ff30fae7eb
:1049d0002de9f04f16461a46002385b00f46336086
:1049e0000df10f0101928246fff7d3ff019a0446b1
:1049f00028b14ff0ff34204605b0bde8f08f9df898
:104a00000f50182d13d008d8022d20d0042df2d02d
:104a1000012deed14ff080081be005f0df03412ba4
:104a200035d0202d14bf4ff0ff340224e3e7504669
:104a30000df10f01fff7adff04460028d9d19df815
:104a40000f30182bd5d14ff0ff333360d3e74ff43d
:104a50008068b94609f8015b012508f1040b5d4542
:104a60000cd8494650460192fff793ff09f101091e
:104a70000028bed10135019aadb2f0e7bb787a7853
:104a8000db43dbb29a42b4d1c6f80080b3e701241d
:104a9000b1e738b50d46002102f58070033313f8f5
:104aa000014b2cb1b1f5807f02d054540131f6e7af
:104ab00000245454ff32195d202905d0102c03d056
:104ac000013402f8011ff6e700210a220155a7f080
:104ad00027fb4ff48063e8602b8138bdf8b51d4695
:104ae000531c04460cd08ab1d0f818644f78f3b246
:104af0009f4213d000681521fff73aff012004e020
:104b000000680621fff734ff0020f8bd0068062189
:104b1000fff72eff0120c4f81404f6e786bbcb781c
:104b200003b30b46069a2946fff7b3ff32463146d8
:104b30002846fef773fc50b118212068fff718ffd4
:104b400020681821fff714ff4ff0ff30dde72b69d5
:104b500006216b602068fff70bff43212068fff7f9
:104b600007ff04e00123c0f81434c0f8103401201a
:104b7000d4f81834c4f820040133c4f81834c4e756
:104b80002a81284600220331fef7bafc50b11821d1
:104b90002068fff7edfe20681821fff7e9fe6ff0af
:104ba0000100b2e76b682a89062113446b60d5e7e0
:104bb0002de9ff411746044600250e464ff4887242
:104bc00000213846a5f0fdfa04f10808c4f8105495
:104bd000c4f81c54c4f82054c4f81854c4f814542d
:104be00041462046636803aafff7f2fe012810d071
:104bf000022819d030bbc4f81c0433464146204675
:104c0000039a0097fff76aff002811dc04b0bde8a3
:104c1000f08118212068fff7abfe20681821fff70c
:104c2000a7fe6ff00200f1e706212068fff7a0fe63
:104c3000d4f81434002bd3d0d4f81034002bcbd0bc
:104c4000f068e3e7d4f82034002b08dbd4f81c34f8
:104c5000432101332068c4f81c34fff789fed4f8df
:104c60001c34052be4dd18212068fff781fe206845
:104c70001821fff77dfe0020c8e70000f0b50446cc
:104c8000c7b040f224400f4617f046fd054618b164
:104c900041f28833046043603946284602aafff790
:104ca00087ff061e48dd002201213846fef7defba5
:104cb000021e31db06212868fff75afe20462a49ea
:104cc0000df08efd204629490df077fd204602a902
:104cd0000df073fd204626490df082fd2046254942
:104ce0000df06bfd0a22314620460df083fd22496e
:104cf00020460df075fd23682046db6998474ff488
:104d00007a7018f0cafb0124284640f2244117f0bb
:104d10000bfd204647b0f0bd182128680192fff72f
:104d200027fe18212868fff723fe2046019a134921
:104d3000fff721fe0024e7e718212868fff718fe97
:104d400018212868fff714fe721c04d10c49204674
:104d50000df046fdeee7b31c01d10a49f7e7033633
:104d60000cbf09490949f2e7b7120c02d7120c022d
:104d70001bda0c02de120c023e3c0c02e5120c02a5
:104d8000fd120c0234130c024a130c025b130c02ca
:104d9000012009f08dbb08b50023c269006b20f02b
:104da000e4f8b0fa80f0400908bd70b505460e463b
:104db0008069002120f0a4f8002304461a463146f9
:104dc000286b20f0f3f818b1201e18bf012070bd29
:104dd0000120fce708b500238269006b20f0e6f8ab
:104de000b0fa80f0400908bd38b50546fff7d3ff9b
:104df000044620b1686a10b1002120f085f82046f1
:104e000038bd012a02d1016000207047022a04bf88
:104e10000b680360f8e7036818470000014b186847
:104e200020f003b944c6001010b5044c236813b930
:104e3000204620f016f9206810bd00bf30c60010d3
:104e400010b50a4cd4e88f3fdb070cd4204619f08c
:104e50009dfb40b1064820f0def8204619f0d0fb5b
:104e60000448a4f060ff024810bd00bff8c5001060
:104e700044c600109d4d0002014b1860704700bff2
:104e8000f4c5001038b5002383608b6804460d46d6
:104e90002bb102229847eb68e360ab68a360204621
:104ea00038bd000030b5214b8db00093204b6946d2
:104eb0000393204b04a80293fff7e4ff4ff4a052a2
:104ec0006423cde908236ff000430a9332231a4c80
:104ed000adf82c300223204600258df82e30174bdc
:104ee00004a940f8043bfff7cdff089b04f128001c
:104ef0006361099b6562a3610a9be361bdf82c3085
:104f000023849df82e3084f8223020f084f80c4b56
:104f100004a8236084f82c502563fdf70bfe684637
:104f2000fdf708fe074b9d600db030bd114d00022e
:104f3000974d0002834d0002fcc5001080130c0247
:104f400090130c0234c6001010b5c36804460bb9a8
:104f5000a4f090fb0369043098470021a0616069c8
:104f6000bde8104020f0dcb810b5c36804460bb9aa
:104f7000a4f080fb03690430984700212076606923
:104f8000bde8104020f0ccb808b504f07ffb00204d
:104f900008bd000007b51346002200920a460146ec
:104fa000054800680ef00bf9002818bf6ff0ef00fd
:104fb00003b05df804fb00bf98ca0010012a70b569
:104fc000054603d10b680360002070bd022a08d09b
:104fd000032af9d100680028f6d0102117f0a4fbad
:104fe000f2e710200e6817f097fb044618b196e818
:104ff0000f0084e80f002c60e6e7012a70b5054633
:1050000003d10b680360002070bd022a08d0032a78
:10501000f9d100680028f6d0102117f085fbf2e7df
:1050200010200e6817f078fb044618b196e80f00c0
:1050300084e80f002c60e6e7012a08bf0160002029
:105040007047012a38b5044602d10b68236003e09b
:10505000022a03d0032a0dd0002038bd0c200d6891
:1050600017f05afb03460028f0d095e8070083e8c4
:105070000700ebe700680028eed00c2117f054fb86
:10508000eae7012a70b5054603d10b6803600020ea
:1050900070bd022a08d0032af9d100680028f6d092
:1050a000102117f041fbf2e710200e6817f034fbd7
:1050b000044618b196e80f0084e80f002c60e6e77c
:1050c000012af8b5064603d10b6803600020f8bd3d
:1050d000022a08d0032af9d100680028f6d014214a
:1050e00017f022fbf2e714200c6817f015fb0746b7
:1050f00020b105460fcc0fc523682b603760e5e76c
:10510000012af8b5064603d10b6803600020f8bdfc
:10511000022a08d0032af9d100680028f6d0142109
:1051200017f002fbf2e714200c6817f0f5fa0746b7
:1051300020b105460fcc0fc523682b603760e5e72b
:10514000012a034602d1016000207047022a04bff1
:10515000d1e90001c3e90001f6e7012a02d10160ab
:1051600000207047022a04bf0b680360f8e7012a99
:1051700008bf016000207047012a02d101600020b1
:105180007047022a04bf0b680360f8e7012af8b5ec
:10519000064603d10b6803600020f8bd022a08d040
:1051a000032af9d100680028f6d0182117f0bcfabc
:1051b000f2e718200c6817f0affa074630b1054641
:1051c0000fcc0fc594e8030085e803003760e3e7e0
:1051d000012a034602d1016000207047022a04bf61
:1051e000d1e90001c3e90001f6e700224ff0ff31e9
:1051f0001ff076bf00224ff0ff311ff071bf00009b
:1052000010b50446034b40f8043bfdf793fc2046e1
:1052100010bd00bfa0130c0210b50446fff7f0ff4d
:105220002046142117f080fa204610bd10b5074b18
:1052300004460360406918b11ff04dff002363610d
:105240002046fff7ddff204610bd00bfb4130c025f
:1052500010b50446fff7eaff2046182117f064fa5c
:10526000204610bd10b50446024b0360fff7deff79
:10527000204610bdc8130c0210b50446fff7f2ff1c
:1052800020461c2117f050fa204610bd10b50446e8
:10529000034b40f8043bfdf74dfc204610bd00bf1a
:1052a000dc130c0210b50446fff7f0ff2046142172
:1052b00017f03afa204610bd10b5074b04460360bc
:1052c000406918b11ff007ff002363612046fff714
:1052d000ddff204610bd00bff0130c0210b50446e0
:1052e000fff7eaff2046182117f01efa204610bdee
:1052f00010b50446024b0360fff7deff204610bde9
:1053000004140c0210b50446fff7f2ff20461c21de
:1053100017f00afa204610bd406a1ff0c8bd000011
:1053200010b404460748134600682ab121460023fa
:105330005df8044b0df028be0a4621465df8044b8b
:105340000df029be98ca0010f0b52e4e044696f80e
:105350002c300d4687b0002b4ad03046fff7dcffdb
:105360000746002844d1284b1c200593274bcde944
:105370000245049317f0d0f90446002831d0244b9d
:10538000c7600360049b3bb1022202a90430984726
:10539000059b2361049be360002520461d4b2a46a4
:1053a0002360012140f8145f1ff08afe1a4b01a907
:1053b0002360f2692b46306b01941ff0d6fd014645
:1053c00050b9706a08b11ff09ffd00224ff0ff3105
:1053d00060691ff085fea569236820469b68984791
:1053e00000e0054602a8fdf7a5fb284607b0f0bd82
:1053f00004f07ef92a46214607b0bde8f0400df0e2
:1054000012bf00bffcc500109d530002c150000236
:10541000dc130c02f0130c0204140c02d0e900019e
:10542000fff792bf054b1b7803f0ff0023b1044b3d
:105430001878003818bf0120704700bfc2c40010a0
:10544000bfc4001008b50948fff766ff68b1002027
:1054500006f08efa20b1bde80840044801f0eebe27
:105460000120bde8084009f023b808bdc4cb0010f6
:10547000002190b583b0044600af084616f040fe08
:10548000c31d23f00703adeb030d014678606846aa
:1054900016f036fe20467a68694604f0b9fd2046cb
:1054a0000c37bd4690bd0000014b186000207047ce
:1054b00094ca00107fb51d4d044695f82c300e4659
:1054c000b3b12846fff728ff90b9194b69460393fb
:1054d000184b2846cde900460293fdf723fc04460d
:1054e00088b905466846fdf725fb284604b070bd1f
:1054f00094b1631c13d021460f4802f05df80e48aa
:1055000002f047f80be04069fff774fe236820467d
:105510009b68a5699847e5e7074802f035f8064813
:1055200004b0bde8704002f08bb800bffcc50010ad
:10553000bd5400025151000248c60010d0e90001dc
:10554000fff7b8bf2de9ff41014640b368460df0b3
:105550007bf8009e9df80940ddf804809df8085016
:10556000fff760ff00b304f07ffd4ff00103d0e8c8
:10557000cf7fc0e8423f002af9d1ffb2002ff6d119
:10558000c660c0f81080057544750023c0e88f3fe1
:1055900006f0b6f90024204604b0bde8f0810546c7
:1055a000804604460646dbe706f0aaf916f0040634
:1055b00025d0002cefd0134c94f82c3013b904f004
:1055c00065f8e7e72046fff7a7fe0028f7d10e4b66
:1055d000694603930d4b20460293fdf7a3fb054656
:1055e00058b14069fff706fe2b6828469b68ac69f6
:1055f00098476846fdf79efacde70446f9e734463a
:10560000c9e700bffcc50010094f0002b94f0002f6
:10561000f0b504462c481f4690f82c300e4615462f
:1056200087b0dbb1fff778fec0b90490102017f007
:1056300073f818b1c0e90046c0e90257234b029045
:105640000593234b204802a90493fdf76bfb044606
:1056500060b9054602a8fdf76dfa04e0012c25d9d2
:10566000022c0cd01b4d284607b0f0bd4069fff757
:10567000c1fd236820469b68a5699847eae729464b
:1056800002a80cf0e1ff04f0effc029b0025d90713
:1056900044bf9df8102002729a0744bf039a4260eb
:1056a0005b0744bf9df811304372dce70a4800975e
:1056b0002b463246214600680df04bfd07b0bde891
:1056c000f0400df07dbb00bffcc500105d56000230
:1056d0007b4f0002f2feffff98ca00100068d0e97d
:1056e0000223d0e90001fff793bf000030b5044664
:1056f00028481d4690f82c3087b00bb3cde9001236
:10570000fff70afedde90012d0b90490102017f06f
:1057100003f828b1019a0099c0e9022504604160ac
:105720001d4b029005931d4b1a4802a90493fdf7e7
:10573000f9fa044670b9054602a8fdf7fbf906e040
:10574000042c19d0052c1cd0032c0cd0144d284649
:1057500007b030bd4069fff74dfd236820469b68c8
:10576000a5699847e8e70f4b1b787bb1082007b085
:10577000bde83040fff70ebc0a4b1b7833b109205f
:10578000f5e7084b1b780bb10a20f0e76ff0d10565
:10579000dde700bffcc50010295700023d4f0002a5
:1057a000f2feffffbfc400100068d0e90223d0e979
:1057b0000001fff79bbf000073b506461c200d4695
:1057c00016f0aaff044628b3144b03600023c360fd
:1057d000ab683bb10222294604309847eb6823614d
:1057e000ab68e360002220460d4b0121236040f8a6
:1057f000142f1ff065fc0b4b304623603368019477
:105800005b6801a99847054620b9236820469b6834
:1058100098472c46204602b070bd00bfa0130c0272
:10582000b4130c02c8130c022de9f04305462e48b0
:10583000994690f82c3087b00e4690460e9f2bb3b9
:10584000fff76afd10bb0490182016f065ff40b109
:105850000f9bc0e90056c0f8088080f80c900761e3
:105860004361224b02900593214b1f4802a90493e8
:10587000fff7a2ff054670bb044602a804f001042e
:10588000fdf758f9204607b0bde8f083b9f10009eb
:1058900018bf4ff00109cde9007816484b46324653
:1058a000294600680df07efb04460028ead0fff789
:1058b000b9fd06460028e5d006f04ef8012803d1d0
:1058c0000d4b1b78002bddd03a4649462846fff7a2
:1058d00027fd3446d6e74069fff787fc2b6828464a
:1058e0009b682c7e9847c8e7fcc500107d580002d5
:1058f0000d51000298ca001044cc001007b5006892
:105900004269037b019202690092d0e901120068aa
:10591000fff78aff03b05df804fb000030b5174cb9
:10592000054694f82c3085b003b32046fff7f4fc0d
:10593000e0b9134b20460393124b6946009502933e
:10594000fff73aff044678b14069fff74efc236841
:1059500020469b68257e9847684605f00105fdf7bf
:10596000e9f8284605b030bd0546f5e703f0c0fe6e
:10597000002105b0bde830400df052bcfcc5001060
:1059800009590002db5000020068fff7c7bf0000a2
:10599000f0b5044622481f4690f82c300d461646b6
:1059a00085b0fbb1fff7b8fce0b90290102016f00b
:1059b000b3fe18b1c0e900450672c760194b0090ec
:1059c0000393194b694616480293fff7f5fe054607
:1059d00058b90446684604f00104fdf7abf82046c8
:1059e00005b0f0bd55b9002415e04069fff7fdfb97
:1059f0002b6828469b682c7e9847ebe75cb12046d5
:105a0000fbf7e0f94028eed820463b4632462946cf
:105a100004f08cfb0446003c18bf0124dfe700bf04
:105a2000fcc50010ad590002035000020068c368b5
:105a3000027ad0e90001fff7abbf00007fb5054651
:105a400022480c4690f82c301646f3b1fff764fc60
:105a5000d8b902900c2016f05ffe10b1c0e90054d6
:105a600086601b4b009003931a4b694617480293bc
:105a7000fff7a2fe044680b90546684605f0010519
:105a8000fdf758f8284604b070bd7db93146204670
:105a900004b0bde8704004f011bc4069fff7a5fbfd
:105aa000236820469b68257e9847e6e7102300215f
:105ab000adf80030084b68460195cde90234adf8e9
:105ac000021004f0fbfb0546dce700bffcc500103c
:105ad0005d5a0002c34f0002019700020368186874
:105ae000d3e90112fff7aabf30b5114c054694f86f
:105af0002c3085b08bb12046fff70efc68b90d4bfa
:105b0000694603930c4b204602930095fef71afa60
:105b10006846fdf70ff805b030bd0022074b11466f
:105b200018680df004fb05b0bde8304003f00cbc74
:105b3000fcc50010c15a0002f950000298ca0010ba
:105b40000068fff7d1bf00001fb50e4c94f82c3051
:105b500083b12046fff7e0fb60b90b4b6946039326
:105b60000a4b20460293fef7edf96846fcf7e2ff88
:105b700004b010bd0021064b186804b0bde8104009
:105b80000df0aabafcc50010235b0002ef50000222
:105b900098ca001008b5fff7d7ffbde80840fff727
:105ba00041bcfff7d1bf00002de9f04705463d4855
:105bb00086b013f0100f1c460e461746ddf83890dd
:105bc00090f82c300df1080822d003f0ff0a002bca
:105bd00046d0fff7a1fb002842d10490142016f014
:105be0009bfd28b1c0e90056c0e90274c0f81090ce
:105bf0002d4b029005932d4b41462a480493fef706
:105c0000a1f94046fcf796ff504606b0bde8f08784
:105c100033b3fff781fb18bb0490142016f07cfd12
:105c200028b1c0e90056c0e90274c0f81090204bba
:105c3000029005931f4b41461a480493fff7bcfda1
:105c4000044658b14069fff7d0fa236820469b68a4
:105c500094f818a098470af0010ad2e78246fae7ba
:105c60000023cde903330c230293b9f1000f05d0d3
:105c7000d9f804300393d9f80830049314f0010fd5
:105c800014bf4522652224f0010313430a48009300
:105c9000cdf804803b463246294600680df016f9df
:105ca0008246b1e7fcc500103d5c00028150000255
:105cb000575c00024150000298ca001007b5006806
:105cc00003690093d0e90223d0e90001fff76cffdc
:105cd00003b05df804fb07b5006803690093d0e9e1
:105ce0000223d0e90001fff75fff03b05df804fb7a
:105cf0000021014801f0eabb48c6001030b5cc1cb9
:105d00002a3114f8035c033405f00f0205f0f003a8
:105d100042ea021243ea1515130243ea05434360bf
:105d200014f8052c02f0f00545ea12152b4302f099
:105d30000f024360827214f8043ca14203eb830318
:105d400003eb83034fea430320f8083fd9d130bd6a
:105d5000002138b504460846fcf7ecf91c25002361
:105d60002046094c05fb0342416801331161817ae9
:105d70000d2b517330f8081f9182f3d10021bde83b
:105d800038400120fcf7d6b958c600100c2808b5d9
:105d90000ad81c22054b02fb0030002201730121ae
:105da000fcf784f9002008bd0120fce758c600106c
:105db00011f0040238b50cd000240b4d0022284607
:105dc00011460134fcf772f90d2c05f11c05f5d1d3
:105dd00038bd0c28fcd81c24034b114604fb0030b2
:105de000bde83840fcf762b958c600100c289fbfc8
:105df0001c22044b02fb0030807b94bf00f00100aa
:105e00000020704758c60010f0b58a0705460c46ba
:105e10009db01cd501256822002102a8a4f0d1f96b
:105e2000214901a80195fff769ff01a8fff790ff3d
:105e3000e30709d5ff232a4640f6af618df803300a
:105e40000df1030017f03ffc00201db0f0bd03680a
:105e5000012b27d1fff77cff14f00100f5d001a939
:105e6000084632262b4668355a68c2f30357c2f3f8
:105e7000033444ea07144c709c7a02f0f00204f0f8
:105e80000f0422438a7033f8082fb2fbf6f29d42ca
:105e900001f8032fe8d10123402240f6af618df8cd
:105ea0000430cfe70120d0e710140c0270b502686f
:105eb000012a18d111f0020105d00c49fff71eff8d
:105ec0000021084670bd0b461c26094d06fb0352f7
:105ed000146901334460547b0d2b8472928a20f83c
:105ee000082ff3d1ede70121ebe700bf10140c02fe
:105ef00058c600100c289dbf1c22024b02fb00302c
:105f00000020704758c60010022803d0032807d08d
:105f100000207047142909d00adc4ff4fa7070474a
:105f2000142907d009dc4ff4fa507047c820704795
:105f3000642070474ff47a6070474ff47a7070476e
:105f40000021224a30b50b4615461c24adb004fb97
:105f5000015001310d29c2e900439360037302f13e
:105f60001c024373837303618382f0d16822002192
:105f700012a8a4f026f90123402240f6af6001a93f
:105f8000119317f06bfb18b99df80430012b1ad050
:105f90000f4b01aa03f1200514461868596808330d
:105fa00003c4ab422246f7d1998818689b79a18037
:105fb0002060a37101a911a8fff7a0fe11a8fff7a7
:105fc000c7fe2db030bd0df10501f4e758c6001035
:105fd00094fe0b022de9f04f4ff0180a91469b46b4
:105fe0000e46154985b0d1e9004103900afb014aec
:105ff000dde90e780c34a4f10c018a4511d054e986
:106000000301039b3140184050ea010307d000947c
:106010005b464a463146039854f8045ca847183456
:10602000e9e72fb140463b4605b0bde8f04f1847c1
:1060300005b0bde8f08f00bfc4c7001030b5d1e98e
:106040000054d0e900232a40234013430cd0836836
:1060500013b18a68934207d1c3683bb158680b6992
:10606000c31a5842584130bd0020fce70120fae72e
:10607000704710b50446282116f056fb204610bd87
:10608000012af8b5064603d10b6803600020f8bd6d
:10609000022a08d0032af9d100680028f6d0182176
:1060a00016f042fbf2e718200c6816f035fb0746a5
:1060b00030b105460fcc0fc594e8030085e8030016
:1060c0003760e3e72de9f043dff8d88093b08146ed
:1060d000d8f800000e4615461c461ef0d1ff12f0ff
:1060e00087fc00230746cde90096cde903330295ee
:1060f00005933cb1628821460c2a28bf0c2203a8d4
:10610000a4f038f86d4606ac0fcd0fc495e8030037
:106110000cae0df1180c84e80300bce80f001f4d15
:106120000fc694e80300d5f80490ab6886e8030036
:1061300099451adb09f10104002c286810dd1821ab
:106140006143a4f0bfff70b9154c384612f054fcff
:10615000d8f800001ef0a3ff204613b0bde8f0837e
:10616000a3f0e2ff00202860ac6018236a6803fbfc
:1061700009f95a432c68a2eb09024c442146e01865
:106180000caea4f004f80fce0fc496e803006b68c1
:1061900084e80300013300246b60d6e7c4c7001015
:1061a000fcfeffffd0c700102de9f04f8fb0019328
:1061b000574b83461868894616461ef061ff12f059
:1061c00017fc1822534fcde902b9d7e90045019bce
:1061d000554304960deb020c05930df108090aae28
:1061e000824699e80f008ce80f0086e80f004a4bc2
:1061f00004eb0508ed105d43ad10002d1ddd2146bb
:106200003046fff71bff30bba3461834214630460b
:10621000fff714fff8b90bf1300421463046fff7c1
:106220000dffc0b90bf1480421463046fff706ffc9
:1062300088b90bf16004013ddfe7a8eb0403302bc4
:1062400027d0482b1ed0182b4cd121463046fff7c3
:10625000f5fe002846d0a04545d004f11806b0450b
:1062600041d031464846fff7e9fe48b92546b446d5
:10627000bce80f000fc59ce8030085e80300183454
:106280001836ece721463046fff7d8fe0028e2d169
:10629000183421463046fff7d1fe0028dbd11834f0
:1062a000d3e71d48e31adb10151b00fb03f304d4ee
:1062b000ed1045435819814200dacd1a182101fb2f
:1062c00005412046521aa3f062ff7b685b1b7b608e
:1062d000504612f091fb0e4b18680fb0bde8f04f1e
:1062e0001ef0ddbe444618267a683b6806fb023382
:1062f0009c42edd02546d7e9003106fb013295429c
:10630000cfd0286910b16b6903b198471835f2e70f
:10631000d0c70010c4c70010abaaaaaa2de9f04745
:106320001f461e4b164693f82c2086b00546dde925
:106330000e890c46eab1586a1ef0b9fdc8b904903e
:10634000182016f0e9f928b1c0e90054c0e9026745
:10635000c0e90489124b02900593124b02a90f4821
:106360000493fdf7effd02a8fcf7e4fb06b0bde8df
:10637000f087dff834a0daf800001ef081fe28462e
:106380003b4632462146cde90089fff723fedaf885
:10639000000006b0bde8f0471ef081bec4cb00107f
:1063a000f163000201600002d0c700102de9f04740
:1063b000dff860c00746dde90898dcf804c00e4647
:1063c000ccf3080c15461c46bcf1000f16d000217a
:1063d000282008f00df90146a0b1002383600a4b84
:1063e000c0e904760360c0e90654c0e90898074b89
:1063f0004360bde8f047064800f04cbfbde8f047f9
:10640000fff78cbfbde8f08740140c02cb6300029d
:1064100074d0001000ed00e010b4039ce40703d535
:106420005df8044bfff7d6bd5df8044bfff7bebf28
:10643000002307b5024600214ff48040cde9003328
:10644000fff7b4ff03b05df804fb13b50446436add
:106450000193036a0093d0e90623d0e90401fff712
:106460005dff0021204602b0bde8104008f0d2b820
:1064700007b501684b6901930b690093d1e90223c9
:10648000d1e90001fff74aff03b05df804fb00000b
:106490000023044a0448c2e90033936003601ef0fd
:1064a000e0bd00bfc4c70010d0c7001013b5002462
:1064b0000622234603210120009407f025fe2246f0
:1064c0002146042000f024fb024670b10023042082
:1064d0001a46194600f0defc002304201a4619462d
:1064e00002b0bde8104000f0c5bd0146042000f038
:1064f0005efb0028ead102b010bd10b4012913469a
:10650000c06808d102685968146803f1080223467c
:106510005df8044b18476ff077005df8044b704747
:1065200038b5144619b904220846226038bd1368ec
:10653000032b07d903685b6898470028f6d104232a
:106540002360f3e76ff0bd00f0e7836900200b6084
:10655000704738b5144619b904220846226038bd80
:106560001368032b07d903685b6898470028f6d1a6
:1065700004232360f3e76ff0bd00f0e78369002098
:106580000b6070471830036800200b6070471830ac
:10659000036800200b60704738b505460c4612f0c2
:1065a00027faab69236012f027fa002038bd0000fb
:1065b00070b5104e8ab019f00cfd736a1bb1c01a89
:1065c000b0f57a7f12d30c4901a80bf0e9fe029bcb
:1065d0000a4c7360039b04adb3600fcd0fc495e804
:1065e000030084e8030019f0f4fc706201480ab06b
:1065f00070bd00bfd8c80010c4d00010e4c800109f
:1066000038b50d46fff7d4ff044688b103685b69cf
:106610009847b5eec00af1ee10fa0cd42368204674
:106620009b699847beeec80a002085ed000a38bd78
:106630006ff07700fbe76ff06300f8e738b50d46c1
:10664000fff7b6ff044688b10368db689847b5eeec
:10665000c00af1ee10fa0cd4236820461b69984753
:10666000beeec80a002085ed000a38bd6ff0770045
:10667000fbe76ff06300f8e738b50d46fff798ffca
:106680000446b8b103685b699847b5eec00af1eefd
:1066900010fa12d4236820465b699847dfed087a28
:1066a00020ee270abceec00a10ee103a00209bb282
:1066b0002b6038bd6ff07700fbe76ff06300f8e701
:1066c0000000804338b50d46fff772ff0446b8b1ad
:1066d0000368db689847b5eec00af1ee10fa12d4f1
:1066e00023682046db689847dfed087a20ee270a0a
:1066f000bceec00a10ee103a00209bb22b6038bdf1
:106700006ff07700fbe76ff06300f8e7000080436d
:1067100010b50c46fff74cff28b103689b689847fb
:106720002060002010bd6ff07700fbe70a4b10b52a
:10673000036014234360012304464381074bc0e9ef
:1067400003200181436100210430fbf749fe044b23
:106750002046236010bd00bfbc140c027b64000205
:10676000c8140c0200487047d4c700102de9f0414e
:106770003d4c082120463d4a0025fff7d7ff1c214c
:1067800014273b4b3b4a23606018a561fff7ceffff
:10679000394bdff85081e361384b394ec4e90f7350
:1067a000384b2946636404f13803a3646563c4f875
:1067b0003880e66404f13c00fbf712fe324b2946b8
:1067c000a363324bc4e91458e365314ba7652366d4
:1067d00004f15403c4e9193604f15800fbf700fe34
:1067e0002c4b092163652c4ae56604f17000fff724
:1067f0009dff2a4bc4f888502367294c294b182247
:10680000236002232946c4e9013504f10c00a3f0fa
:10681000d8fc6562244c21212046244afff786ffdc
:10682000234b25212360234c234a2046fff77eff7c
:10683000224b22212360224c224a2046fff776ff7a
:10684000214b23212360214c214a2046fff76eff74
:10685000204b24212360204c204a2046fff766ff6e
:106860001f4b2360bde8f081d4c7001048140c0210
:10687000d8140c0251140c02e8140c020c00020093
:106880007b6400025e140c02f8140c021b00020070
:1068900068140c0208150c0274140c0218150c0272
:1068a000d8c80010c02d0c0278c800107c140c024f
:1068b00038150c02a8c8001087140c0258150c02d9
:1068c00060c8001093140c0228150c0290c8001028
:1068d0009f140c0248150c02c0c80010ac140c0226
:1068e00068150c02bc140c0230b5134b8db01d782a
:1068f000e5b10024042022460df10f011c708df833
:106900000f40fcf75dfc9df80f3093b12023cde9db
:1069100004340a4b1e200a49009304aa2346fbf7bd
:10692000e1fa224621460420fcf732fc28460db04d
:1069300030bd1d46fae700bf5251001070150c0221
:1069400018100c02012a02d1016000207047022aaf
:1069500004bf0b680360f8e7012a034602d1016017
:1069600000207047022a04bfd1e90001c3e90001f9
:10697000f6e7012a02d1016000207047022a04bf15
:106980000b680360f8e7012a034602d1016000208a
:106990007047022a04bfd1e90001c3e90001f6e70c
:1069a000012a02d1016000207047022a04bf0b684f
:1069b0000360f8e707b5016811f00101019107d103
:1069c00005f08efc019903b05df804eb05f056bdaf
:1069d00005f086fc03b05df804eb05f0b1bd0000e6
:1069e00007b5006850b101a9c0b223f0a1f928b9d8
:1069f00003f0f4ff0122019904f0c0fd03f0eeff63
:106a000004f0befb0122044b1a700022034b1a70e3
:106a100003b05df804fb00bf03c9001002c90010f9
:106a200030b50d46044685b010bb03460a460090bb
:106a30000321012007f068fb194b1c700122194b40
:106a4000c3e88f2f03f0caff0722214604f0cefed1
:106a500003f0c4ff294604f00afcf0b903f0beffbe
:106a600004f058fa022818d0012016f016fdf5e7b8
:106a700003a9c0b223f05cf948b903f0afff2a467e
:106a8000039904f0b3fe03f0a9ff04f0f4f903f056
:106a9000a5ff04f09ef90028dad005b030bd00bf94
:106aa00003c9001004c9001001790068fff7b8bfde
:106ab00008b503f093ff04f049fb03f08fffbde836
:106ac00008400722002104f091be0000042810b500
:106ad00019d10e4c7e2200212046a3f072fb4ff00c
:106ae000ff33c4f87e30a4f88230c4f85730a4f8dd
:106af0005b306ff07b03237000232046637014f03b
:106b00007ef8204610bd0020fce700bf05c900103c
:106b100073b50d46d8b911f0ff0506d103f05eff3d
:106b200002b0bde8704004f09eb9012d06d103f01b
:106b300055ff02b0bde8704003f082bf022d34d192
:106b400003f04cff02b0bde8704003f080bf01a924
:106b5000c0b223f0edf830bb03f040ff019904f020
:106b6000fdf80446f8b103f039ff019904f042f949
:106b7000064603f033ff019904f044f915f0ff05d0
:106b800006d1022e01d002280dd1204602b070bde0
:106b9000012d04d1022e14bf00240124f5e7022d9b
:106ba00001d10228f7e70024efe70446ede713b52b
:106bb00030b903f013ff02b0bde8104004f049b94a
:106bc0006946c0b223f0b4f868b9019001a90098f1
:106bd00023f073f9002806db019800f0410001283a
:106be00001d102b010bd0020fbe70020704713b5b3
:106bf000044638b903f0f2fe214602b0bde8104069
:106c000004f08fb801a9c0b223f092f830b903f0b4
:106c1000e5fe019904f085f802b010bd0020fbe705
:106c200013b5044638b903f0d9fe214602b0bde8d9
:106c3000104004f084b801a9c0b223f079f830b94b
:106c400003f0ccfe019904f07af802b010bd0120e7
:106c5000fbe713b5044638b903f0c0fe214602b085
:106c6000bde8104003f05cbf01a9c0b223f060f89a
:106c700030b903f0b3fe019903f052ff02b010bd2a
:106c80000020fbe770470020704708b505f028fb9f
:106c9000bde8084005f028bb07b50c4b5b68cde9a3
:106ca0000012c3f3080343b905f01afbdde9001233
:106cb00003b05df804eb05f07bbc05f011fbdde9ea
:106cc000001203b05df804eb05f038bb00ed00e006
:106cd00010b5042886b011d11046059213f0f0fecd
:106ce000059b044638b9cde901000090012210202f
:106cf0000021fff791fb204606b010bd004cfae7db
:106d0000f2feffff13b5044648b903f067fe2146c3
:106d100003f032ffb0fa80f0400902b010bd01a9c3
:106d2000c0b223f005f840b903f058fe019903f012
:106d300023ff003818bf0120efe70020ede74ff0f8
:106d4000ff3070474ff0ff30704708b505f0c8fac4
:106d5000bde8084005f0ccba704700007fb5104e82
:106d6000044696f82c300d4693b1706a1ef09ff8d9
:106d700070b90c4b694603930b4b30460293cde937
:106d80000045fdf7dff86846fbf7d4fe04b070bda0
:106d90002046e9b204b0bde87040fff741be00bf35
:106da000fcc50010296a00020769000237b50446d5
:106db0000068a8b900220121174b10461a70174b22
:106dc00019700321fff7caff03f008fe04f0e6f98b
:106dd0006368db071dd503b0bde8304004f090bd0b
:106de00000220321fff7baff207801a922f0a0ffbb
:106df000054628b903f0f2fd2a46019904f0befbce
:106e00002368002bd6d003f0e9fd03f0e2ff002851
:106e1000d0d003b030bd00bf03c9001002c90010bc
:106e200030b5174d044695f82c3085b08bb1686aa3
:106e30001ef03df868b9134b28460393124b694680
:106e400000940293fdf77ef86846fbf773fe05b0e9
:106e500030bd54b16946e0b222f06aff28b903f0b0
:106e6000bdfd0122009904f089fb03f0b7fd04f099
:106e700087f90122054b1a700022054b1a70e6e7cc
:106e8000fcc5001061690002f368000203c900102c
:106e900002c900107fb5234e044696f82c300d46eb
:106ea00093b1706a1ef003f870b91f4b304603931c
:106eb0001e4b6946cde900450293fdf743f868464d
:106ec000fbf738fe04b070bda4b900220121184bb5
:106ed00010461a70174b19700321fff73fff03f09c
:106ee0007dfd04f05bf9eb07ecd504b0bde8704024
:106ef00004f006bd204600220321fff72fffe0b279
:106f0000694622f015ff044628b903f067fd2246c2
:106f1000009904f033fb03f061fd03f05aff0028f1
:106f2000d3d0cfe7fcc500102d6d0002d968000258
:106f300003c9001002c9001030b5214b0c465b6834
:106f400087b0c3f3080343bb1e4d95f82c308bb1bb
:106f5000686a1df0acff68b91b4b284605931b4bb4
:106f600002a904930294fcf7edff02a8fbf7e2fdef
:106f700007b030bd14f00101019107d105f0b0f95f
:106f8000019907b0bde8304005f078ba05f0a8f9de
:106f900007b0bde8304005f0d3ba11f0010201920c
:106fa00008d105f09df90121019a07b0bde83040f4
:106fb00005f0c4b905f094f900220221f5e700bffd
:106fc00000ed00e0fcc5001035690002c568000254
:106fd00037b50122244b05681a700022234b1a7022
:106fe000234bc3e88f2ffff77ffc044638b1002204
:106ff0001146104603b0bde83040fff79dbf03f0d7
:10700000edfc214603f08cfd0028f0d01db301a952
:10701000e8b222f08dfe40b903f0e0fc019904f0e3
:10702000d5fb03f0dbfc03f026ff03f0d7fc03f0f5
:1070300008ff18b903f0d2fc04f0a2f803f0cefc6c
:10704000002103f06dfd60b103f0c8fc03b0bde8a2
:10705000304004f0b5b803f0c1fc294604f0b6fb9b
:10706000e3e703b030bd00bf03c9001002c9001040
:1070700004c9001030b5304d044695f82c3085b069
:107080008bb1686a1df013ff68b92c4b2846039337
:107090002b4b694600940293fcf754ff6846fbf7bc
:1070a00049fd05b030bd0122264b1a700022264b47
:1070b0001a70264bc3e88f2ffff716fc054638b130
:1070c00000221146104605b0bde83040fff734bf3e
:1070d00003f084fc294603f023fd0028f0d024b3fc
:1070e0006946e0b222f024fe40b903f077fc009933
:1070f00004f06cfb03f072fc03f0bdfe03f06efcc9
:1071000003f09ffe18b903f069fc04f039f803f0ae
:1071100065fc002103f004fd0028c2d003f05efcf2
:1071200005b0bde8304004f04bb803f057fc2146f1
:1071300004f04cfbe2e700bffcc50010516f0002f9
:107140002169000203c9001002c9001004c900101f
:1071500070b505f0c5f805f0c7f800283cd1224eff
:107160003378ebb9214c2378d3b904f0cffb98b333
:107170001f4bd3e88f3fdbb20bb1237863bb03f027
:107180002dfc03f070fe38bb03f028fc03f061fe19
:10719000034608bbbde8704002460146fff76abfe0
:1071a00003f01cfc03f05ffeb8b100220f4c104648
:1071b00025782378edb2002b14bf07210621fff7b5
:1071c000cdfd00231a4619461846fff763fe00233b
:1071d000084a33701360257070bd03f0fffb03f0a5
:1071e00038fe0028e1d1f7e701c9001002c90010fc
:1071f00004c90010a8d0001013b543690446cde9b6
:1072000000030a4990f82220094b24301df038fe73
:1072100020b10a20074a0849f9f7e2fe94f82c3019
:1072200013b91df04cfef9e702b010bd7d150c023c
:107230000d72000221d401028b150c02002313b53c
:107240000193036801a91b689847044620b101987f
:1072500028b103681b689847204602b010bd044659
:10726000fae708b5012380f82c30044615f048fcf5
:10727000a3f098fe251d2046fff7e0ffe3680bb959
:10728000a2f0f8f9284623699847f4e708b5fff714
:10729000e8ff000070b505460c4611f0a9fb6b68cd
:1072a0006bb19c600026a6606c6011f0a5fb054bdd
:1072b000586a30b13146bde870401df025be2c60e3
:1072c000f0e770bdfcc5001038b50446006868b131
:1072d00011f08efb2568ab682360236803b96360f7
:1072e00011f08afb28466b689847012038bd70472b
:1072f00010b504460c2115f017fa204610bd43695d
:1073000013b183690c301847704713b50021044648
:1073100008461df0cbfe0023204601a901931df075
:1073200035ff019c0cb101232371002101201df0c8
:10733000bdfe2cb1236820469b689847002323712b
:1073400002b010bd08b5fef76df848b10cf036f983
:10735000002204210bf0b7fdbde808400bf030bd62
:107360006ff0d10008bd000009490c2008b5a2f05b
:107370007df9014650b1074b036000238360064b43
:107380004360bde808400548fff784bf08bd00bf63
:10739000751d0e02d4150c028173000274d000100a
:1073a00010b403685a689968541001eb6200d20760
:1073b00048bf0a591b685df8044b48bfd3581847ab
:1073c000012a38b5044602d10b68236003e0022a83
:1073d00003d0032a0dd0002038bd0c200d6815f015
:1073e0009bf903460028f0d095e8070083e80700e2
:1073f000ebe700680028eed00c2115f095f9eae7dc
:1074000008b510b103685b689847bde80840fff70e
:1074100099bf07b5806830b10023cde900131a4643
:1074200002211df0bffe03b05df804fb38b5836890
:1074300004469bb16ff00041fff7ebff0021a0680d
:107440001df0abfe237903f0ff0513b11df037fdee
:10745000f8e72946a0681df0effea56038bd0000e2
:1074600038b505460446054b45f80c3bfff7defff3
:107470002846fbf75ffb204638bd00bfe4150c0231
:1074800010b50446fff7ecff20461c2115f04cf91f
:10749000204610bd10b50446064b03608068fff718
:1074a000c5ff237b23b1a06810b103685b689847d0
:1074b000204610bdf8150c0210b50446fff7eaff90
:1074c0002046102115f030f9204610bd284b2de93b
:1074d000f04103604ff0ff3306460d4688b043602d
:1074e000002943d11c2015f017f90446002834d098
:1074f0000c20d6f80480069515f00ef918b11d4b36
:107500008660c0e900351c4b0490236000230df118
:10751000080c04af97e803008ce803002371a36014
:1075200004f10c0292e8030087e803009ce80300e2
:1075300082e80300114a06936261a26941460792fc
:107540000f4a04f10800a261cde900330d4a234639
:107550001df00afe3846fbf7edfab5fa85f5304620
:107560006d09b460357308b0bde8f0810c46f4e7ee
:10757000f8150c02e9720002e4150c0241730002d6
:10758000217300028b7200026ff000418068fff7e8
:1075900040bf13b5846800212046fff73affa0687a
:1075a00040b100236ff000421946cde900231a468e
:1075b0001df0f8fd02b010bdf0b58368054698686f
:1075c0000e468bb0f0b100211df045fe041e18bf21
:1075d0000124ab689868b8b100226ff000474ff4ff
:1075e0007a7303217343cde900721df0dbfd03467e
:1075f00050b9a8686e60a4b939460bb0bde8f04038
:10760000fff707bf0446e4e720220023cde9022369
:10761000094a32200092094902aafaf763fc0bb02a
:10762000f0bd80680028fad01a460121cde9007328
:107630001df0b8fdf3e700bfa3150c0218100c02f3
:10764000fff780be2de9f04f0025b5b081460c460e
:1076500092460995002a78d05378002b75d0294698
:107660002a221da81c95a2f0acfd08230c20cde910
:107670000130cde90c550cad00959af800102e2381
:1076800050461caa21f02cff014600285dd1102293
:1076900018a8a2f096fd4c2314939af80130b9f182
:1076a000110f15930cbf022301232946169314aa28
:1076b00009ab1ca8cdf85c9021f0d8fe002844d17d
:1076c0000125099b4bb92022cde91c23a44a322075
:1076d0000092a4491caafaf705fc202100236ff0b0
:1076e000e508a14acde91c13009201209d490195ae
:1076f0001caafaf7f7fbdff86cb2099c002c00f02b
:10770000aa81d4e90212606822f0f2f80026202350
:10771000071ecde91c3680f29880d4e90173e26837
:1077200007930692a2f020fb079b0168069acde919
:1077300001738e4b049103920093594633463220d5
:107740001caafaf7cffbe469d8e7894b5a6822b143
:107750009b6813b102250993b3e7002c73d02578f9
:107760001db1012d35d00025abe71022294620a8f8
:10777000a2f027fd02264c23b9f1110fcde91c36ea
:107780000cbf33460123d4f802001e93cde91455f3
:10779000cde91655cde90c55cdf87c900a9523f02e
:1077a000ecf910230a9014aa30460aa923f0e1f953
:1077b000002886d00821b4f842306e4a0ca8a3f005
:1077c00037fd09ab1caa0ca914a821f04ffe032514
:1077d00077e71c2200210da8a2f0f3fc4823b9f1a1
:1077e000110f4ff000060c930cbf022301235c2203
:1077f00031461da80aaf0e93cdf83c901c96a2f01e
:10780000e0fc60225c4b1ca9a01ccde90a6607f0d5
:1078100022fc0821b4f84230564a3846a3f008fd4d
:107820002023cde914361cab0193544b28464d4917
:10783000009314aa33460297faf754fb394609ab72
:107840000caa1ca8c1e725463be7e3685946049308
:10785000a3680120039363681caacde90173484b18
:1078600000933346faf73efb2a2231461da81c96a8
:10787000a2f0a7fc6068022846d00a2850d0202237
:107880000023cde914231caacde901723d4a5946d3
:1078900000921e20039614aafaf724fbb9f1110fe7
:1078a00076d1626800230a2a72d11c2219460ca8dc
:1078b000a2f087fc1c228df830206368022b8df823
:1078c000313032d00a2b30d0012304220a9340f603
:1078d000ff71384600920aab21f0d5ff60b3202338
:1078e0000026cde91436a2f03ffa03685946cde9e7
:1078f0000173254b3220009314aa3346faf7f2faab
:10790000384621f0e7ff1ee72e2361691caa0431e7
:1079100023f02ff96369588823f035f90646aee75e
:1079200061692e231caa0831f2e741f2346023f08a
:1079300028f9adf83200c7e706901c2238460ca99a
:1079400021f062ff069b18b32022cde914230f4ad1
:1079500059460092322014aafaf7c4fad0e700bfc1
:1079600010160c0218100c0233160c0244160c02ee
:1079700054510010843e0c02fd99000200160c02c6
:1079800083160c02b4160c02d9160c020f170c0247
:107990003846d4e9042121f09fff20238046149328
:1079a00090b100231593a2f0dff902681cabcde97a
:1079b00003622c4acde9017300920023594632201c
:1079c00014aafaf78ffa9be71cabcde90173264b9b
:1079d00015900093254903460396012014aafaf74f
:1079e00081fab9f1110f224b0ad1023d012d07d8be
:1079f0005968e26931b19a604ab90991c3f80480c3
:107a0000012505e0002afbd00999c3e9011245468a
:107a10001f60baf1000f04d0d4e904215046a2f04f
:107a2000a9fb00260c960ca96068fcf78dff0122cb
:107a30000c996068fcf730ff304603f099ff01288d
:107a400008d130461df031fa0a49149014aa38467c
:107a500021f089ff15b1099821f006fd404635b0a7
:107a6000bde8f08f39170c026f170c0218100c02ca
:107a7000545100100873048030b50a46014611487d
:107a8000002300688db021f02fff041e15daa2f04c
:107a90006bf9036800250c2b12d02023cde90435a7
:107aa000a2f062f903680849cde90143074b32208f
:107ab000009304aa2b46faf715fa20460db030bd04
:107ac0002c46fae75451001018100c0293170c02c0
:107ad00030b50a4601461748082300688db021f0ea
:107ae000fffe041e07daa2f03ff903680b2b05d155
:107af000a2f03af9002420460db030bda2f034f9ce
:107b000003680b2bf4d0a2f02ff903680c2befd0f5
:107b100020230025cde90435a2f026f903680649a3
:107b2000cde90143054b3220009304aa2b46faf716
:107b3000d9f9e0e75451001018100c02ac170c02f0
:107b400030b5144c89b02368002b1fdbc20715d554
:107b50000121184621f05afe80b918f03afa05467c
:107b6000002220216846fff7b3ff002806db18f04b
:107b700030fa41f28732431b9342f1d9206821f059
:107b8000a9fe4ff0ff33236009b030bd6ff0d10084
:107b9000fae700bf5451001013b501a824f06cf8a7
:107ba000002242f21073114601a824f0f9f80446ad
:107bb00001a824f072f8204602b010bd6ff07700e3
:107bc00070470000014b1868c017704754510010ef
:107bd000014b1868704700bf5451001010b504469f
:107be00050304ef080fa04f144004ef07cfa20460a
:107bf000faf724fd2046bde81040b02114f094bdf2
:107c000038b5044606204ef05dfa054668b12046b8
:107c10004ef064fa0022294620464ef0b7fa034699
:107c200028b1bde8384024f0dfbc6ff07703184678
:107c300038bd08b54ef0eafa18b1bde8084024f0a6
:107c4000d3bc08bd08b54ef0fdfa18b1bde8084038
:107c500024f0cabc08bd00221421c0e90022c0e9fa
:107c60000222026101800275427582617047000044
:107c700010b50a4cd4e88f3fdb070cd4204616f031
:107c800085fc40b10648fff7e6ff204616f0b8fc39
:107c90000448a2f048f8024810bd00bf90c9001087
:107ca00094c90010797d00022de9f0478469a0b0e5
:107cb000289f002c00f09480d4f8a0509d4211d34e
:107cc0009e18ae420ed9eb1a761b3246194404f1c7
:107cd0004400fff7b7ff002869dbd4f8a030334435
:107ce000c4f8a030d4f8a030bb4229d200217c22b5
:107cf00001a80091a2f065fa18f040ffd4f8a03076
:107d0000c61900eb030904f14408b14516d2a6ebed
:107d1000090abaf1800f28bf4ff0800a694652461f
:107d2000484618f05dff002841db52466946404650
:107d3000fff788ff00283adbd144e6e7c4f8a070db
:107d4000d4f8a030ab4229d904f15006304604f1f2
:107d500044014ef0f5f930bb304604f17c014ef0a1
:107d60008bfa18b124f040fc002820db4822204682
:107d700004f15c01faf75cfd002818dbd4f8ac30a4
:107d8000ab4203d118f025f9c4f8a400d4f8a83008
:107d9000d4f8a02013445d1bc4f8a850d4f8a83030
:107da00043b9002003e024f01ffc0028d4da20b0ff
:107db000bde8f08718f00df9d4f8a430c01a47f2e6
:107dc0002f539842edd92046faf7a8fb0028eedba6
:107dd00018f0fff8c4f8a4000020c4f8a800e6e7f3
:107de0006ff0d100e3e710b50446006808b1fff773
:107df000f5fe204610bd000008b50248fff7f3ff6e
:107e000008bd00bfacc900100368016013b118467b
:107e1000fff7e4be7047000070b5856906468ab07a
:107e20003db3d5e927329a4226d1202205f15c01e3
:107e300005f17c00a2f08ef9044688b100232022cf
:107e40000e4ccde9022332200d49009402aafaf724
:107e500049f82046f9f702fe0a4c20460ab070bde8
:107e60002846faf7ebfb214606f11800fff7ccff96
:107e7000f3e76ff0d104f0e7034ceee7d0170c0204
:107e8000c5170c02cdfaffffb9faffff10b5044683
:107e9000806992b040b1faf7e5fb002104f11800c7
:107ea000fff7b2ff12b010bd054901a8faf726fb93
:107eb00001a8faf7d7fb01a8faf7c0fbf2e700bf69
:107ec000ff170c0270b5037d05468ab0c3b1846903
:107ed000b4b1d4f8a8309bb118f07bf8d4f8a43032
:107ee000c01a47f22f5398420ad92046faf716fbd8
:107ef00000284ff0000605db18f06bf8c4e92906ee
:107f00000ab070bd2023cde90236074b01900093e3
:107f100032203346054902aaf9f7e4ff28460ab0a1
:107f2000bde87040fff7b2bf10180c02c5170c0275
:107f300030b5037d04460d4685b0d3b1183000211d
:107f4000fff762ff607d08b90af093fb00230a4a3d
:107f50009d4213702375cde90133009318bf0122b0
:107f6000234608bf4ff0ff324ff480700021fef728
:107f700053fa05b030bd00bfc3c4001070b511f096
:107f800008020546047d01f0040301f0010626d134
:107f90008cb3e3b984691cb1fff73eff041e10db0c
:107fa0007eb9002018f050fe0446e1432846c90f70
:107fb000fff7beff002c10db4620fbf79bf90024e7
:107fc0000be02846fff762ff002ceedbe9e74221d9
:107fd000012018f007fe00eae074204670bd002c76
:107fe000fbd0002bebd10eb1fff750ff002128464c
:107ff000fff79effe3e76ff0d104eee72de9f043d2
:108000001f46037d0446894616468db0002b57d087
:108010004ff000082c4bc3f8008018f0affd43462a
:10802000c1193246484618f0cbfd0546c8b1202399
:10803000264e04aacde9043825494346019000960e
:108040003220f9f74fff29463046f9f707fd414640
:108050002046fff76dff6ff0da0528460db0bde84a
:10806000f083a369bbb1149b3246009349463b465b
:108070002046fff719fe70b12023cde90435154bda
:108080000190009332202b46114904aaf9f72affe8
:108090002046fff7fbfe637d13b9e720f9f70cf9e3
:1080a000236902223b44636000234ff48070cde9d2
:1080b00001330093002123462681fef7adf9cce77a
:1080c0006ff0d105c9e700bfc4c4001034180c021a
:1080d000c5170c0210180c022de9f04fa5b0019045
:1080e0008846b02066491646a1f0c0fa044698b109
:1080f00000256449faf702fa48222946c4e91155d5
:10810000c4e91355c4e9155504f15c00a2f059f80f
:10811000c4e92955c4f8ac500394002c00f0ad809c
:1081200004f14400fff76cfd041ec0f29680039832
:108130005030fff765fd041ec0f28f80039d48227a
:1081400005f15c0739462846faf7f4fa4828044650
:1081500040f08a80d5f89c30434552d1d5f8a03004
:1081600043454ed8202231463846a1f0f3ff8246df
:10817000002846d103984430fff75bfd041e6cdbfa
:1081800051467c2205a8cdf810a0a2f01af818f0ec
:10819000f5fc8346d5f8a03000eb030ad34517d28f
:1081a000aaeb0b09b9f1800f28bf4ff080095846a0
:1081b0004a4604a918f014fd041e4edb03984a46f3
:1081c00004a94430fff73efd041e46dbcb44e5e73f
:1081d000039800f1440150304df0b2ff002838d12f
:1081e000039804a950304ef047f818b124f0fcf978
:1081f000041e32db202204a905f17c00a1f0aaffb5
:10820000d8b10398faf72efa06f1200356f8042b9a
:108210009e4247f8042bf9d12022002105f17c0071
:10822000a1f0cfff00230398c5f89c80c5f8a030cb
:108230004430fff7fefc041e0fdb00240399d5f841
:10824000a0300198c1f8ac3018300394fff7dcfd82
:1082500003e024f0c9f9041ec2da03a8fff7c3fd46
:10826000204625b0bde8f08f0028cada10f1aa0f29
:10827000c7d010f58c7ff0d1c3e7034cede700bf0a
:10828000751d0e02ff170c02fcfeffff2de9f047e3
:108290008cb0149e04460f461d46904606f0040915
:1082a00006f0010abab1b3b1c6f34006227da2b10d
:1082b00000232021634ccde904133220624904aa33
:1082c0000094f9f70ffe2046f9f7c8fb6ff0d100d4
:1082d0000cb0bde8f0870126e8e7012004a98df87d
:1082e0001020faf76dff9df8102012b16fb95748b2
:1082f000eee7092004a98df81020faf761ff9df838
:108300001030002bf2d15248e2e718f03dfcb842a1
:10831000edd3baf1000f1ad1ceb942463946204604
:10832000fff7dafe002866da20220023cde90423d5
:10833000484a019000923220434904aaf9f7d2fd3d
:10834000b9f1000f76d12046fff7a0fd07e0b9f1a3
:10835000000f6ad12046fff799fd002eddd018f0fe
:108360000dfc3946002218f019fc014600284ed0b9
:108370004ff00008002211461046faf709fff9f7fe
:1083800031f80646607558b901200af072f9314695
:108390000b20fdf7affd002840d000690af08cf9f2
:1083a000012300262c4a237513701423a446cde91b
:1083b0000466cde907660696adf810300df1100e93
:1083c000bee80f00ace80f00ccf80060e76018f0e2
:1083d000d5fb206118f0defb236920816360a67263
:1083e000234632464ff480700021cde901660096a5
:1083f000fef712f820e0a369d3f8a080b9f1000fce
:108400000fd0002104f11800fff7fefc14e004f186
:108410001800fff7f9fc6ff0da0059e74ff0ff1092
:10842000bce7b8f1000fa5d199e71eb9baf1000f6a
:108430003ff473af4ff000080db1c5f80080002085
:1084400046e700bf55180c02c5170c02b9faffff2a
:108450009cfaffff7c180c02c3c4001048b101381d
:10846000222896bf05230723b0fbf3f34ff47a705d
:108470009840704708b578b103881b2b0cd943236b
:108480000371012343710223837103231422c371f7
:1084900002490830a3f0defc1c2008bda30f0c022b
:1084a00010b50446007c10b1d4e90230984720741e
:1084b00010bd036802224068184770470eb4f0b53b
:1084c000002692b017ad55f8047b3c223146044695
:1084d00003a80296a1f075fe3a462b46402102a859
:1084e0000195a4f0a3f83f28024605dd267412b0da
:1084f000bde8f04003b07047204602a9fff7d0ff67
:10850000f5e710b50446142114f00ef9204610bd0d
:1085100013b5044608460191f8f754fc024620467c
:10852000019902b0bde8104009f0babd37b56fea55
:1085300041416fea5141adf8041001a904461546c6
:10854000fff7b7ff30b104222368606801950deb97
:108550000201984703b030bd13b5044608460191a7
:10856000f8f730fc02462046019902b0bde8104001
:1085700009f086bd38b5044615460068fff7ecffe4
:10858000206809f0cbfc06492068fff7e5ff294683
:1085900009f0d0fc206809f09ffc2368187c38bde6
:1085a000661e0c027fb50e461546044608b10369e7
:1085b00023b90a20094a0a49f8f712fd0c23cde92c
:1085c00001362b68012103932046236901aa9847ad
:1085d00008b9039b2b6004b070bd00bf21d4010219
:1085e000af180c0237b5c3880446012b0d4604d0e2
:1085f0000a20074a0749f8f7f3fc042329462046d6
:108600000deb03020193fff7cdff03b030bd00bfb8
:1086100021d40102d5180c0237b5c3880446022bb9
:108620000d4604d00a20074a0749f8f7d9fc04236d
:10863000294620460deb03020193fff7b3ff03b079
:1086400030bd00bf21d4010201190c0273b5cb88e3
:108650000546012b0c4605d0022b17d06ff0770092
:1086600002b070bd0023694620460093fff7baffb1
:108670000246f0b9a388286801a9009eadf804302d
:10868000fff717ff48b96ff0bd00e9e7002369461f
:1086900020460093fff7c0ffeae704222b6801960b
:1086a0001c6858680deb0201a0470028ebd00020a1
:1086b000d6e7a1882868fff739fff6e70b460146a1
:1086c0001846fff7c3bf73b5054688680c4630b13e
:1086d000cb88012b05d0022b19d06ff0770002b0a8
:1086e00070bd0023204601a90193fff77bff0246de
:1086f000f0b9019ea1682868fff72eff314609f006
:108700003dfc2b681b7ccbb96ff0bd00e7e7002375
:10871000204601a90193fff77fff024640b9019e61
:10872000a1682868fff718ff314609f039fce8e72f
:108730002846a168fff71eff0028e5d00020cee7fd
:108740000b4601461846fff7bebf00002de9f04f6b
:10875000994b99b01546039300240123cde90501f7
:10876000964903a88df81c308df81040fff7f4fef1
:10877000698809f0dffb24272b8aa3420dd907fb68
:1087800004f6eb6803a89959fff7e6fee96801349f
:1087900031440431fff7bcfeeee7894903a8fff737
:1087a000dbfe03a809f0aefb4ff00008dff84492af
:1087b0002b89434540f2f880782606fb08f6d5f869
:1087c00004b00beb060494f82230052b00f2d180a4
:1087d000002b00f0d280a37b012b04d1b4f87030c1
:1087e0009b0740f1ca8004f114073846f8f76cfb88
:1087f000824603a809f092fb724903a8fff7acfe7a
:108800005bf8061009f0ccfb6f4903a8fff7a4fe44
:10881000a37b032b96bf6d4a6d4952f82310fff7d7
:1088200077fe6c4903a8fff797feb4f86e1009f0c5
:1088300081fb694903a8fff78ffeb4f8701009f0b7
:1088400079fbbaf1050f2dd100213c2209a808912e
:10885000a1f0b7fc614903a8fff77efe04f16c06a6
:1088600004f14c0308a913f8012b120902f1300c92
:10887000bcf1390f88bf02f1370c01f802cb13f8b5
:10888000012c02f00f0202f1300cbcf1390f88bf4d
:1088900002f1370c9e4201f801cce4d1402208a934
:1088a00009f0fefb4e4903a8fff756fe0646384680
:1088b000f8f70afb082898bf59f8201030464ff007
:1088c000000688bf4249fff723fe38460896f8f7ae
:1088d000fefa444a0346042108a8a2f0a9fc424932
:1088e00003a8fff739fe08a9fff712fe3f4903a8c6
:1088f000fff732fe82463846f8f7eefa0146504658
:1089000009f018fb3a4903a8fff726fe03a809f06f
:10891000f9fadff8ccb094f8247094f82530b4f864
:1089200026a0052f34d8002f35d003a8019309f0d5
:10893000f5fa594603a8fff70ffe59f82710fff77d
:10894000e7fd019b274a042108a8a2f071fc2649f3
:1089500003a8fff701fe08a9fff7dafd234903a8e2
:10896000fff7fafd514609f0e5fa03a809f0b4fa59
:1089700011e0073b012b7ff62eaf08f1010817e746
:10898000012694f8287094f82930b4f82aa0c8e792
:10899000f91f0129c9d9002ef2d003a809f093fad2
:1089a00003a809f099fae8e703a809f08cfa9df802
:1089b0001c0019b0bde8f08f94190c02b5240e020a
:1089c000df060c02de1c0c02ca660c027c190c02cb
:1089d0002f2b0c02768b0c022e190c02853e0c02fa
:1089e000b4220e02843e0c02c8250e02aa140c0208
:1089f0008d1b0c0258190c0218b10022012117f02e
:108a0000ccbf0148704700bff2feffff18b1002243
:108a1000114617f0c2bf0148704700bff2feffffca
:108a200030b587b004460d461222002101a8a1f0fe
:108a3000c8fb14230022adf804300123114601a81d
:108a4000adf81630fff7d8ff294601aa2046fff7f8
:108a50007dfe0446002101a8fff7d8ff204607b09d
:108a600030bd0000036824221b680149184700bf7d
:108a700031190c02f0b512f0010489b00e4605461a
:108a80000e9933d0cde9033103ab0193022302a940
:108a900003a8adf80830fff70cfd10b96ff0bd006a
:108aa00022e00423019802a9adf80830fff701fd88
:108ab0000028f3d095b100242746a64233d00022e7
:108ac00035f8140002a90297f9f7ecfc60b9029995
:108ad00001a8fff7bbfd38b90134eee72b46294664
:108ae0001f4801aaf9f7bafc09b0f0bdcde905317c
:108af0001c4b8df81040039301238df81c3003ab01
:108b00001846019309f00afa019b1b7c002bc5d083
:108b1000e5b12746a64208d1019809f0ddf9019b8d
:108b20001b7c002bbad00020dee7002235f81400b1
:108b300002a90297f9f7b6fc0028d5d1029901a83d
:108b4000fff7c1fd0028cfd10134e3e72b462946ca
:108b5000054801aaf9f782fc0028ddd0c4e700bf70
:108b60003d86000294190c02c186000213b5002450
:108b70000346cde9001420462146fff77bffb0fafb
:108b800080f0400902b010bd70470000014b18781a
:108b9000704700bfc0c900104c22034b5b6802fb4a
:108ba00000300830704700bfc0c90010014b187872
:108bb000704700bfb8c900105022034b5b6802fb2e
:108bc00000300530704700bfb8c900100368c1f815
:108bd000d030d1f8e03043f00403c1f8e030704702
:108be0000368c1f8dc30d1f8e03043f00803c1f885
:108bf000e03070470368a1f8e830d1f8e03043f086
:108c00001003c1f8e03070470368a1f8ea30d1f8ea
:108c1000e03043f02003c1f8e03070470368c1f84a
:108c2000e430d1f8e03043f04003c1f8e030704761
:108c30000368a1f8ec30d1f8e03043f08003c1f8cc
:108c4000e0307047002381f8e03081f8e13081f8ae
:108c5000e23081f8e3307047f0b404460f46bab909
:108c60000388b3f5837f0cd10b4e051d06f120025e
:108c7000334603cb9342286069601e4605f1080520
:108c8000f6d100233a462146f0bc184610f06abae5
:108c90004ff0ff30f0bc7047d4c500101fb5002462
:108ca0000a460094014603ab2046039410f06afa8a
:108cb00000b10394039804b010bd10b5002488b02f
:108cc0002146cde9040404a8cde9064417f0cefa04
:108cd000234601224ff480400021cde90144009455
:108ce000fdf79afb08b010bdf7b50d4616461f46b6
:108cf0000446fef7bdff33462a4621460097fff79c
:108d00007df903b0f0bd07b50190fef7b1ff019901
:108d100003b05df804ebfff731b9f7b50d46164621
:108d20001f460446fef7a4ff33462a462146009715
:108d3000fff7acfa03b0f0bd1830036800200b60f9
:108d400070471830036800200b60704700b50b4a6d
:108d50008bb0137873b10121094b1e2019700023c9
:108d600013702022cde90223064a0749009202aa85
:108d7000f9f7b8f80bb05df804fb00bfc1c40010f0
:108d8000c0c40010a4190c0218100c0208b510b1d0
:108d900003685b689847bde80840fdf787bb13b5db
:108da00004460191f8f70ef80199a0f1180204f1b8
:108db0001800a3f03bf8b0fa80f0400902b010bdf3
:108dc000f0b5edb005460c46f7f7fcff17282ad999
:108dd000182228466249a3f029f8074618bb204606
:108de000f7f7f0ff5f4902462046a3f01ff85e49ff
:108df000b0fa80f42846fff7d2ff6409064638b17e
:108e00003a46214609206db0bde8f040faf7c0b9f6
:108e100028465649fff7c3ff002800f09e803246df
:108e200021463046efe7132228465149a2f0feffc3
:108e3000064680b92023cde922304e4b4e4900939f
:108e400022aa03460120f9f74df830466db0bde87f
:108e5000f04018f06fb828464849f7f7a9ff0028f6
:108e600046d1002c79d02378002b76d02146444877
:108e7000f7f79eff20b96db0bde8f04009f079be6c
:108e800021464048f7f794ff20b96db0bde8f040a7
:108e900009f054be21463c48f7f78aff20b96db06f
:108ea000bde8f04009f062be21463848f7f780ff80
:108eb0000446002851d12023cde92230344b2e49dd
:108ec000009322aa03462820f9f70cf831490c2018
:108ed000a0f0ccfb014600283fd02f4b84600360fc
:108ee0002e4b43602e486db0bde8f040fef7d2b97e
:108ef000182228462b49a2f099ff70bb2023cde908
:108f00002230294b1c4922aa009303461e20f8f761
:108f1000e9ff032010f008f804464ff49372ff2194
:108f200022a8a1f04ef98022ff2102a8a1f049f960
:108f30005cb11e4b1e491a6822a8a1f01bf91d4bfb
:108f40001d491a6802a8a1f015f9214622a818f0b7
:108f500044f8214602a818f04bf86db0f0bd00bff0
:108f6000a31f0c02a80e0c02831f0c02bc1f0c02d4
:108f70006f1f0c02cf190c0218100c025c1f0c02a0
:108f8000051a0c020f1a0c02131a0c023a1a0c02e0
:108f90001a1a0c02751d0e02d4150c020d8d00025a
:108fa00074d000108a1f0c02421a0c0284090c02b1
:108fb00028090c0224090c020b090c02f7b506461d
:108fc000184fd7e88f5f15f0010522d1384615f00c
:108fd000ddfaf0b12a4614210f20fcf795ff1e227e
:108fe0000221114c0346cde9002120460f226ff0eb
:108ff0007f4109f0e1fd0d4b384623600c4b84f8ae
:10900000225063616423238415f0fafa0948a0f022
:109010008afe00223146084803b0bde8f040f9f767
:1090200045b800bfb0c900106cca0010cc1f0c02bc
:10903000ee82ee00e591000270ca0010012a38b5f8
:10904000044602d10b68236003e0022a03d0032afe
:109050000dd0002038bd0c200d6813f05dfb0346d9
:109060000028f0d095e8070083e80700ebe70068e8
:109070000028eed00c2113f057fbeae7012af8b5df
:10908000064603d10b6803600020f8bd022a08d011
:10909000032af9d100680028f6d0182113f044fb08
:1090a000f2e718200c6813f037fb074630b105468d
:1090b0000fcc0fc594e8030085e803003760e3e7b1
:1090c000012a08bf016000207047012a02d1016017
:1090d00000207047022a04bf0b680360f8e7012aea
:1090e00002d1016000207047022a04bf0b680360b0
:1090f000f8e7012a02d1016000207047022a04bf6c
:109100000b680360f8e7012a02d101600020704774
:10911000022a04bf0b680360f8e7012a02d101604c
:1091200000207047022a04bf0b680360f8e7012a99
:1091300002d1016000207047022a04bf0b6803605f
:10914000f8e7012a08bf016000207047012a08bf24
:10915000016000207047012a70b5054603d10b68f5
:109160000360002070bd022a11d0032af9d10468df
:10917000002cf6d004f1180009f094fb04f108006b
:1091800009f090fb2c21204613f0cefae9e72c20c1
:109190000e6813f0c1fa044688b1338806f108015d
:1091a00003807368083040f8043c09f011fc06f1b4
:1091b000180104f1180009f00bfcb36aa3622c60db
:1091c000cfe7002307b5009342f001033c22fcf7f0
:1091d000ebfc03b05df804fb10b58ab002f0bcfbf9
:1091e000042813d100242023cde90234084b02aa1d
:1091f00000931e2023460749f8f774fe22460649cd
:1092000006480ab0bde81040fff7dbbf0ab010bd4a
:109210007a1a0c0218100c021bda0c02921a0c02b9
:10922000002210b50446044b114640f8043bf8f701
:109230003dff204610bd00bfcc1e0c0210b50446f9
:10924000fff7eeff2046202113f06efa204610bdf6
:1092500010b50446024b0360fff7e2ff204610bd45
:10926000cc1f0c020148fff7f3bf00bf6cca00100f
:1092700010b50446fff7ecff2046242113f054fa02
:10928000204610bd038c8b4211d890f82230013358
:10929000dbb2072b08bf002380f8223090f8222091
:1092a000044b53f8223043616423038470475b1af4
:1092b000fbe700bf401f0c0207b50068036901937c
:1092c00002238df8033083680bb9a0f0d3f9c3688b
:1092d0000df1030201a9984703b05df804fb0000fb
:1092e00070b500242026144b8ab0144d1e2014495a
:1092f000009302aa2346cde90264f8f7f3fd224663
:109300000221286809f0dffd044620b10ab0bde85b
:10931000704009f055bd0b4bcde90260009302aae5
:10932000034607491e20f8f7ddfd2868214609f0ad
:10933000fbfe20460ab070bda81a0c0298ca0010a5
:1093400018100c02c51a0c0230b500248bb023464d
:1093500022460f49cde900440e48fcf765fa234642
:1093600005462246cde9004409490b48fcf75cfa62
:1093700000b155b920220023cde90223074a32204b
:109380000092074902aaf8f7adfd0bb030bd00bf4f
:10939000418d0002db1a0c02e41a0c02ea1a0c02dc
:1093a00018100c022de9f047adf5896d0823002453
:1093b000934d02afdff8d0920022394628683b80f7
:1093c00009f0bffec9f8004002f0c6fa042800f018
:1093d000f3807988204613f00efb0120b98813f042
:1093e0000afb03200ff0a0fd38248046224600210e
:1093f00007f14000a0f0e5feb8f1000f14bf022312
:109400000123a7f8404087f8423000f0f3807d4bfd
:109410007b647d4bbb647d4bbb667d4bfb667d4bac
:109420003b677d4b4ff0000afb647c4b07f17804ef
:109430003b657b4b07f1b4067b657a4b4ff4937227
:10944000bb65794bff21fb65784b30463b66784b1b
:10945000c7f894a07b66774b7b673c232360764bf1
:109460006360764ba360764be360764b2361764b6b
:109470006361764ba361764ba363764b2362764b95
:109480006362764ba362764b6363764be362764b03
:109490002363a0f096fe07f5ee7318464ff4197299
:1094a000ff21a0f08efe10223a820822ba6001222b
:1094b00007f108013a73c7e9050617f0f5fc3046d5
:1094c00017f0dbfc97f8b430ff2b1ad12023c7e943
:1094d000083a664b282000936549534607f120025d
:1094e000f8f700fdb8f1000f05d0624b30461a685e
:1094f0006149a0f03ffed9f8003043f00103c9f8fc
:1095000000300021084612f0fbfd0026c1b2cb1d41
:1095100003f4fc73adeb030d0df10808404612f0a7
:10952000effd4146286807f1400307f11002cde93d
:10953000004609f0abfc334632460221286800960b
:1095400009f007fe1bf0b0feb0f57a7f06d3334674
:10955000012203212868009609f0fbfd002440f653
:109560008c42234604212868009409f0f2fd2e68fd
:1095700017f00afb2346024605213046009409f005
:10958000e8fd2e6817f006fb23460246062130460a
:10959000009409f0defd08233b84384b07f12001dd
:1095a0001b6828687b6209f06bfcfff7cdfe07f5ae
:1095b0008867bd46bde8f087204613f01ffa788023
:1095c000012013f01bfa4ff6ff737988b880994297
:1095d00004d023462246286809f0affd4ff6ff73fa
:1095e000b98899423ff4fdae002328681a4609f075
:1095f000a6fdf6e6224b7b64224bbb6411e700bf5d
:1096000098ca0010ad470002fd470002d4c5001003
:10961000d98b00021d8c00029b8c0002878c0002fb
:10962000698c0002618d01023d8f000253ff01022f
:109630003b8c0002cd8c00020d8b0002198b0002c6
:10964000e9a600022d8b0002398b0002a99a0002c4
:10965000f1a40002f30d0202f70d0202a18900023b
:10966000ed8a000269a20002e9980002061b0c02c2
:1096700018100c0284090c0228090c0294ca00106c
:1096800061470002b147000290ca001010b50023e4
:109690002024144accb01e20134900920aaacde916
:1096a0000a43f8f71ffc00234ff4837219460aa8f7
:1096b000a0f087fd00234ff483711a460aa8fff734
:1096c000cbfa00284ff0000309da084a0190009213
:1096d0003220054902aacde90243f8f703fc4cb059
:1096e00010bd00bf2e1b0c0218100c02441b0c02f4
:1096f00010b5044c236813b909f060ff206020689e
:1097000010bd00bf98ca00102de9f84305464ff080
:1097100050090b4b5f681c7807f10508013c0cd31e
:1097200009fb04f040223e1829464044a2f07efb8b
:109730000028f3d13046bde8f8830026fae700bfe1
:10974000b8c900102de9f84305464ff04c090b4b02
:109750005f681c7807f10808013c0cd309fb04f092
:1097600040223e1829464044a2f060fb0028f3d175
:109770003046bde8f8830026fae700bfc0c90010f4
:1097800010b588b00446684609f0d7f8694604a8c1
:1097900009f01ef904a8a047044604a809f082f8bd
:1097a000684609f07ff8204608b010bd10b50446a1
:1097b000f7f708fb01462046bde810400ff010bb4c
:1097c000f8b500254c27074e3478013c07d3706864
:1097d00007fb04000830fff7e9ff0544f5e72846da
:1097e000f8bd00bfc0c900102de9f84300274ff0b5
:1097f0005009dff8388098f80060013e12d309fb69
:1098000006f5d8f8040028440530fff7cfff0446da
:10981000d8f804000121284404300ff0e1fa204474
:109820000744eae73846bde8f88300bfb8c900102e
:1098300007b5fff7d9ff0090fff7c2ff082101909d
:1098400068460ff0cdfa03b05df804fb10b50c4686
:10985000fff7eeffd4f8e030c4f8d40043f0020381
:10986000c4f8e03010bd70b5142486b02246002143
:1098700001a8a0f0a6fc7826adf804400024002240
:10988000012101a817f089f8bdf80650bdf80c3089
:10989000a34209dd0298202106fb04004c300ff0a2
:1098a0009ffa01340544f1e7002201a8114617f0a0
:1098b00074f8284606b070bd10b50c46fff7d3ff0c
:1098c000d4f8e030c4f8d80043f00103c4f8e03025
:1098d00010bd10b410461a46d1e9103424b1014627
:1098e00020465df8044b184711465df8044b1847b5
:1098f0001b681268fff7edbf07b501680a468b6a5f
:1099000032f8080b009301f118034968fff7f0ffe4
:1099100003b05df804fb30b5c3b04ff4837200218f
:1099200004466846a0f04dfc00234ff483711a46ac
:109930006846fff7b3f9b0f5837f12d1bdf8005048
:10994000b5f5837f0dd1a3680bb99ff093fe6946ef
:109950002046e3689847002329461a466846fff7e1
:109960007bf943b030bd000003291fb515d128b1e4
:1099700001280ed0002005b05df804fb2d4b0393a9
:109980002d4b68460293fff7c6ff6846f9f7d2f8f9
:10999000f0e72a4b03932a4bf3e7022932d102382e
:1099a0000628e7d801a353f820f000bf4999000228
:1099b00053990002f59800025d9900026799000230
:1099c000719900027b9900021e4b009203931e4b7b
:1099d000d7e71e4b009203931d4bd2e71d4b00921d
:1099e00003931d4bcde71d4b009203931c4bc8e71f
:1099f0001c4b009203931c4bc3e71c4b0092039338
:109a00001b4bbee701290cd130b10128b2d105b002
:109a10005df804ebfff727bf05b05df804ebfff737
:109a200007bf0429a6d10428a4d1124b0393124bdb
:109a3000a7e700bfcd970002cd9000023998000241
:109a4000c39000024d8b0002af900002618b0002b8
:109a50009b900002758b000287900002898b0002a8
:109a6000739000029d8b00025f900002b18b000298
:109a70004b900002c58b0002419000022de9f0439b
:109a800002291646984691b03dd10a4601461f4824
:109a9000a0f060fb0446002835d11c2501a8fbf787
:109aa000e7fc2a46214609a8039fa0f08afb21462d
:109ab00009a8adf82450fef7ddfc9df82b201449d1
:109ac00005a808f0c7ffddf81c9007eb0905a845bd
:109ad00013d93a4601993046a0f04cfb4a46059905
:109ae000f019a0f047fb05a808f0dcfe01a808f07b
:109af000d9fe284611b0bde8f08305a808f0d2fed3
:109b000001a808f0cffe0025f3e700bf2d210c02cd
:109b10005c1b0c0208b5fff7f7fd08b1007908bd22
:109b20004ff0ff30fbe7000008b5fff7f3ff013807
:109b3000082896bf014b0220185c08bd351f0c0297
:109b40000138c0b208289abf014b185c0220704748
:109b50002c1f0c02042906d0092907d0012914bfa3
:109b600004200120704718b1f7f72cb9082070477e
:109b70007047000010b5184b8cb01b7803f0ff0045
:109b80001bb1164b1c7814b101200cb010bd16f09f
:109b900020fa134b1b78002bf6d043f69821114a7c
:109ba0001368c31a8b42efd92023cde9043413681c
:109bb0000d49cde901030d4b2820009304aa23464b
:109bc000f8f790f92046234622462146009404f0f7
:109bd0009bfa2046d9e700bfc2c40010acd00010e9
:109be000bfc40010b4c9001018100c02611b0c0295
:109bf00008b5fff77dfd054b186809f05bf918b94a
:109c0000bde80840fff7cebb08bd00bf98ca0010f2
:109c100008b50120f9f7f4fa0920f9f7f1fa002064
:109c200008bd00002de9f04300244ff02008b14b9f
:109c3000b1b01c70b04bb14e20ad2a46b049019076
:109c40000093074623461e20cde92084f8f74af901
:109c50002146306809f021f90d28034657d12346e3
:109c6000032240200021cde901440094fcf7d4fbfd
:109c7000a44ba3492a461e2000932346cde9208405
:109c8000f8f730f9fff7a8fafff7c2ff204616f001
:109c9000d3fa014628b9fbf757fb0146002800f02c
:109ca000e58001f059fe012840f00081964b1b78b9
:109cb000002b40f0fb80954b1868b0b101230a22bd
:109cc000294608f000ff00242023cde91034904bf2
:109cd0001e208b49009310aa23460195f8f702f93c
:109ce000224629468b48fff76cfa00220823306889
:109cf00010a9cde91022adf8403009f0a4fa0446cd
:109d0000002800f0dd8009f05bf80446d4e020b1c3
:109d100031b0bde8f04309f053b802220021cde98b
:109d2000010000900df140094020fcf775fb402137
:109d3000484617f02cf90446b0b99df84030013b75
:109d4000dbb2fd2b10d8744b2a46cde920806c493c
:109d50000093cdf8049003461e20f8f7c3f822467e
:109d600049466e48fff72dfa00234022494618461f
:109d7000009312f0ebf9044690b99df840307bb1a6
:109d80002023cde92030664b2a465d4900930346e7
:109d90001e20f8f7a7f8224649466248fff711fa55
:109da000fff71afa002206200df117018df817208f
:109db000f9f706fa0446002852d19df81730002b17
:109dc0004ed0024601460620f9f7e2f9224607a9dd
:109dd00006a8cde906440ef0f7ff002840d1ddf8d3
:109de0001880b8f1000f3bd05ffa88f3502b079c26
:109df0007bd047d8282b7bd03cd8142b00f0b280e6
:109e00001e2b00f0b1800a2b00f0b0804346464a7a
:109e100040212846a1f00cfab8f1820f01460ed17c
:109e2000631edbb20c2b2844c1f140013bd83f4af2
:109e300052f82330002b36d03d4aa1f0f9f9002426
:109e40002023cde908343b4b1e202d49009308aa5e
:109e50002346f8f747f8224629463748fff7b1f975
:109e6000fff7d6fe0fb1faf714fd0021306809f0b4
:109e700033f916e73c2b7bd0462b7bd0322bc5d158
:109e80002e4b33e0782b77d007d8642b76d06e2b0f
:109e900076d05a2bbad12a4b28e0822b72d08c2b49
:109ea000b4d1284b22e02346274ac6e7fff718fa29
:109eb000044600283ff4ffae204631b0bde8f083f1
:109ec000119b012013f0010f0cd0204b2a46187073
:109ed0002023cde920341e4b094900932346f8f78f
:109ee00001f8e9e71b4b1870e6e71b4b1b4a8fe7ad
:109ef0001b4bfbe7d0c500100f1c0c0298ca0010ca
:109f000018100c02381c0c0244cc001090ca00102f
:109f10001b1d0c02401d0c025f1c0c028e1c0c024f
:109f2000a61c0c02c61c0c028c1b0c02f81e0c0298
:109f3000db1c0c02e01c0c02031d0c02ac1b0c020f
:109f4000fb1b0c020a1c0c028a1b0c02c1c4001071
:109f5000571d0c02c0c40010ee1b0c02dd1c0c02cd
:109f6000e31b0c02084bc1e7084bbfe7084bbde7fa
:109f7000084bbbe7084bb9e7084bb7e7084bb5e719
:109f8000084bb3e7084bb1e78f1b0c02c91b0c024f
:109f90003f6a0c02da1b0c02ce3a0c02a31b0c0225
:109fa000bb1b0c02991b0c02dc030c02024b0021b0
:109fb000186808f074bf00bf98ca001010b5104ba5
:109fc0008ab01b78bbb1fff7f1ff044698b9202394
:109fd000cde902300b4b0c49009302aa034628201e
:109fe000f7f780ff2346224601212046009404f023
:109ff0008bf80ab010bd15f0ecff044b1860f8e7c1
:10a00000c2c40010a01d0c0218100c02b4c900102c
:10a01000f8b50c4616461149054608f08efc264454
:10a02000a64219d02746237828461b0903f13001a0
:10a03000392988bf03f1570108f0ecfc3b7828462a
:10a0400003f00f0303f13001392988bf03f15701f1
:10a05000013408f0dffce3e72846f8bd1bda0c0208
:10a0600000487047c8c900100048704754ca001023
:10a070002de9f0419846057843780446ab420f46f7
:10a08000164690b00bd883781d44ff2d29dc502153
:10a0900040686943a1f016f818b3606065702378d2
:10a0a000626803eb830502eb05150133502241463c
:10a0b00023702846a0f05ef80c210223cde9051399
:10a0c00009f07cfa002205a909f0baf8c0b9bdf878
:10a0d0001e20bdf81c309a421dd223780bb1013be3
:10a0e000237000252023cde908350d4b3220009345
:10a0f000cde901672b460b4908aaf7f7f3fe0ae002
:10a1000020220023cde90823074a1e20009205499a
:10a1100008aaf7f7e7fe284610b0bde8f08100bfb7
:10a12000ed1d0c0218100c02cf1d0c02f0b50f46ed
:10a1300016461c4695b005464c22002101a8a0f009
:10a1400040f800978df8046034b163681293238857
:10a150000b2b84bfa36813932b460df1050205f169
:10a16000400153f8040b8b4242f8040bf9d1284606
:10a17000fff7cafa044648b96b462946064a07481b
:10a18000fff776ff0446204615b0f0bd5022694621
:10a190009ff0f0fff7e700bf1a1e0c02b8c90010cd
:10a1a0002de9f0419846057843780446ab420f46c6
:10a1b000164690b00bd883781d44ff2d27dc4c2128
:10a1c00040686943a0f07eff08b3606065704c2270
:10a1d00020786568414600fb025501302070284612
:10a1e0009ff0c8ff0c210223cde9051309f0e6f921
:10a1f000002205a909f024f8c0b9bdf81e20bdf859
:10a200001c309a421dd223780bb1013b23700025ec
:10a210002023cde908350d4b32200093cde90167ad
:10a220002b460b4908aaf7f75dfe0ae0202200231f
:10a23000cde90823074a1e200092054908aaf7f72e
:10a2400051fe284610b0bde8f08100bfed1d0c02a4
:10a2500018100c02cf1d0c0270b50c4694b04422ad
:10a260000546002103a89ff0acffa36803aa029350
:10a27000e3680193636803f140061446186859685f
:10a28000083303c4b3422246f7d12846fff75afaef
:10a29000044630b14c2201a99ff06cff204614b057
:10a2a00070bd2946034a044801abfff779ff044615
:10a2b000f4e700bf231e0c02c0c9001038b5846843
:10a2c00005465cb144684cb12046f6f77bfd40285a
:10a2d00008d820462946fff7bfff0446201e18bfb6
:10a2e000012038bd0024f9e7f0b50c461d46096c85
:10a2f0003d4ba5b0994206462a9f08d12b462146e0
:10a3000030462a9725b0bde8f040fff7e2ba0020ba
:10a31000019201f02dfb019a0028efd0114602a80e
:10a3200008f00bfb294606a808f007fb2f4b93f813
:10a330002c203ab906a808f0b5fa02a808f0b2fa3b
:10a3400025b0f0bd586a1af0b2fd05460028f1d1db
:10a3500002a910a80f94adf8386008f039fb06a9df
:10a3600014a808f035fbbdf8383010a9adf86430fa
:10a370000f9b1ba81a93189708f02afb14a91fa873
:10a3800008f026fb189b2c2023930c9512f0c4f99f
:10a39000044680b1bdf864301ba903801a9b0830c5
:10a3a00040f8043c08f0fafa1fa904f1180008f07c
:10a3b000f5fa239ba3620e4b1fa80d930d4b0a9435
:10a3c0000c9308f06ffa1ba808f06cfa0aa907486a
:10a3d000f9f7b8fd0aa8f8f7adfb14a808f062fa7f
:10a3e00010a808f05ffaa5e7418d0002c4cb001069
:10a3f00079980002d79000022de9f0431f46194bcf
:10a40000164693f82c2085b00446dde90c890d46ec
:10a41000eab1586a1af04bfdc8b90290182012f040
:10a420007bf928b1c0e90045c0e90267c0e90489a9
:10a430000d4b694603930d4b00900a480293f9f7c0
:10a4400081fd6846f8f776fb05b0bde8f0833b4632
:10a45000324629462046c446cdf8309005b0bde8c6
:10a46000f0436047fcc50010f1a30002fd8f00021d
:10a4700007b500684369019303690093d0e902239b
:10a48000d0e90001fff7b8ff03b05df804fb00005e
:10a490002de9f041304b174693f82c2004460e4628
:10a4a00088b0d2b1586a1af002fdb0b906900c20fb
:10a4b00012f032f910b1c0e900468760274b0490d2
:10a4c0000793274b244804a90693f9f73bfd04a8fa
:10a4d000f8f730fb08b0bde8f0810023cde9033385
:10a4e000e36c25688bb1284603aa04a99847002885
:10a4f00025da00231e201a461946cde90067fff72a
:10a500007bff04989ff010fee4e7d4f84880b8f190
:10a51000000f04d02a462179601dc0470546284611
:10a520002179fff717fb8046039040b19ff0f4fdbf
:10a5300004900028ddd0424629469ff01bfe20797a
:10a54000fff7fefadde903320146cde9006700209e
:10a55000fff752ffbee700bfc4cb0010e5a4000226
:10a56000bd8f000203681868d3e90112fff790bf9e
:10a5700037b50c461546fff7c7f8034630b12a46f3
:10a58000214603b0bde83040fff782bf02460146d6
:10a5900000951d20a04703b030bd38b5002383606f
:10a5a0008b6804460d462bb102229847eb68e360a6
:10a5b000ab68a360204638bd012a70b5054603d1bb
:10a5c0000b680360002070bd022a0dd0032af9d168
:10a5d0000468002cf6d004f10800f8f7abfa182153
:10a5e000204612f0a1f8ede718200e6812f094f85a
:10a5f000044648b1336806f1080103607368083007
:10a6000040f8043cfff7c9ff2c60dbe7012a70b576
:10a61000044603d10b680360002070bd022a0cd0f1
:10a62000032af9d10468002cf6d02046f8f782fa04
:10a630001421204612f078f8eee714200e6812f08c
:10a640006bf8054620b13146fff7a7ff33692b6150
:10a650002560e1e713b56c460b460246d0e90001e0
:10a6600084e8030093e8030082e8030094e8030011
:10a6700083e8030002b010bdf0b517461c46002267
:10a6800043688fb000680d469847064627b11db154
:10a690000121284612f048f8264b93f82c20002a76
:10a6a00039d0586a1af003fc0546002833d12146f8
:10a6b00004a8fff772ff04a909a80896fff76dff29
:10a6c000089b14200d93029512f026f8044670b1f1
:10a6d0000146856009a8fff7bdff0b9ba268a36038
:10a6e0000c9b0b92e268e3600d9b0c922361124b72
:10a6f00009a80393114b00940293f8f71bfa6946db
:10a700000c48f9f71ffc6846f8f714fa04a8f8f7a4
:10a7100011fa0fb0f0bd02238df81030a36809962e
:10a720000bb99ef0a7ff2046e36804aa09a9984741
:10a73000efe700bffcc50010399200028da50002b2
:10a7400030b5016885b0d1e9004568460831fff7aa
:10a7500024ff6b46012229462046fff78dff6846fd
:10a76000f8f7e8f905b030bdf0b591b00d461746e1
:10a77000fef7e8ff0446002855d02846a0f000fe6a
:10a780002a4b064693f82c20002a40d0586a1af02b
:10a790008efb054600283ad1394606a8cde9044685
:10a7a000fff7fbfe049b06a90a93059b0ca80b93dd
:10a7b000fff7f3fe1820029511f0aeff044688b1b2
:10a7c0000a9b056103600b9b00f1080143600ca824
:10a7d000fff740ff0e9b226923610e920f9b626977
:10a7e00063610f92124b0ca80393124b00940293d7
:10a7f000f8f7a0f969460d48f9f7a4fb6846f8f7a1
:10a8000099f906a8f8f796f9002011b0f0bd39467d
:10a810000aa8fff7c2fe2046012231460aabfff725
:10a820002bff0aa8eee74ff0ff30eee7c4cb001095
:10a83000c1a6000239a500022de9f8434ff4a02279
:10a8400000254ff014082b4b2b4cc3e900252b4b54
:10a850000a21c3e900252046294afbf767ff294b57
:10a86000294a1e2104f11c002360a561fbf75eff4d
:10a87000264bdff8c090e361254b264fc4e90f83d8
:10a88000254b2946636404f13c0004f13803a364ba
:10a890006563c4f83890e764f7f7a2fd1f4b204ebc
:10a8a000e365204b2946236604f1580004f1540364
:10a8b000c4e91937c4e91459a663c4f85880f7f7f6
:10a8c0008ffd194a0d2104f170006665e566fbf7fe
:10a8d0002dff47f23052154bc4f888502367144bb4
:10a8e000c3e903551d705a601d725d729d82bde8fb
:10a8f000f88300bfb8c90010c8c90010c0c9001053
:10a900002c1e0c02e01e0c02371e0c02f01e0c0264
:10a910000e0002007b640002461e0c021d000200b5
:10a9200008150c02521e0c02601e0c0218150c02b7
:10a9300054ca0010bc140c0209490c2008b59ef042
:10a9400095fe014650b1074b036000238360064b20
:10a950004360bde808400548fcf79cbc08bd00bf4b
:10a96000751d0e02d4150c02f1a8000274d000105f
:10a9700010b510b103685b689847faf753fd40b112
:10a98000fef7b6febde81040002304211a4608f089
:10a9900040bc10bdc0e8af1f7047002108b503469a
:10a9a000c0e9001101620a460830c0e8af1f03f198
:10a9b0000c00fff7efff03f11000fff7ebff03f1cf
:10a9c0001401c1e8af2f03f11801c1e8af2f012135
:10a9d00003f11c02c2e8af1f184608bd10b50a4caf
:10a9e000d4e88f3fdb070cd4204613f0cffd40b1f5
:10a9f0000648fff7d2ff204613f002fe04489ff0fe
:10aa000092f9024810bd00bf9cca0010a0ca0010f5
:10aa1000b5a9000210b50446006818b11ff0e8ffa0
:10aa200000232360606818b11ef0eefc0023636011
:10aa300010bd00000148fff7edbf00bfa0ca001025
:10aa40000c30d0e8af0f831e584258417047103089
:10aa5000d0e8af0f831e5842584170471fb51c30d5
:10aa6000d0e8af3f022b0fd193681b78022b0bd19c
:10aa700000230522cde90133009320200021fbf7bc
:10aa8000cbfc05b05df804fbd0e8af3f002bf8d15c
:10aa900092681278012af4d10322cde901330093a0
:10aaa000ebe773b50024054601a801941ef08efb68
:10aab000a04219db0198264603465bb15a682ab1c9
:10aac0005278022a04d00a2a08bf01241b68f4e73e
:10aad0000126fbe71ef072fb05f11403c3e8af6f1c
:10aae00005f11803c3e8af4f02b070bd002307b5ee
:10aaf000084669460093adf804301ff0dcfa0222e4
:10ab000068460649a1f092f930b90ef0e7fe0ff061
:10ab1000abfa03b05df804fb0120fae7d81f0c0282
:10ab2000f7b506460c4611bb684600911ff08ef83b
:10ab3000002819db2746009d9db1686878b101a9fe
:10ab400001971ff0baf9002809db019b1b0706d407
:10ab500030466968fff7caff002818bf04462d6811
:10ab6000eae700981ff09ef8204603b0f0bd03b05e
:10ab7000bde8f040fff7babf2de9f0430e4689b0bb
:10ab80000021fff7cdff4ff00008002845d004a8b2
:10ab9000cdf810801ff05af8404504da204c2046ca
:10aba00009b0bde8f083049d1d4cdff878902db30b
:10abb000686808b305a9cdf814801ff07ef9002855
:10abc0001adb059b13f0080316d16f6806a93846f7
:10abd0000693adf81c301ff06efa0eb1be420bd1d9
:10abe0000222494606a8a1f021f9074620b90ef035
:10abf00075fe3c460ff02afa2d68d8e704981ff03e
:10ac000051f8002ccbd12346022210200021cde99f
:10ac100001440094fbf700fcc1e70446bfe700bf16
:10ac2000f2feffffd81f0c02006a20b183688b423e
:10ac300001d00068f9e77047f0b5002585b01646e9
:10ac40000c468df8075031bb02a802911ef0feffa2
:10ac5000a8421ddb2746029dbdb1686898b103a9d3
:10ac600003971ff02af900280ddb039b1a070ad46b
:10ac700068680df107011ff038ff20b99df8073013
:10ac8000b34208bf01242d68e6e702981ff00af8d6
:10ac9000204605b0f0bd20460df107011ff025ff4d
:10aca00028b99df80740a31b5c425c41f0e72c46a5
:10acb000eee77fb500250c46019539bb02a802914d
:10acc0001ef0c4ffa8421edb2646029dc5b168687f
:10acd000a0b103a903961ff0f0f800280edb039b38
:10ace00013f008030ad1686801a901931ff054f812
:10acf00020b9019b13f4801f18bf01242d68e5e7dc
:10ad000002981ef0cfff204604b070bd204601a976
:10ad10001ff042f818b9019cc4f30054f3e72c4625
:10ad2000f1e738b5022204460d46fff785ff28b14a
:10ad300029462046bde83840fff7bbbf38bd38b5cf
:10ad4000012204460d46fff777ff30b12946204621
:10ad5000fff7afff80f00100c0b238bd08b5fff7c4
:10ad600063ff00b1007908bd2de9f043002485b0f0
:10ad7000064602a80f4602941ef068ffa04224db9c
:10ad8000a146029df5b16868d0b103a9cdf80c9039
:10ad90001ff093f8002813dbddf80c8018f0080f83
:10ada0000ed1696830460191fff7a0fe40b13046f0
:10adb0000199fff7d3ff18b137ea080308bf013440
:10adc0002d68dfe702981ef06dff204605b0bde854
:10add000f08370b505460026046a4cb123792bb187
:10ade0002846a168fff782fe00b101362468f4e727
:10adf000304670bd08b5fff717ff10b10c30d0e832
:10ae0000af0f08bd08b5fff70fff10b11030d0e845
:10ae1000af0f08bd0a4608b5036a73b112b199684d
:10ae2000914208d103f10c000021fff7b3fd03f1bb
:10ae30001000fff7affd1b68efe708bdd0e8af0fcc
:10ae4000704708b50830fff7f9ff013818bf012037
:10ae500008bd08b50830fff7f1ff043802288cbfa1
:10ae60000020012008bd08b50830fff7e7ffc31f29
:10ae70005842584108bd2de9f3410546fff7e9ff67
:10ae800058b14ff000086846cdf800801ef0defe95
:10ae9000002808da02b0bde8f0812846fff7e3ff9a
:10aea0000028eed1f6e7009c7cb3606820b301a9ce
:10aeb000cdf804801ff001f800281ddb019f3b073f
:10aec0001ad4666828463146fff710fea0b1314615
:10aed0002846fff7a9fe78b1037907f001076bb1a7
:10aee00057b9012130461ff041f8002804db4ff428
:10aef000803130461ff093f82468d5e7002ffbd04f
:10af0000012130461ff05ff8f6e700981ef0cafef8
:10af10002046bfe708b50830fff790ff08bd0000e6
:10af2000f0b500f1080504468db028460e46fff73f
:10af300085ff072813d1072e00f0e580002104f1da
:10af40000c00fff727fd04f11000fff723fd04f1cb
:10af50001402c2e8af1f04f11802c2e8af1f731e4b
:10af6000062b1ed8dfe803f00439698793c8cf00a9
:10af7000002704f11c03c3e8af7f2a213b463a4671
:10af80003846faf703ff3b46022200212020cde994
:10af900001770097fbf740fafbf7e4fb00f1180399
:10afa0001f60202300272846cde90437fff746ff1e
:10afb000634b644953f8262053f8203002920193e2
:10afc000614b1e20009304aa3b46f6f78bff04f169
:10afd0000803c3e8af6f0db0f0bd00232a211a4665
:10afe0000120faf7d3fefbf7bdfb022200f11803a4
:10aff0001a602846fff722ff03280ed1072204f12a
:10b000001c03c3e8af2f00230b22cde901330093cb
:10b0100020200021fbf700fac3e72846fff70effc8
:10b020000128bed1022204f11c03c3e8af2f002384
:10b030000422cde901330093eae7062204f11c0360
:10b04000c3e8af2f2846fff7f9fe072803d1fbf727
:10b0500089fb0023c36600230a22cde90133009354
:10b0600020200021fbf7d8f9fbf77cfb052200f13b
:10b0700018031a6095e700232a211a460220faf7de
:10b0800085fefbf76ffb032200f11803f1e70422b2
:10b0900004f11c03c3e8af2f2846fff7cffe0728b3
:10b0a0000fd1fbf75ffb012200f134031a60fbf7bd
:10b0b00059fb07460df09cfc3b6d01333b650df0e1
:10b0c0009bfc00232a211a460220faf75ffe002388
:10b0d0000622cde90133009300212020fbf79cf9e3
:10b0e000fbf740fb032200f118031a60fbf73afb61
:10b0f000c36e0133c36654e700232a211a46032096
:10b10000faf744fe4de7052204f11c03c3e8af2f14
:10b1100000232a211a460420faf738fefbf722fb07
:10b12000042200f118031a602846fff787fe07285b
:10b130003ff437af00230722cde90133009367e7df
:10b14000fc200c02db1f0c02e51f0c0210b503688b
:10b15000044623b9014608481ff03afc20606368a2
:10b1600023b9214605481ef039f960602046bde844
:10b1700010400121fff7d4be5db6000251b40002b9
:10b1800010b504460830fff759fe012803d102210b
:10b190002046fff7c5fe6ff0d10010bd10b5044684
:10b1a0000830fff74bfe012808d0022803d1012107
:10b1b0002046fff7b5fe6ff0d10000e0002010bd83
:10b1c0002de9f74307460830fff738fe02284bd138
:10b1d000002504213846fff7a3fe684600951ef0bf
:10b1e00035fd041e37db2c46a946ddf80080b8f19a
:10b1f000000f2bd0d8f8040028b301a9cdf8049093
:10b200001ef05bfe00281edb019e32071bd4d8f81f
:10b21000045038462946fff769fca0b12946384654
:10b22000fff79cfd78b1f3070dd4012128461ef0ed
:10b230009dfe002807db4ff4803128461ef0effe0c
:10b240000028a8bf0134d8f80080d0e700981ef08d
:10b2500029fd24b14446204603b0bde8f083052112
:10b260003846fff75dfef6e76ff0d104f3e7f7b578
:10b27000054608300c46fff7e1fd0138012846d9a4
:10b280002846fff7f0fd88b1fbf76cfa06466cb173
:10b2900000f134031c60012c01d0062c06d10df006
:10b2a000a7fb336d013333650df0a6fb00270321a7
:10b2b0002846fff735fe684600971ef0c7fc041ebf
:10b2c0001ddb3c46009eaeb1706888b101a90197b4
:10b2d0001ef0f3fd00280bdb019b1a0708d4db07e7
:10b2e00006d5012170681ef06efe0028a8bf01344b
:10b2f0003668e8e700981ef0d5fc1cb134462046bd
:10b3000003b0f0bd02212846fff70afef7e76ff011
:10b31000d104f4e710b5936804461b78083093b164
:10b32000fff78cfd04281ad105212046fff7f8fd10
:10b3300040212046fff718fd88b106212046bde8d0
:10b340001040fff7edbdfff779fd032807d101217c
:10b350002046fff709fd012801d80221eee710bdc4
:10b360002de9f347002700210646fff753fd684605
:10b3700000971ff0cbfab842c0f28580b846ddf8de
:10b380000090b9f1000f56d0d9f8083013f0080436
:10b3900034d103f04103412b30d1d9f80c306bb3d9
:10b3a000196859b34d78022d2bd11a7c002a3fd051
:10b3b0009b68002b3ad0a845b8bfa84699f8100062
:10b3c000a74201a9b8bf27461ef0b2fcb0b930466b
:10b3d0000199fff729fc034680b10c30d0e8af2f6c
:10b3e000954202dd2946fff7d5fa03f11000d0e8b7
:10b3f000af3f9c4202dd2146fff7ccfad9f800901e
:10b40000bfe70a2d15d1da681c7c8b6943b984b17a
:10b4100072b1147814f002040bd002240025cae79c
:10b420003cb12ab11478c4f34004f7e71c46f5e7b1
:10b4300000242546bfe700981ff07bf806f10c0ab0
:10b44000dae8af9f06f11004d4e8af5f3046fff7ab
:10b4500028fb41465046fff79dfa39462046fff744
:10b4600099fab8f1020f11d0022f16d0002406f17c
:10b47000080a5046fff7e2fc072816d1acb90621ae
:10b480003046fff74dfd02b0bde8f08706f114032a
:10b49000d3e8af4f012ce7d1e9e706f11803d3e871
:10b4a000af4f631e5c425c41e1e75046fff7c6fccc
:10b4b000062800d154b95046fff7c0fc0728e2d156
:10b4c000002ce0d0c84501d1af42dcd00721d7e73e
:10b4d000fff746bf38b5936804461b7800f10805ae
:10b4e000d3b12846fff7aafc052807d1062120463c
:10b4f000fff716fd2046fff733ff09e02846fff768
:10b500009dfc0728f6d02846fff798fc0628f1d0c6
:10b51000bde83840fff710bafff77cfc2846fff77c
:10b520008dfc07280ad141212046fff71dfc002889
:10b53000e0d105212046fff7f3fce9e72846fff7b5
:10b540007dfc0628e4d1eee738b500f10805044695
:10b550002846fff773fc072806d12046fff700ffb7
:10b56000bde83840fff7e8b92846fff767fc062832
:10b57000f6d1f2e7d0e88f0fc0b2704770b58cb04b
:10b58000fff752fb0e46044670b92023cde9043084
:10b59000254b2649009304aa03463220f6f7a2fc65
:10b5a0006ff0a9000cb070bd00f114051ab30223ae
:10b5b00028468df80c30fff7ddff022807d028461b
:10b5c000fff7d8ff042802d00422c5e88f2f2021de
:10b5d0000023cde90413164a0092012004aa13495e
:10b5e000f6f780fc0023009301233046194603aa96
:10b5f0001ff030fad6e7012328468df80c30fff70c
:10b60000b9ff012809d02846fff7b4ff032804d06a
:10b61000032204f11403c3e88f2f20220023cde975
:10b620000423044ad8e700bffd1f0c02db1f0c02f5
:10b6300018200c023a200c02f0b58fb00d461646c9
:10b64000fff7f2fa60b92023cde90630164b17490f
:10b65000009306aa03463220f6f744fc0fb0f0bd73
:10b6600000f114073846fff785ffb3681b7898424e
:10b67000f4d0c7e88f3f0df1170128461ef0fffbfd
:10b68000202200239df81710cde90623d7e88f2f3d
:10b69000d2b2cde90112064a01200092034906aa5e
:10b6a000f6f720fcdae700bffd1f0c02db1f0c02df
:10b6b0005d200c021368033b052b0ed8dfe803f076
:10b6c0000305070d090bfff725befff703bffff7c3
:10b6d0003bbffff7b1bffff7c1b97047fff7eabf44
:10b6e00000232de9f04f93b0054608a80591089373
:10b6f0001ef0acfa00285fdb089cdff8c8a0dff87a
:10b70000c8b0002c55d06068002850d0002309a98b
:10b7100009931ef0d2fb002849db099b13f00808af
:10b7200045d1666828463146fff77efa074680b95c
:10b73000594618209df09aff0746002837d02b6afb
:10b74000c0e9038880f8048080f814808660036074
:10b750002862059b30463b7100230df11e018df8d8
:10b760001e301ff0c2f9814608bb07f1140840469d
:10b77000fff700ff9df81e10884218d0c8e88f1f01
:10b780000df11f0130461ef07afb20229df81f109c
:10b79000cde90a29d8e88f2f094bd2b2cde90112a1
:10b7a000009351464b4601200aaaf6f79bfb2468fa
:10b7b000a7e708981ef076fa13b0bde8f08f00bf37
:10b7c00082200c02db1f0c02751d0e0210b521b980
:10b7d0000121fff785ff002010bdfff725fa10b10a
:10b7e00001230371f7e76ff0a900f5e770b505468f
:10b7f0000c461646faf7b6ff00f134031e602146e8
:10b8000028461cb9fff76cff204670bdfff70cfa05
:10b8100010b100240471f7e76ff0a900f5e7f7b560
:10b82000174613f0010205460e461c4605d10b468d
:10b8300001200521009202f067fc032d0ad0042d9f
:10b840000cd0022d0dd1c4f340000df063fa00209e
:10b8500003b0f0bd00200df045faf8e70df030fa26
:10b86000f5e70022394630460df01cfaefe7006894
:10b870000179d0e902230078fff7d1bf012a70b522
:10b88000054603d10b680360002070bd022a08d072
:10b89000032af9d100680028f6d0102110f044ffe7
:10b8a000f2e710200e6810f037ff044618b196e852
:10b8b0000f0084e80f002c60e6e7000010b50124bb
:10b8c00000220d4b1c700d4b1a70fef7cdfbd0e81b
:10b8d000cf3fc0e8424f002af9d1dbb2002bf6d1ae
:10b8e000c2680361c36003754375c0e88f3fd30727
:10b8f00058bf037a10bd00bf6051001002c900108c
:10b900000022014b1a70704760510010024b1878ea
:10b91000003818bf01207047605100100b4b28b948
:10b920001a788ab901221a70fff7c8bf0328187065
:10b9300008d80128f8d00022054b1a700122054bc7
:10b940001a7001e00428efd0704700bfc5ca00108c
:10b950006051001002c90010014b1878704700bff9
:10b96000c5ca0010014b1870704700bfc4ca001050
:10b97000014b1878704700bfc4ca0010f0b51c46d0
:10b98000431e032b06460d46174685b04fd8294a5d
:10b99000d35c002908bf1d46274b5b68c3f308032f
:10b9a0005bb144f00104e9b223463a46f0b2fff736
:10b9b00036ff0025284605b0f0bdf9f733fd002815
:10b9c000efd0fef751fb037a002bead0e307ead46d
:10b9d0001a4b93f82c20002ae5d0586a19f067fa20
:10b9e0000028e0d10290102010f096fe18b1c0e9b6
:10b9f0000065c0e90274124b00900393114b694635
:10ba00000e480293f7f78ef9044670b100224ff00a
:10ba1000ff31406919f064fb236820469b68a569e3
:10ba200098476846f7f786f8c4e70546f9e7064df4
:10ba3000c0e700bf1c210c0200ed00e0fcc50010b7
:10ba4000efb70002fdb70002f2feffff704701767c
:10ba50007047417670470368db69184780f8251006
:10ba600070478163828770470164a0f84420704763
:10ba70008164a0f84c207047c161704710b503681d
:10ba80001446db689847031b5842584110bd08b55f
:10ba90004068fff7f3ff08bd70b5037a04460d4612
:10baa00016462bb9d0e90312fff7f1ff01232372e9
:10bab000324629462046fff7eaff70bd70477047bf
:10bac00070470139012908b505d800211030f7f772
:10bad000cffb012008bd0020fce713b50446084653
:10bae0000191f5f76ff9013082b220462368019980
:10baf0001b6b02b0bde81040184713b5044608465a
:10bb00000191f5f75ff9013082b22046236801996f
:10bb1000db6a02b0bde81040184713b5044608467a
:10bb20000191f5f74ff9013082b22046236801995f
:10bb30009b6a02b0bde81040184710b5044608469d
:10bb4000216311b9a086204610bd002a02daf5f75c
:10bb500039f9f7e7a286f6e710b504460846a16270
:10bb600011b9a085204610bd002a02daf5f72af99e
:10bb7000f7e7a285f6e710b504460846a16011b9bb
:10bb8000e060204610bd002a02daf5f71bf9f7e75e
:10bb9000e260f6e710b504460846216111b960611c
:10bba000204610bd002a02daf5f70cf9f7e76261ca
:10bbb000f6e7002201211046fbf7beb90022012161
:10bbc0001046fbf7b9b910b50446502110f0acfd92
:10bbd000204610bd10b50446242110f0a5fd2046d6
:10bbe00010bd10b504468c2110f09efd204610bdfe
:10bbf0004c22002104309ef0e4baf8b504460d460c
:10bc0000d1b1c8b190f82570b7b101f12406304622
:10bc1000f5f7d8f887423a4604f1040138bf0246e6
:10bc20003046a0f003f938b994f82c3085f8883004
:10bc300094f82d3085f88930f8bd002108b5022030
:10bc400002f0fefc19f023fab0fa80f0400908bdba
:10bc500008b50021022002f0f3fcbde8084019f00d
:10bc60001eba38b500f1100504462846fff7e5ff77
:10bc7000e8b1284606f0ebfbb0b1284606f0d8fb49
:10bc8000011e11db236820465b69c9b2984758b989
:10bc9000284606f0dcfb38b1284606f0c1fb2368d5
:10bca000c1b21b69204698472846fff7d1ff38bd2f
:10bcb00038b50c460546014620469ef05bfa2846fc
:10bcc0001349f5f775f828b9124920469ff03ffb54
:10bcd000002038bd28461049f5f76af808b90f4921
:10bce000f3e728460e49f5f763f808b90d49ece784
:10bcf00028460d49f5f75cf808b90c49e5e72846f0
:10bd00000b49f5f755f80028e2d10a49dde700bff5
:10bd100020210c0225210c022a210c0230210c02c8
:10bd2000431e0c0236210c0244210c0247210c0256
:10bd300055210c025c210c0238b503460446124a18
:10bd400004f1100543f8042b07c983e807002846cf
:10bd500006f0c4fb0021022002f072fc19f090f9f9
:10bd60002846fff775ff284606f0acfb20b94ff4d4
:10bd70001651284606f0a2fb044b20462360ff2301
:10bd8000a4f8883038bd00bf84240c0210250c02b2
:10bd90004ff0ff30704770b50d46002400f11006db
:10bda0002846f5f70ff8a04205d9295d304606f080
:10bdb00055fb0134f4e770bd38b5044600f11005b9
:10bdc0002846002306f098fc20460649fff7e3ffcb
:10bdd000284606f03cfb002803dd284606f020fb41
:10bde000f6e738bdb8230c022de9f0436929044673
:10bdf000a5b070d1142500212a4607a89ef0e1f9cc
:10be00000022012107a8adf81c500df09bfc002575
:10be10002023cde90c35bdf82c3001200193914b46
:10be2000914900930caa2b46f6f75cf8bdf82c302c
:10be3000002b3fd08d492046fff7adff03a8f9f74f
:10be400017fb20460399fff7a6ff20468849fff716
:10be5000a2ff2427dff85c82dff81492bdf82c30b3
:10be6000ab421cdd07fb05f60a9b142298590ca96e
:10be7000fff71eff88b920460ca9fff78cff41464b
:10be80002046fff788ff0a99204631440431fff726
:10be900082ff49462046fff77eff0135dee703a813
:10bea00006f000fd002207a811460df04bfc25b05e
:10beb000bde8f0836f492046fff76dff0ca8f9f746
:10bec000d7fa20460c99fff766ff20466849fff72e
:10bed00062ff0ca8e4e76d293ed16749fff75bffdd
:10bee0005d2200210ca89ef06cf90022042011466e
:10bef000faf7ecfd014638b102882ab15d2a28bf65
:10bf00005d220ca89ef036f901220df1870107a8e9
:10bf1000fef77ef820460799fff73dff07a806f0d9
:10bf2000c1fc0525554f0df18d0639462046fff71a
:10bf300032ff0122711b07a8fef76af82046079915
:10bf4000fff729ff07a806f0adfc013dedd1204623
:10bf50004749fff720ffaae766290bd11034204696
:10bf6000474906f03dfc0021204625b0bde8f043de
:10bf7000f7f77eb9782905d10368db6825b0bde8fd
:10bf8000f0431847732919d13e4b00220f93012328
:10bf900010933d4b1034119303230d943b4c0ca98b
:10bfa0003b488df838200c941293fcf739fddde9fd
:10bfb00011120ca80c94fff76ffd78e7762908d1d1
:10bfc000344b0c9300f110030ca80d93fcf74afdc1
:10bfd000bde74c290ad1002201210420f7f7d8f847
:10bfe000002025b0bde8f04306f0c3bd632910d1a1
:10bff000002014f0deff054627492046fff7cbfe60
:10c000002649274b002d08bf19462046fff7c3fedf
:10c010009de7432917d12349fff7bdfe3f22204664
:10c020000ca9fff7c9fe0ca8f4f7ccfe3f2808d1f5
:10c030000ca814f07fff1c492046fff7acfe0ca9aa
:10c04000e3e71a49e1e764297ff431af002200f108
:10c050001003009311461046154b0192fcf70afda0
:10c0600075e700bf76210c0218100c0296210c0215
:10c07000b8230c02a2210c02b5210c02520f0c02b3
:10c08000d2210c02d6340c0212220c0204250c021e
:10c09000dd3b0002f8240c0216220c026f210c0278
:10c0a00073210c0227220c0243220c0257220c029d
:10c0b000fdb90002cb220c022de9f041044600f14b
:10c0c0002407bab021220021384604f145059ef02c
:10c0d00078f84122002128469ef073f8ff230021c2
:10c0e000a4f88830674b4c22a4f8861027a8269322
:10c0f0009ef067f8dff8bc8104f1860641462046d1
:10c10000fff749fe202239462046fff755fe94f8f6
:10c110002430002bf2d021465b480ef01dfe94f82f
:10c120008830ff2b12d1dff8908141462046fff77f
:10c1300032fe012231462046fff73efe94f886305b
:10c14000303bdbb2032bf0d884f8883094f8883089
:10c1500013b1312384f845304ff0ff32394626a819
:10c16000fff709fd4ff0ff32294626a8fff712fd21
:10c17000b4f888304c22adf8b030032327a90deb7a
:10c1800002008df8bc3027929df0f4ff4c226846e7
:10c190000deb02019df0eeff01226946a368e06805
:10c1a0009847023002d094f88930e3b9374f3946c6
:10c1b0002046fff7f0fd012231462046fff7fcfd47
:10c1c00094f88620a2f13103022bf0d8322aa2f192
:10c1d000300302d0032b18bf012384f8893094f870
:10c1e00089308df8b13094f88830013b022b0ed89d
:10c1f00020462749fff7cffd402229462046fff77a
:10c20000dbfd4ff0ff32294626a8fff7c3fc20468e
:10c210002049fff7c0fd4c22032327a90deb0200a4
:10c220008df8bc3027929df0a5ff4c2268460deb9f
:10c2300002019df09fff00226946a368e0689847cd
:10c24000f0b920461449fff7a6fd20461349fff731
:10c25000a2fd20461249fff79efd20461149fff737
:10c260009afd11492046fff796fd10492046fff739
:10c2700092fd236820469b6998473ab0bde8f0815b
:10c280000b49f3e7a8240c027bbb0002ce220c0270
:10c29000fa220c0205230c0238230c0258230c024c
:10c2a00088230c02bb230c02fa230c022e240c025e
:10c2b00047240c029a220c02a1220c02772908b50d
:10c2c00003d1bde80840fff7f7befff78dfd08bdbd
:10c2d000d0e88f0fc0b2003818bf012070470000af
:10c2e00000487047c8ca001008b5fff7f1ff08bd45
:10c2f0007fb50546fff7ecffe0b1686810b1036851
:10c300009b68984713f065feeb68c01ab0f57a7f1a
:10c310000ed313f05efe00240646aa682346821a56
:10c3200000210420cde901440094faf775f8ee608d
:10c33000002001e06ff0d10004b070bd38b51420ca
:10c340000d460021144602f053f9014640b1054b59
:10c350000573046143600448faf79cff002038bd70
:10c360000248fce751c5000274d00010fcfeffff3c
:10c3700010b514466ab971b1134604200a46214625
:10c38000faf7a6fc002805db224602210348fff746
:10c39000d5ff002010bd0846fce700bfc8ca00104a
:10c3a00030b58bb0fff794ff002857d0002420232e
:10c3b000cde902342b4b1e202b49009302aa2346c1
:10c3c000f5f790fd21460920f9f794fd08b30469bb
:10c3d000002214210120f9f797fd282202210346ab
:10c3e000cde9002102a82146012206f0e5fb00224a
:10c3f000012103a8f5f75afe1a24013c0bd09df841
:10c400001a30322083f002038df81a3011f045f80b
:10c41000f3e7ff24dce7fef7e1fa2146fef7acfb89
:10c420000446a8b14ff47f031a2507939df81a30ec
:10c4300003f0fd038df81a30013d09d09df81a3044
:10c44000322083f002038df81a3011f026f8f3e75a
:10c4500002a8fcf7e5fe20460bb030bd6ff0d1041a
:10c46000f9e700bf3a250c022c250c020368016095
:10c470001bb11a68184652681047704730b58db026
:10c480000546fff769fa042807d12846fff720ff81
:10c49000044650b16ff0d10049e009200cf044fd92
:10c4a0000028f2d06ff0810041e00123c5e88f3f02
:10c4b0002023cde904301f4b1f49009304aa0346f3
:10c4c0001e20f5f70ffd234622460421012000948b
:10c4d00001f01afefef782fa0721fef7c8fe234696
:10c4e0002246a2210920f9f751fc234622460021c9
:10c4f0000220cde901440094f9f78eff13f069fda5
:10c50000c5e9020000f0c4f800f0c4fc0b4b8c201d
:10c5100004940694059310f0fff8044610b104a9a2
:10c52000fff70afc281d2146fff7a0ff00200db0f1
:10c5300030bd00bf54250c022c250c02f1c20002b4
:10c5400030b58db00546fff7c3fe48b30024202365
:10c55000cde90434144b04aa00931e20234613494a
:10c56000f5f7c0fc224621460920f9f721fc2146b7
:10c57000281dfff77bffc5e88f4f13f02afdaa683f
:10c580002346821a00210820cde901440094f9f7de
:10c5900043ff00f07df800f013f920460db030bde8
:10c5a0006ff0d100fae700bf6c250c022c250c02bd
:10c5b000022906d0032906d0012906d10021fff760
:10c5c0005dbffff7bdbffff7ebbe6ff077007047b1
:10c5d00013b5047b02690021019202f01bf8214689
:10c5e000019a034802b0bde81040fff7e1bf00bf69
:10c5f000c8ca00100022024b1a705a60704700bf70
:10c60000c8ca001010b50378044613b100201af010
:10c6100067fc204610bd00004ff0fa73194a10b5b0
:10c62000c0e90023184b00f10d028360002303735f
:10c63000164b03f1100153f8044b8b4242f8044ba4
:10c64000f9d102220023426540f26262c0e9083358
:10c65000c0e90a33c0e90c33c0e90e33c0e917332f
:10c66000c0e91933c0e91b33036480f84430c0f8d3
:10c670004630c0f84a30c0f84e30a0f85230a0f82a
:10c68000582010bd1800280020006400bbfe0b02db
:10c6900010b50a4cd4e88f3fdb070cd4204611f0cc
:10c6a00075ff40b10648fff7b7ff204611f0a8ff1d
:10c6b00004489df038fb024810bd00bfd8ca0010e6
:10c6c000dcca001045ca000290f85700704780f895
:10c6d00057107047a0f858100020704773b5374bbb
:10c6e00005461e78002e65d130468df804601af09c
:10c6f000c9fbd5e90801012332468df804301af050
:10c700005cfd041e2bdbd5e90b0132461af089fdd6
:10c71000041e24db314605f146001af0dafc041e43
:10c720001ddb314605f138001af017fd041e16db3b
:10c73000314695f944001af0fafc041e0fdb31462d
:10c7400095f854001af0b8fd041e08db95f8521055
:10c7500059b1314630461af078fe90b1002401a854
:10c76000fff750ff204602b070bd95f853306bb113
:10c7700008461af06afe0028f0d195f85430022bd2
:10c7800014d11af082fd00eae074e8e71946184671
:10c790001af05bfe50b195f85430022bded1012027
:10c7a000002185f854001af087fdece700201af00c
:10c7b00099fde8e76ff0d104d4e700bf61510010a4
:10c7c00070b51b4e044635788cb06dbb28468df88d
:10c7d0000c501af057fb012328468df80c301af044
:10c7e000a3fb94f8563083b1204684f85650fff7e7
:10c7f00075ff50b12023cde904350e4b3220009354
:10c800000d492b4604aaf5f76dfb002221460b4883
:10c810001af0d4fb01233370002303a8636223635f
:10c820002366e366fff7eefe00200cb070bd00bf8c
:10c830006151001095250c0283250c02adc9000240
:10c84000f0b52d4b06461d7889b0002d50d12846f5
:10c850008df804501af016fb012328468df8043099
:10c860001af062fb041e38db0c2733882946adf82a
:10c870000c30738802a8adf80e30f388adf808507c
:10c88000adf81230b388adf80a70adf810301af078
:10c8900020fc041e21db33892946adf8183073894a
:10c8a00005a805950795adf81670adf81a301af081
:10c8b00054fc041e11db294602201af0fdfc041e64
:10c8c0000bdb294696f90c001af031fc041e04db40
:10c8d00028461af027fb041e08da3046fff770ffdf
:10c8e00001a8fff78ffe204609b0f0bd2c46f7e700
:10c8f0006ff0d104f7e700bf61510010037a2bb944
:10c9000003681b7813b94068fff75abf70470000ef
:10c91000f0b52a4b05461b7885b0002b3fd190f827
:10c92000523013b990f85330cbb395f855607ebbb5
:10c93000012730468df800601af0a4fa0df10303c8
:10c940003046cde901358df800708df803608df823
:10c950000c601af0e9fa041e24dbd5e9080132461e
:10c960001af02bfc041e1ddbd5e90b0132461af030
:10c9700058fc041e16db30461af0d4fa041e11dbf4
:10c9800001a88df80370fff7b9ff6846fff73afe7c
:10c9900095f8553083f0010385f855305bb96ff099
:10c9a000d10405e001a8fff7a9ff6846fff72afeba
:10c9b000204605b0f0bd0024fae700bf6151001029
:10c9c00073b5194b06461d7855bb28468df80450a3
:10c9d0001af058fa012328468df804301af0a4fa08
:10c9e000041e12dbd6e917012a461af0e6fb041ee4
:10c9f0000bdbd6e91a012a461af013fc041e04dbed
:10ca000028461af08ffa041e08da3046fff7d8fedf
:10ca100001a8fff7f7fd204602b070bd2c46f7e7ee
:10ca20006ff0d104f7e700bf6151001030b5144b2f
:10ca30000c461d788bb0adb90368012b12d10846a6
:10ca4000fff766ff80b12046fff7baff60b12023f1
:10ca5000cde902350b4b00932b4632200a4902aa3e
:10ca6000f5f740fa0bb030bd00201af00efc00289c
:10ca7000f8d020220023cde90223044a0092ece7fb
:10ca800061510010bb250c0283250c02f1250c021c
:10ca900010b5044600689df047fb204610bd10b558
:10caa00004466830fff7f4ff04f15c00fff7f0ff85
:10cab00004f12c00fff7ecff04f12000fff7e8ff82
:10cac000204610bd0148fff7eabf00bfdcca0010d6
:10cad00003680a6802600b6043684a6842604b6002
:10cae00083688a6882608b607047002310b50446b3
:10caf000c0e900338360fff7ebff204610bd38b577
:10cb00000d1e0446006803dd9ef0dcfa18b938bd3e
:10cb10009df00afb00202060a5600120f7e770b5ba
:10cb200000260d1e0446c0e9006686600bddfff797
:10cb3000e6ff40b123685a199a4203d003b11e7030
:10cb40000133f9e76560204670bdf8b5d0e90153bf
:10cb50009d4204460e460cda276862687919521b1a
:10cb6000481c9df014fb01207e556368013363600f
:10cb7000f8bd691cfff7c3ff0028edd1f8e72de9e8
:10cb8000f041476883688846b918994204461546bb
:10cb900012dc266862683e443146d21b70199df053
:10cba000f6fa2a46414630469df0e4fa01206268d2
:10cbb0002a446260bde8f081fff7a1ff0028e8d1b8
:10cbc000f8e7000070b5674b06461c7898b0002c5b
:10cbd00040f0c580022104a8cde90444cde9064413
:10cbe000cde90844fff7b1ff48b95f4d07a8fff74b
:10cbf0004fff04a8fff74cff284618b070bd012175
:10cc000004a8fff7a2ff0028efd0062104a8fff731
:10cc10009cff0028e9d01122214613a812949df010
:10cc2000d0fa2246152112a81af015fa051edddbee
:10cc300012a8f4f7c7f80130c1b204a8fff785ffc6
:10cc40000028d2d0092104a8fff77fff0028ccd00c
:10cc500012a8f4f7b7f812a9024604a8fff78fff4d
:10cc60000028c2d02023adf80430b6f85830062191
:10cc700002a8adf806300294adf80c4016f0a0fa08
:10cc8000051eb3db0b2104a8fff75fff0028acd023
:10cc9000ff2104a8fff759ff0028a6d002220df1ba
:10cca000060104a8fff76bff00289ed0022201a90d
:10ccb00004a8fff764ff002897d0062202a904a861
:10ccc000fff75dff002890d0f7f79ef800f11801fc
:10ccd0000da802f0b9fb9df84430012b2fd1112192
:10cce00007a8fff732ff00283ff47faf072107a80e
:10ccf000fff72bff00283ff478af10220da907a8fb
:10cd0000fff73dff00283ff470af04a90aa8fff722
:10cd1000ecfe0aa906f15c00fff7dafe0aa8fff7ad
:10cd2000b7fe07a90aa8fff7e0fe0aa906f1680006
:10cd3000fff7cefe0aa8fff7abfe002556e703215a
:10cd400007a8fff702ff00283ff44faf032107a811
:10cd5000fff7fbfe00283ff448af0222cee76ff05a
:10cd6000d10549e761510010fcfeffff38b543686b
:10cd700005468b420c4612da836899420adcd5e9f3
:10cd800000230021134422449a420ad003b11970af
:10cd90000133f9e7fff7b3fe0028f0d138bd0029d1
:10cda000fcdb6c60fae7000070b5394b05461e7875
:10cdb0008ab0002e68d11f2101a8fff7b0fe1f2105
:10cdc00004a8fff7acfe32461f2101981af00ffab3
:10cdd000041e50db214601a8fff7c8ff32461f2181
:10cde00004981af038fa041e45db214604a8fff720
:10cdf000bdff0c2331466b8705f138001af0c5f9e9
:10ce0000041e38db314605f144001af09bf9041e7c
:10ce100031db314605f146001af066f9041e2adbc3
:10ce2000314605f154001af052fa041e23db304655
:10ce30001af06ffa314685f8520030461af005fbb9
:10ce400001a985f8530007a8fff74ffe07a905f1d0
:10ce50002000fff73dfe07a8fff71afe04a907a868
:10ce6000fff743fe07a905f12c00fff731fe07a8e5
:10ce7000fff70efe344604a8fff70afe01a8fff7ed
:10ce800007fe20460ab070bd6ff0d104f9e700bf7d
:10ce90006151001037b50024264b054620461c7012
:10cea0008df8044019f0eeff012320468df8043080
:10ceb0001af03cf820b10a201f4a2049f4f790f8f4
:10cec00000201af02ff8041e2fdb2846fff77afe09
:10ced000041e2adb2846fff767ff041e25db01231b
:10cee000284685f85630fff76bfd041e1ddb2846eb
:10cef000fff7a6fc041e18db0022294610481af092
:10cf000042f8041e11db95f8523033b1002401a819
:10cf1000fff778fb204603b030bd95f8530000289a
:10cf2000f4d11af0b2f9041ef0da2846fff748fcf3
:10cf3000ede700bf6151001021d4010214260c025c
:10cf4000adc90002c0687047c2684068101a7047d7
:10cf500010b500200c4613f02ff84ff47a7200231e
:10cf6000f3f782fd2060002010bd70b5202488b04a
:10cf7000224606460d46684600219df022f9002112
:10cf80006846adf800400cf0a7f8044630b9684692
:10cf9000b36998472860204608b070bd6ff0630001
:10cfa000fae70000012208b5094b1a70fef7d4fc1d
:10cfb00001280cd1f8f736fa28b9064b1b7813b9bb
:10cfc000054b1b781bb1bde80840fcf789b908bdcb
:10cfd00044cc0010c1c40010c0c40010fff7e2bf71
:10cfe000438c8b422cd890f82030012b16d0022b8a
:10cff00011d03bbb90f82430013bdbb280f82430e9
:10d00000c3b1012380f820304ff4af7343844ff451
:10d0100020634361704790f824203ab1002380f8e0
:10d020002030322343844ff47f43f2e7114604302b
:10d03000f5f73cb8022380f8203040f2ee23e5e714
:10d040005b1a43847047012a08bf016000207047c3
:10d0500010b50446024b0360fcf7e2f8204610bd11
:10d06000d0260c020148fff7f3bf00bff8cb001039
:10d0700010b50446fff7ecff204628210ff054fbc3
:10d08000204610bd10b50446024b0360fcf7c8f8fb
:10d09000204610bde4260c020148fff7f3bf00bf95
:10d0a00024cc001010b50446fff7ecff20462021e9
:10d0b0000ff03afb204610bd028c002304213030d3
:10d0c00017f048bf024610b508b1002010bd014658
:10d0d000f9f7dbfd0028f8d1054c23889bb2002b23
:10d0e000f3d012f076ff2388c01a80b2eee700bfbb
:10d0f00058cb001070b58eb02a4905a805f050f93c
:10d1000005a805f0cdf8b5eec00af1ee10fa47db40
:10d1100005a805f0c5f8b3ee047ac0ee077af8fe6c
:10d12000677afdeee77a17ee905a1f4ed6e88f2ffa
:10d1300012f001021d4c1cd13046039211f026fa68
:10d14000039ab0b114210f20f8f7defe1e2202214f
:10d150000346cde9002120460f226ff07f4105f004
:10d160002bfd134b3046236011f04afa11489cf016
:10d17000dafd002210481146f4f798ff022384f8e4
:10d18000203040f2ee2363844ff42063002201211b
:10d19000094884f824506361f4f788ff0eb070bd2d
:10d1a0000025c2e7c4d0001050cb0010f8cb00100f
:10d1b000d0260c02e5cf0002fccb001008b50023fe
:10d1c000a2211a460c20f8f7e1fd0122024b1a7049
:10d1d000bde8084001f000ba45cc001010b5094c7c
:10d1e0002378012bdab204d0022a07d0002323705f
:10d1f00010bd0028fcd1fff77dfff7e7fff7deff4a
:10d20000f4e700bf60cb00101fb5002310490a7877
:10d210000b70104902f0ff040b60bab101220093b9
:10d22000cde901324ff4005022460021f9f7f4f81d
:10d23000094b1c70094b5868c0f30800003818bf30
:10d24000012004b0bde81040fff7c8bf04b010bd16
:10d2500068cb00106ccb001060cb001000ed00e03c
:10d2600030b51d2885b025d9b0f5fa7f04d305b0b7
:10d27000bde83040fff7c8bf104c23780133dbb264
:10d2800023702378042b17d812f0a3fe4ff47a7280
:10d2900000250b4b18600b4b1a60002301214ff443
:10d2a0008050cde90131227800210093f9f7b4f8dc
:10d2b000002ddcd105b030bd0125eee768cb0010b4
:10d2c00064cb00106ccb00107fb506462a4de0b150
:10d2d000002211461046f9f7d8fc284c207012f0b5
:10d2e00078fe80b22880227802f0ff0342b9012242
:10d2f0008020cde9013200211a460093f9f78cf81d
:10d3000000221f4b1a7004b070bd2b889bb2002bfb
:10d31000f9d012f05efe2c883246041b31463046ae
:10d32000a4b2f9f7b2fc60b901230090cde9010382
:10d330002246034600218020f9f76ef82046fff7c9
:10d340008fff41f286330022a4f6b934a4b29c4286
:10d350002a80d8d8094b1b78002bd4d01146104610
:10d36000f9f793fc00220028cdd00121104604b02b
:10d37000bde87040f9f7e0bd58cb001070cb00104d
:10d3800071cb0010012802d80846fff79dbf7047f7
:10d3900010b5394c2288013a92b222802ab911463e
:10d3a0001920f4f7effe19232380344c2388013b26
:10d3b0009bb223801bbbfcf7ddfb4ff47a73238009
:10d3c0002f4b1a68b2f57a7f51d300221a600bf006
:10d3d00019fb4ff6ff700ef0abff2a4c10f0fefc6d
:10d3e0002368002b47d012f0f4fd274b1a682368fe
:10d3f000801a98423fd9bde81040fff705bf0022d0
:10d4000011461046f9f741fc80b142f210700bf062
:10d4100036fc58b11d4b197801f0ff0231b90121da
:10d42000104619700321f9f737fcc9e700221146ad
:10d430001046f9f72afc0028c2d140f6b8300bf0ac
:10d440001efc0028bcd0124b1b7803f0ff04002bfd
:10d45000b6d101f0c1f82046fff736ff204622463c
:10d460002146f9f769fd0120fff72effa8e71a68aa
:10d4700001321a60b1e710bd625100106451001012
:10d480005ccb00106ccb001064cb001071cb001093
:10d4900070cb001013b501200bf052feff281ed0f8
:10d4a000c3071cd50420fef739fa002100240846e2
:10d4b000fef758fa224604200df107018df80740c7
:10d4c000f5f77efe9df807304bb122462146042039
:10d4d000f5f75efe224621462046f9f72dfd02b003
:10d4e00010bd000010b50446fef736fa022801d040
:10d4f000002010bd002cfbd1fef708fa0028f7d061
:10d50000f7f790ff0028f3d1024b1878b0fa80f0bb
:10d510004009eee702c9001030b50d4d02462c78e7
:10d5200085b034b108200b4a0b49f3f759fd9cf044
:10d53000f3fb01234ff48020cde901432b70002140
:10d5400023460094f8f768ff2c7005b030bd00bf8b
:10d5500020cc001021d4010256260c0201287fb5f0
:10d560000c463fd00a2843d1224dd5e88f2f12f028
:10d5700001021cd12846039211f008f8039ab0b1b9
:10d5800014210220f8f7c0fc02221e211a4e034685
:10d59000cde9001230466ff07f4105f00dfb174bcf
:10d5a0002846336011f02cf815489cf0bcfb14f0b1
:10d5b000010212d000210846f8f79cfc50b1036923
:10d5c000002201210c484361043004b0bde87040e2
:10d5d000f4f76cbd6ff07f43f2e7a30708d511465f
:10d5e0000848f2e7084604b0bde87040fff794bf72
:10d5f00004b070bd54cb001024cc0010e4260c0203
:10d6000019d0000228cc001070b5044686b0062060
:10d610000ef08efe002c65d1204600f049ff3e4bf7
:10d620001b78002b5ad1fef771f9002856d0f7f776
:10d63000f9fe002852d1394b1b78002b4ed1fef752
:10d640008bf901284ad106b070bdfef749fefef7fe
:10d650004bfe0028f7d14ce007200ef069fefef7e4
:10d660007bf9042801d0f3f783fc01232c4e2b70a7
:10d6700096f82c303bb9fff795fc2046fff732ffb8
:10d680000028e0d139e0706a17f011fc0546002847
:10d69000f1d1244b14200593234b04930ff03cf855
:10d6a000044690b1214b02a940f8043bf7f7eafb8e
:10d6b0001f4b3046236001a90194f7f76cfb40b182
:10d6c000706a10b1294617f01ffc02a8f5f732fa6c
:10d6d000b9e7236820469b689847f6e7154b1b7807
:10d6e000002bb0d12046fff7fdfe0028abd1002c67
:10d6f000abd00a4d2b78012baed108200ef018fece
:10d70000fef72af904289ed0f3f73efc092006b064
:10d71000bde870400ef00cbe02c9001021cc001014
:10d72000fcc500105dcf0002c7cf0002ec0f0c0259
:10d7300000100c02c3c400100120fff765bf0000f9
:10d7400030b593b01cf05efaf3f706fc0bf01cfa50
:10d75000002000f025fa05200ef0eafd00232a2122
:10d760001a461846f8f712fb1ef0dafc474bda8827
:10d77000012a04d100229a71da711ef0edfcf5f74e
:10d78000f1f800220024202511460220f4f7aafe19
:10d7900006a8f7f76dfe069b3d4901933d4b0aaa8b
:10d7a0001e2000932346cde90a54f4f79bfb204644
:10d7b0001af040ff1af042ff224601203449f4f7e4
:10d7c0004ffcb0b1224605a904a8cde904440bf0f2
:10d7d000fbfa70b9049b63b1059acde90a50cde913
:10d7e00001322d4b2a4900930aaa03460120f4f77f
:10d7f00079fb0ff079faf6f707fbf6f7effafff788
:10d8000049fe16f0e1fb254816f092fd0020fef7d8
:10d81000aff860b3fef7a0f8041f18bf0124002181
:10d82000084613f0c1fa012807d864200ff035fe2e
:10d830000022462011460bf035fa204600f0eef9a2
:10d84000174db4b11748fff737fc1648f9f7d4fc69
:10d850002846fff731fc002017f027fb68622846b6
:10d86000f9f7fffc06a805f01df813b030bd04461b
:10d87000d5e7204617f019fb0a4b5862204617f0ef
:10d8800014fb68620020fff7bffefbe7b8000c0046
:10d8900018100c0262260c0274260c022d320002b3
:10d8a000c4cb0010fcc500102de9f0433d4b8db0fa
:10d8b00000933d4b694603933c4b04a8002502931b
:10d8c000f7f7e0fa4ff44063cde9083541f28833c9
:10d8d000374c0a930223204614268df82e30354b00
:10d8e00004a940f8043badf82c60f7f7cbfa089b8d
:10d8f00065626361099b04f12800a3610a9bdff85c
:10d90000f480e361bdf82c302b4f23849df82e303a
:10d91000dff8e49084f8223017f07dfb274b84f881
:10d920002c502360256304a8f5f704f96846f5f741
:10d9300001f92946224812f051fb224c224b29467c
:10d94000a360224bc4e90086c4e903346761201d4b
:10d95000f4f746fd1e4b294623601e4c1e4bc4e9be
:10d960000086a3601d4b6761c4e90334201df4f7f2
:10d9700037fd1b4bc4f80090a3611a4c1a4b294683
:10d98000a3601a4bc4e90086c4e903346761201d13
:10d99000f4f726fd164bc4f80090a3610db0bde866
:10d9a000f08300bfb9d60002974d0002834d0002fc
:10d9b000c4cb001080130c027b640002c0260c0252
:10d9c000ddd4000274cb00100600020099260c0280
:10d9d000f8260c02a8cb001019000100a4260c02a6
:10d9e000c5ce00028ccb00101a000100ad260c023f
:10d9f000c9ce0002bc140c0208270c02f0b5024686
:10da0000406890b10831d46821f003039168201a6e
:10da1000091a043399424ff0000107d3c4e90013f7
:10da2000d1680b4401f10800d360f0bd0d460846f3
:10da3000146974b166689e4205d338b14768be4226
:10da40003cbf0d46204621462468f2e70d4620469d
:10da5000f9e70028e9d003684db12b602b465169e6
:10da6000814208bf5361002340f8083bdde71361a2
:10da7000f5e7704710b5044618210ef055fe204614
:10da800010bd0000014b586a17f011bac4cb00104a
:10da9000012a38b5044602d10b68236003e0022a4c
:10daa00003d0032a0dd0002038bd0c200d680ef0e5
:10dab00033fe03460028f0d095e8070083e807000e
:10dac000ebe700680028eed00c210ef02dfeeae70f
:10dad00030b5002939d051f8044cc268a1f10803cf
:10dae0001d19aa4214d1121bc2600024426962b3fc
:10daf0005168c3685518ab4227d15b1ac3600369ec
:10db000013b119688a421cd14361e3b90361ede79f
:10db1000056900222c4624b19c4238bf2246246865
:10db2000f9e72ab905b9436141f8085c0361dce70c
:10db3000146841f8084c136041699142d5d14361a2
:10db4000d3e70b46dce71c60d0e730bd438c8b424b
:10db500023d890f8203013b1012b0ad0704701234d
:10db600080f82030fa234384837c43f002038374db
:10db7000704790f82420013ad2b280f8242042b1b4
:10db8000002380f82030fa234384837c03f0fd03d4
:10db9000ede711460430f4f789ba5b1a4384704705
:10dba00038b50c4cd4e88f3f13f0010f0a4d09d162
:10dbb000204610f0ebfc28b117f0caf92860204687
:10dbc00010f01efd17f0c4f92b681b1a584258417b
:10dbd00038bd00bf4ccc0010a4d0001010b50446d6
:10dbe000024b0360fbf71cfb204610bdb4280c025f
:10dbf0000148fff7f3bf00bf7cd0001010b504460a
:10dc0000fff7ecff204628210ef08efd204610bdc8
:10dc1000014b586a17f04bb9fcc50010002210b533
:10dc2000044611461046f8f743ff6cb1fdf794fe29
:10dc3000042805d100231a4619461846f9f71afa9e
:10dc4000bde81040fbf7d4bffdf786fe0128edd1fb
:10dc5000f0e7000008b5064b1b78032b06d104f053
:10dc600057fcbde808400021f5f702bb08bd00bf26
:10dc7000c3c4001070b52d4a8cb01378002b52d05d
:10dc80000023157813702022cde90423284aedb231
:10dc9000009228202749019504aaf4f723f9264c7d
:10dca000d4e88f2f12f001021dd12046039210f00c
:10dcb0006dfc039ab8b114210f20f8f725f91e2244
:10dcc00002211e4e0346cde9002130460f226ff09f
:10dcd0007f4104f071ff1a4b2046336010f090fc36
:10dce00018489cf020f8012d1bd8e5b14ff47f06b1
:10dcf0000022124c1146201df4f7d8f9fa23002215
:10dd0000012166616384a37c201d03f0fd0384f878
:10dd1000245084f82020a3740cb0bde87040f4f7c0
:10dd2000c5b9094ee4e70cb070bd00bf46cc001089
:10dd300010270c0218100c0248cc00107cd00010e8
:10dd4000b4280c0271db00020060ff00002270b5f5
:10dd5000314d8cb007200df10f018df80f20f5f734
:10dd60002ffa2b685a1c2a601bb912f032f92b4b80
:10dd700018609df80f301bb312f02bf9274e336853
:10dd8000c01a274b98421bd900242023cde9043424
:10dd900005230193234b04aa0093282023462249fc
:10dda000f4f7a0f80122214b34601a70204b2c604c
:10ddb0001c709df80f300bb91e4a13600cb070bd7b
:10ddc000f6f75efd1c4cc8b110f1aa0f14d01b4a27
:10ddd0001b4b10f1a00f08bf1a460023202101920f
:10dde000184acde90413009228200f4904aaf4f739
:10ddf00079f802232370dce7134aeee72023cde90c
:10de00000430124b0849009304aa03462820f4f773
:10de100069f80323eee700bfa8d0001054cc00102f
:10de2000df9304002d270c0218100c0201c900100a
:10de300058cc00108cc9001046cc00103a1a0c02c5
:10de40009c3d0c027b270c0229270c0294270c0214
:10de500008b5074a1378ff2b1cbf0133137012f06b
:10de6000b8f8044b1860bde80840fff76fbf00bf6b
:10de700058cc001050cc001000222de9f041114682
:10de80008cb01046f8f744fe00287ed0404b1b783b
:10de9000002b7ad13f4f3b7803f0ff04002b74d165
:10dea0002346224652210520f7f770ff12f091f821
:10deb000394b1d68394b451b1878faf7cffa854264
:10dec00063d34ff02008364b04aa364900931e2036
:10ded0002346cde90484f4f705f8fcf7c1f80122e4
:10dee000054600f118031a60402023460021cde9c1
:10def00001440094f8f790faeb6e0133eb66f6f705
:10df00007ffb061e10db01233b70274b1e20009376
:10df10002449234604aacde90484f3f7e3ff0cb0b7
:10df2000bde8f041fff7a6be204b019600932820e4
:10df300023461c4904aacde90484f3f7d3ffe6364f
:10df400009d1224621460620f7f732ff2246214614
:10df50000520f7f72dff002305f118023b70136031
:10df600040201a46cde9013300930021f8f754fa16
:10df70000f4b1b7803f0ff023bb911461046f8f730
:10df800084fe10b9fff764ffc9e70cb0bde8f0816b
:10df900002c90010c2c4001050cc001058cc0010b0
:10dfa000bc270c0218100c02ce270c02e5270c022d
:10dfb00001c9001008b503200af0b6ff034b187022
:10dfc000bde8084080f00100fbf72cbeacd000108b
:10dfd00008b5fef785f9fef787f948b109200af080
:10dfe000a3ff28b1fef77cf9bde80840fef7a8ba08
:10dff00008bd08b5002000f0a3fd40b109200af0db
:10e0000093ff014618b9bde8084000f005be08bd01
:10e010002de9f74f0f46044600284cd0dff8a480c6
:10e020004ff47a79d8f80030dff89cb00344c8f890
:10e03000003011f0ceff054611f0c7ff06460af08a
:10e04000e1fc11f0c6ffa0eb050a544533d3621e74
:10e05000924510d34ff47a7000fb0464174d11f011
:10e06000b4ff201aa84226d84008012828bf012062
:10e070000ff016faf3e701200ff00ffa104b1a78a1
:10e08000002adcd1002fdad1ca4504d2d8f800200a
:10e09000b2f57a7fd3d30020fdf76afc0af57a79ce
:10e0a0000190f7f7cff901980028c8d19bf800300c
:10e0b000002bf5d1c3e703b0bde8f08fa0860100c7
:10e0c00002c90010b0d00010c3c4001013b50c4b2f
:10e0d0000446586a019116f0eafe58b1094b0199bd
:10e0e0005b68c3f308032bb9204602b0bde81040bb
:10e0f000fff78ebf204602b0bde810400ff0cdb94b
:10e10000c4cb001000ed00e02de9f04fdff8b0b116
:10e1100093b005939bf8003080460e469246604fc0
:10e120001bb93b78002b00f0ad8020230024cde903
:10e130000a345c4b1e205c4900930aaa2346f3f77d
:10e14000d1fefbf78dff3b780546b3b1c4663eb107
:10e1500000f134031e60012e02bf036d013303651d
:10e16000032205f118031a60002309224020002130
:10e17000cde901330093f8f74ff9fbf775ff4ff046
:10e180000102d0e8cf3fc0e8412f0029f9d1dbb22e
:10e19000002bf6d1c2680169047d90f81590c36028
:10e1a000036103754375c0e88f3fd3075cbf047af2
:10e1b000e4b2930758bf416853073b7858bf90f8c3
:10e1c000099018f0010f08bf002413b3002c5fd092
:10e1d0001023adf81830059badf81a60adf81e306d
:10e1e0001c9badf81ca0cde9083105f0e7f9002231
:10e1f000022106ab05f00df858b120220023cde92d
:10e200000a232a4a01900092282027490aaaf3f7f4
:10e2100069feb9f1000f01d0fbf738fa18f0020fd0
:10e2200002d12046f6f7cefa0024214b3c701c7038
:10e23000204b2246214607201c708bf80040f7f740
:10e24000b7fd224621460620f7f7b2fd22462146b9
:10e250000520f7f7adfd2023cde90a34164b0aaab5
:10e2600000931e2023461049f3f73cfe224605f199
:10e2700018031c60402023460021cde9014400948e
:10e28000f8f7caf800220d4b1a7013b0bde8f08ff2
:10e2900005f094f923462246032104f0baffb8e7bb
:10e2a000bfc4001008280c0218100c021d280c0214
:10e2b000c1c40010c0c400104f280c0246cc00108e
:10e2c000c2c40010f0b5634b05461b788db0002b1f
:10e2d00000f0bd80604f3b78002b40f0a1805f4b89
:10e2e0001b7803f0ff04002b40f09a805c4e3278dc
:10e2f00002f0ff03002a3dd0fbf758fe002800f093
:10e3000097802023cde90434564b04aa5649009344
:10e310001e202346f3f7e6fd01233b70534b347078
:10e320001c70fbf79dfe022200f118031a60082200
:10e33000234600214020cde901440094f8f76cf811
:10e34000fdf70afb0428234622464ff052010cbf7a
:10e3500008200720f7f71afd002205201146f7f7dd
:10e3600027fd002206201146f7f722fd0022404b30
:10e370001a6055e01a4652210620f7f707fdfff70d
:10e3800019fe04460028f1d03a4b1b7803f0ff0237
:10e39000002b3ad111461046f8f777fca8bbfff7df
:10e3a00057fd062c46d0082c14bf4ff47f074ff0c2
:10e3b000ff1700262023cde904362f4b28202a49b9
:10e3c000009304aa33460194f3f78cfd32461421de
:10e3d0000120f7f799fd1e2202210346cde9002115
:10e3e00004a80122394604f0e7fb3246012105a8c2
:10e3f000f3f75cfe11f0edfd064611f0eafd831b1c
:10e40000f92bfad904a8faf70bfffbf729fe002332
:10e41000c0f888401a46072118460093fff774fe9b
:10e42000164b1b7843b10db0bde8f040fbf7c6bdfd
:10e430000a24a9e7124fbce7002df4d1fdf78cfaae
:10e440000328f0d12846fdf793fa0128ebd00db050
:10e45000f0bd00bfc2c40010bfc40010c1c4001092
:10e46000c0c4001063280c0218100c0258cc001015
:10e47000a8d0001001c9001073280c02c3c40010fa
:10e480000060ff0013b50446fdf740fa034638b9b3
:10e490000246009002210120fff736fe02b010bdb7
:10e4a000fff7eafc204602b0bde81040fff70abfc4
:10e4b00010b504460af0a6fa0022194b19481a6052
:10e4c000f8f702ff184b1b7803f0ff0023bbfef7a1
:10e4d00085fefff7bffbf8f73bfef8f736fcf8f7d1
:10e4e0003bfc2046fff7cefff9f7c2fbf9f7eafc49
:10e4f000fdf732fa042801d0fff76afdf5f784fc36
:10e50000f5f77ffcfdf728fa042801d0fff771fd2d
:10e51000bde81040f4f74abf8c20f4f7ebfeede7be
:10e52000b0d0001074d0001045cc0010f0b5224ed1
:10e53000044696f82c300d46174687b0002b38d08d
:10e54000706a16f0b4fc002833d104900c200ef051
:10e55000e3f810b1c0e900458760184b02900593bd
:10e56000174b142004930ef0d7f80446d8b1154b7e
:10e5700003600023c360049b3bb1022202a9043064
:10e580009847059b2361049be3600f4bf26923606e
:10e59000306b002301a9019416f0e7fc18b1236841
:10e5a00020469b68984702a8f4f7c4fa002007b0f9
:10e5b000f0bd2846a047f9e7c4cb00104de50002a6
:10e5c00011da0002ec0f0c0200100c02036818684c
:10e5d000d3e90112fff7aabf08b5002301211a46ab
:10e5e0001846f8f702fbbde80840f6f7f3b800005c
:10e5f00037b501900af0fcf9019905460448fff788
:10e60000fdf9044628460af0f7f9204603b030bd6c
:10e610005cd0001013b501900af0eaf904460199a4
:10e620000448fff755fa204602b0bde810400af052
:10e63000e3b900bf5cd000106ff0770070470000b6
:10e64000032809d8dfe800f00a02040604487047ee
:10e65000f6f7eabbf9f7bcba0020704701487047eb
:10e66000fcc50010c4cb001013b500240b4a234690
:10e670000b490c480094f2f77fff0b4b0b4a1c60d0
:10e680005c600b4bc2e904445360d3604ff4806379
:10e690009360084b136002b010bd00bf05da0002a2
:10e6a00091db000221db000274d000105cd000106e
:10e6b0005ccc00109c280c02012a38b5044602d11b
:10e6c0000b68236003e0022a03d0032a0dd0002048
:10e6d00038bd0c200d680ef01ff803460028f0d05e
:10e6e00095e8070083e80700ebe700680028eed014
:10e6f0000c210ef019f8eae721b18b88834201d092
:10e700008968f9e70846704708b50a46c1680e20cf
:10e71000fff7f2ff40b1037b934202d1c389db07cd
:10e7200001d58168f3e7012008bd4ff00102d0e870
:10e73000cf3fc0e8412f0029f9d1dbb2002bf6d141
:10e74000704700002de9f04fb84b144693f82c2089
:10e75000064689468db0dab1586a16f0a8fbb8b9fa
:10e7600006900c200df0d8ff10b1c0e9006984605c
:10e77000af4b04900793af4bac4804a90693f4f752
:10e78000d1fa044670b9074604a8f4f7d3f905e0b6
:10e79000002130460df026fc071e0fda38460db07a
:10e7a000bde8f08f00224ff0ff31406916f098fc71
:10e7b000236820469b68a7699847e5e7f9f758fa68
:10e7c0000821f9f7dbfb04213046fff79dff804667
:10e7d000002842d10420f168fff78eff002858d1ad
:10e7e0004546b368dc072bd5f6f71cfe40b3fbf7b4
:10e7f0003bfc0446fff799ff0023e268d4f810a021
:10e80000677de360236123756375c4e88f3fd0079c
:10e8100058bf237a910758bfd4f804a0520758bfb5
:10e82000677afbf721fc0446fff77fff0723e360cd
:10e830000123c4f810a0237567750023c4e88f3f37
:10e84000002306211a4601200095fff75dfcfdf725
:10e850005df88246fdf754f804e0f6f7e3fd4ff06b
:10e86000000a804604213046fff74eff68b97388de
:10e87000022b16d9f1680e20fff73eff88b1037b0b
:10e88000042b0cd1c389db070bd500252c46ab46e6
:10e890004ee04ff47a73c568b5fbf3f5a1e78168e4
:10e8a000e9e7002204201146f8f781f9024690b109
:10e8b000002204201146f8f77af928b1002301213b
:10e8c0001a460420f8f791f9002205210420f8f7f0
:10e8d00045fa012506e001460420f8f719f9002859
:10e8e000e6d1054600210420f8f79af904460028ed
:10e8f0007ed1042004a91bf01bfa70b9fcf76ef856
:10e9000002220499fcf798f900286fd1fcf766f809
:10e9100004220499fcf790f90446002303222020e6
:10e920000021cde901330093f7f776fd4ff0010b9d
:10e9300000210846f3f7fefbe720f2f7a5fc0120d3
:10e94000f4f711f80022494630460df091fb0746d6
:10e95000f4f70af801200021f3f7ecfbe720f2f7c7
:10e960006ffcbbf1000f12d054b100210420f8f766
:10e9700057f928b1002304201a461946f8f750fa2f
:10e980002db1002304201a461946f8f773fbbaf19b
:10e99000000f3fd0fcf792fffcf7deff044600209b
:10e9a000fcf7e6ff054600287ff4f8ae013ce4b230
:10e9b000012c3ff6f3aefcf7a9ff00283ff4eeaec2
:10e9c000284611f0f9fa4ef660250446002011f0b1
:10e9d000f3fa001b61f10001a84271f1000316d2a5
:10e9e000f6f720fd98b9f6f72dfdefe7012494e73f
:10e9f00000242023cde90434042301930e4b01208d
:10ea000000930e49234604aaf3f76cfa8ee7f6f753
:10ea100009fdc3e6b8f1000f3ff4c0aefaf768fe97
:10ea200053465246042104f0f4fbb7e6fcc500103f
:10ea3000c1e9000239e60002cd280c02c0280c0210
:10ea400003681868d3e90112fff77cbe70b5002394
:10ea50001646202204460d468ab0cde90223074a15
:10ea600001200092064902aaf3f73cfa32462946f1
:10ea700020460ab0bde87040fff764bee9280c02ea
:10ea8000c0280c02012a034602d101600020704711
:10ea9000022a04bfd1e90001c3e90001f6e7012a17
:10eaa000034602d1016000207047022a04bfd1e969
:10eab0000001c3e90001f6e7012a034602d1016023
:10eac00000207047022a04bfd1e90001c3e9000118
:10ead000f6e7012a034602d1016000207047022aae
:10eae00004bfd1e90001c3e90001f6e7012a0346aa
:10eaf00002d1016000207047022a04bfd1e9000161
:10eb0000c3e90001f6e7012a02d101600020704745
:10eb1000022a04bf0b680360f8e7012a034602d10a
:10eb2000016000207047022a04bfd1e90001c3e957
:10eb30000001f6e700224ff0ff3116f0d1ba0000d5
:10eb400070b52d4e044696f82c3086b0002b4bd075
:10eb50003046f6f7e1fb0546002845d1274b1c203f
:10eb60000593274b029404930df0d6fd044600282c
:10eb700031d0244bc5600360049b3bb1022202a943
:10eb800004309847059b2361049be36000252046e1
:10eb90001d4b2a462360012140f8145f16f090fabd
:10eba0001a4b01a92360f2692b46306b019416f0d1
:10ebb000dcf9014650b9706a08b116f0a5f90022d7
:10ebc0004ff0ff31606916f08bfa257e23682046ee
:10ebd0009b68984700e0054605f0010502a8f3f799
:10ebe000a9ff284606b070bdfdf752fd06b0bde88e
:10ebf0007040fdf769bd00bffcc5001091eb00023d
:10ec000087ea0002a0130c02b4130c02c8130c0212
:10ec10000068fff795bf000070b5534d044695f8a6
:10ec20002c300e468ab0bbb12846f6f775fb98b972
:10ec30004e4b284605934e4b02a98df8084003968b
:10ec40000493f4f76ff80546c0b9044602a8f3f739
:10ec500071ff20460ab070bd09200af065f9b0b90d
:10ec60002023cde90230434b4349009302aa0346d7
:10ec70003220f3f737f96ff08104eae74069fff7d4
:10ec800059ff2b6828469b68ac699847dee7002c43
:10ec90004cd0fdf7fdfcfdf717fd044608b100243c
:10eca000d7e7fdf71dfbfdf71ffb90b109200af028
:10ecb0003bf970b12023cde90234304b2e4902aa32
:10ecc000012000932346f3f70df9fdf709fbfdf74b
:10ecd00037fc002520262a4b02aa27490120009351
:10ece0002b46cde90265f3f7fdf8fdf7d1fc0121d4
:10ecf000fdf7edfcf5f788f8183000f0a5fcfdf7fe
:10ed0000c7fcfef7c7f804460028a2d01d4b1a49dd
:10ed1000009302aa2b460120cde90265f3f7e2f841
:10ed2000fdf7b6fc2946fdf7d2fc92e7fdf7b0fcf3
:10ed3000fdf7cafc0028b2d02023cde90234124be3
:10ed400002aa0d49009301202346f3f7cbf8fdf703
:10ed50009ffc2146fdf7bbfcfdf79afc0ab0bde81d
:10ed60007040fdf72dbd00bffcc500100ded000289
:10ed70009bea000205290c0218100c023a290c0229
:10ed800088290c029d290c02bb290c0241680078dd
:10ed9000fff742bf7fb51c4d044695f82c300e4658
:10eda000b3b12846f6f7b8fa90b9184b6946039301
:10edb000174b2846cde900460293f3f7b3ff04460c
:10edc00048b905466846f3f7b5fe284604b070bd5d
:10edd00054b9104df9e74069fff7acfe23682046af
:10ede0009b68a5699847ede709200af09df840b1b6
:10edf000f5f70af82146183004b0bde8704000f07d
:10ee0000c3ba6ff08105e0e7fcc5001099ed000280
:10ee10006dea0002f2feffffd0e90001fff7babf82
:10ee20007fb51c4d044695f82c300e46b3b12846ec
:10ee3000f6f772fa90b9184b69460393174b2846b8
:10ee4000cde900460293f3f76dff044648b9054645
:10ee50006846f3f76ffe284604b070bd54b9104df4
:10ee6000f9e74069fff766fe236820469b68a569bd
:10ee70009847ede709200af057f840b1f4f7c4ffce
:10ee80002146183004b0bde8704000f095ba6ff02c
:10ee90008105e0e7fcc5001025ee000253ea000200
:10eea000f2feffffd0e90001fff7babf7fb51c4dae
:10eeb000044695f82c300e46b3b12846f6f72cfae6
:10eec00090b9184b69460393174b2846cde9004685
:10eed0000293f3f727ff044648b905466846f3f75f
:10eee00029fe284604b070bd54b9104df9e74069b9
:10eef000fff720fe236820469b68a5699847ede749
:10ef000009200af011f840b1f4f77eff21461830cd
:10ef100004b0bde8704000f067ba6ff08105e0e72b
:10ef2000fcc50010b1ee000239ea0002f2feffff5c
:10ef3000d0e90001fff7babf7fb51c4d044695f834
:10ef40002c300e46b3b12846f6f7e6f990b9184bc7
:10ef500069460393174b2846cde900460293f3f721
:10ef6000e1fe044648b905466846f3f7e3fd284646
:10ef700004b070bd54b9104df9e74069fff7dafdf0
:10ef8000236820469b68a5699847ede7092009f0aa
:10ef9000cbff40b1f4f738ff2146183004b0bde88c
:10efa000704000f039ba6ff08105e0e7fcc5001051
:10efb0003def00021fea0002f2feffffd0e9000170
:10efc000fff7babf7fb5174d044695f82c300e46b3
:10efd00003b32846f6f7a0f9e0b9134b694603934b
:10efe000124b2846adf8004001960293f3f79afec3
:10eff000044668b14069fff79dfd236820469b6881
:10f00000a56998476846f3f795fd284604b070bd9a
:10f010000546f7e7fdf73cfb214604b0bde870402c
:10f02000fdf758bbfcc50010b1ef000205ea000275
:10f0300041680088fff7c6bff8b5044605462f466d
:10f0400015f8016b30469af041ff0028f7d15f2e8a
:10f05000f5d0381bf8bd2de9f8430c461746994604
:10f0600078b119b38e18a64205d9054615f8013bab
:10f070004bb904f8013b0023781e341b06f8013c11
:10f08000001bbde8f883242b0dd12846fff7d4ffe1
:10f09000804630b122460146331b2846c8474544c6
:10f0a00004442846dfe704f8013bfae70846e8e7ae
:10f0b0007047704737b50446019109f099fc0199f2
:10f0c00005462046fef79afc0446284609f094fcc3
:10f0d000204603b030bd10b5044604210df024fbda
:10f0e000204610bdc86910b50c4608b10df01afbda
:10f0f0000023c4e90133e36110bd000010b5044be7
:10f1000004460360406808b10df00cfb204610bdba
:10f11000e42b0c0210b50446fff7f0ff204618213f
:10f120000df002fb204610bd084611469bf0cabff9
:10f1300008469af0f9bf08469af0eebf2de9f04173
:10f140000c461e46174605460368ddf818805b68c6
:10f150009847c4e90968e762a86915f06bffeb6896
:10f1600043b19c610023a361a869ec60bde8f04154
:10f1700015f06fbfac60f5e737b50546019109f0b2
:10f1800037fc044601992846fef7a2fc204603b04e
:10f19000bde8304009f030bc10b5084cd4e88f3fd2
:10f1a000db0709d420460ff0f1f928b120460ff013
:10f1b00027fa03489af0b7fd024810bdb4d00010fa
:10f1c00031f000026851001008b547f055f818b149
:10f1d000bde808401df008ba08bd38b50446062051
:10f1e00046f070ff054668b1204646f077ff0122e1
:10f1f0002946204646f0caff034628b1bde83840fc
:10f200001df0f2b96ff07703184638bd08b547f026
:10f21000d1f818b1bde808401df0e6b908bd13b536
:10f22000044608460191f1f7cdfd019902462046ba
:10f23000fff7ecff02b010bd10b5c368044623b958
:10f240000a200e4a0e49f1f7cbfee3685a68198985
:10f25000023a5a60e268936802339360e3685b683d
:10f260001980d4e90223916a29b10b600021196049
:10f270009362e16010bd5362f8e700bf21d4010240
:10f28000d1290c0270b500250446394bc0e902555e
:10f290000360c0e90455416040f8185f15f0bbfefb
:10f2a000344be56163654ff6ff732562a4f86c305b
:10f2b000a4f86e30c4e909552f4bc4e90b55c4e9d5
:10f2c0000d55c4e90f55c4e91155c4e91355c4e9f6
:10f2d0001955c4e91755c4e91c55e567a56584f8b7
:10f2e0008050a56784f8815084f8825004f184022c
:10f2f00003f11006154618685968083303c5b34270
:10f300002a46f7d118681d4b286004f1980203f1d2
:10f310001006154618685968083303c5b3422a46d3
:10f32000f7d11868164b286004f1ac0203f11006ff
:10f33000154618685968083303c5b3422a46f7d101
:10f340001868104b286004f1c00203f1100615463e
:10f3500018685968083303c5b3422a46f7d11868bc
:10f36000002328602046a4f8d430a4f8d83070bd1b
:10f37000782c0c02e42b0c02482c0c025c2c0c02a6
:10f38000302c0c021c2c0c0230b581b10b4600f164
:10f39000840201f11005144618685968083303c443
:10f3a000ab422246f7d118682060002030bd0148ea
:10f3b000fce700bff2feffff30b581b10b4600f164
:10f3c000ac0201f11005144618685968083303c4eb
:10f3d000ab422246f7d118682060002030bd0148ba
:10f3e000fce700bff2feffff30b581b10b4600f134
:10f3f000c00201f11005144618685968083303c4a7
:10f40000ab422246f7d118682060002030bd014889
:10f41000fce700bff2feffff30b581b10b4600f103
:10f42000980201f11005144618685968083303c49e
:10f43000ab422246f7d118682060002030bd014859
:10f44000fce700bff2feffff70b50246054601f182
:10f45000840601f19403344603cc9c421060516051
:10f46000264602f10802f6d120681060284670bdd9
:10f470008b890022a0f86e301423c36780f88020a7
:10f4800090f88030dbb280f8813000f17803c3e877
:10f49000af2f00f1740353e8001f0131c3e8e01ff0
:10f4a0000028f8d110467047b0f86e308a899bb2b8
:10f4b0009a4202bf4b68033bc36700207047b0f815
:10f4c0006e308a889bb29a4212d1ca88b0f8d63080
:10f4d0009a420dd1002380f880308a689a42c8bfd2
:10f4e000012380f8803090f88030dbb280f88130e2
:10f4f000002070472de9f041044690b0002017f03d
:10f5000015fd20b10a204a4a4a49f1f769fd94f8ed
:10f510008250002d40f089802b4601200df102021f
:10f5200004f1840118f012fe00287bdb424f2822f0
:10f53000294606a8059708ae9af043fe04f1980cf8
:10f54000bce80f000fc6dcf800302a463360022307
:10f550008df81830bdf8023001a905a8adf8343097
:10f5600018f026fc00285ddb2b4601223349bdf84c
:10f570000a0018f02bf8002854db2022294606a8a0
:10f58000059708ae9af01dfe04f1ac0cbce80f0024
:10f590000fc6dcf80030dff8ac80336010238df844
:10f5a0001830bdf802302a4601a905a8cde90e841d
:10f5b000adf8343018f0fcfb002833dbbdf80a301e
:10f5c0002022a4f8d430bdf80e302946a4f8d63055
:10f5d000059706a808ae04f1c0079af0f2fd0fcf18
:10f5e0000fc63b682a4633600c238df81830bdf8ef
:10f5f000023001a905a8cde90e84adf8343018f029
:10f60000d7fb00280edbbdf80a302a4621460c48fd
:10f61000a4f8d83018f008fc002803db01232846a2
:10f6200084f8823010b0bde8f0816ff0d100f9e7c6
:10f6300021d4010214260c0203002c00442c0c02dd
:10f64000adfe000229f90002002238b50446114639
:10f6500010460cf004fe2046fff74cff054660b94b
:10f660004ff4806007499af003f840b14ff480638b
:10f67000c4e91955a0652066e365284638bd024dea
:10f68000fbe700bf751d0e02fcfefffff8b5064646
:10f690000d4638201049174699f0e8ff0446c0b1de
:10f6a000382200219af08dfd0b4905f1100099f0e8
:10f6b000dfffe06148b10db1083060600020336fba
:10f6c000a560236366613c60f8bd382120460df0db
:10f6d0002bf80248f8e700bf751d0e02fcfeffff85
:10f6e00070b50d4616681446fff756fd036831469f
:10f6f0001b6905f10c02984746b948b1066000f154
:10f700000c03c0e901352060002070bd0028f6d14f
:10f710000048fae7fcfeffff70b5c36804460d46db
:10f72000164623b10a200c4a0c49f1f759fca0688f
:10f7300004f10c02b11cfff7d3ff00280adb002004
:10f74000e268536802335360e2689368023b936057
:10f75000e3682b6070bd00bf21d40102e7290c02d1
:10f7600030b5002585b04ff4007202a90446029519
:10f77000fff7d2ff00280edb114b02990093019591
:10f7800003ab04f12800d1e90112039541f0b8fb65
:10f7900018b11cf029ff05b030bddde9023204f1db
:10f7a0001c0059689a60f8f74dfa0028f3db2046f0
:10f7b000fff742fd03230120c4f8c831ebe700bf87
:10f7c00031c50202f0b5002685b020226946054603
:10f7d0000096fff7a1ff041e23db009b05f11c0729
:10f7e00038465968fff7f0fc041e1adb384646f02d
:10f7f0007afc01a8cde901660396fff7eefc041e32
:10f800000cdb202205f5d47101a846f073fd58b930
:10f810001b4901a8fff703fd041e0ada01a846f000
:10f8200062fc204605b0f0bd1cf0defe041ef5dbd8
:10f83000eee7144901a8fff7f2fc041eeedb1249c3
:10f8400001a8fff7ecfc041ee8db009b01a8d3e94c
:10f850000112fff7dbfc041ee0db009b01a85968e6
:10f8600046f0b8fd38b92846fff7e6fc0723002428
:10f87000c5f8c831d2e71cf0b7fe041ecedbf2e7b4
:10f88000fe290c02052a0c02b36b0c0230b50025d0
:10f8900085b04ff4007202a904460295fff73cffc1
:10f8a00000280edb114b02990093019503ab04f184
:10f8b0002800d1e90112039541f07cfa18b11cf03f
:10f8c00093fe05b030bddde9023204f11c00596839
:10f8d0009a60f8f7b7f90028f3db2046fff7acfc95
:10f8e00004230120c4f8c831ebe700bf31c5020290
:10f8f00038b515460c4601f1200205f11001fff75d
:10f90000effe002806db35b1236a5b680833002070
:10f91000c4e9033538bd2b46f9e7000038b554304b
:10f920000c460c311546fff7c5fb40b102460023db
:10f9300042f80c3bc0e901242860184638bd014854
:10f94000fce700bffcfeffff73b5b0f86e308a889d
:10f950009bb29a4205460c461fd1b0f8d830ca88ef
:10f960009a424ff000031dd1c96801aa0193fff725
:10f97000d5ff002812dbd4e90321019b58689af0d7
:10f98000f9fb019e09f034f82b6a4bb12b6a1e601b
:10f99000002434602e6209f02ff8002002b070bd00
:10f9a000ee61f5e71846f9e770b503680546092bdf
:10f9b0000c468cb003d00b2b26d00cb070bd01468a
:10f9c0002046fff7c1ff0028f7d020230026cde90d
:10f9d00004362b68029001930e4b04aa0093322048
:10f9e00033460d49f2f77efa4ff6ff72b4f86e30e7
:10f9f0009bb29342e1d03146b4f86e0080b20cb0b5
:10fa0000bde8704017f03ebd01462046fff757fda8
:10fa1000d9e700bf1c2a0c020c2a0c0210b50446c0
:10fa2000006808b10cf07efe204610bd03681bb1d3
:10fa30009a69026002b942601846704710b50379ae
:10fa4000044613b9012099f0acfe036823b118688d
:10fa500015f0fffa0023237110bd03681bb11a686b
:10fa6000026002b942601846704738b5056804461e
:10fa70004db108f0bdff25682b682360236803b9ea
:10fa8000636008f0b9ff284638bd0b46014618b13f
:10fa90001a681846d2681047704710b50c4629b14d
:10faa000fff77afb01462046fff7efff10bd70b568
:10fab0000c46a1b1d1e90956096afff7eeffe069ea
:10fac00008b10cf02ffe382120460cf02dfe35b188
:10fad00031462b46bde870406ff06300184770bd9b
:10fae0002de9f04390f8813004468bb023b900250e
:10faf00028460bb0bde8f083436c23b90a20304a96
:10fb00003049f1f76dfad4f87c8004f12409a66c31
:10fb1000b0451fd9656aedb1aa68a8eb0607974200
:10fb200028bf1746606c3a46696830449af022fb59
:10fb30006b683b446b60ab68db1bab6033b948461a
:10fb4000fff78bff29462046fff7a7ffa36c3b4436
:10fb5000a364dce7beb904f17803d3e8af3f002b20
:10fb6000c5d104f110073846fff760ff05460028ad
:10fb7000bdd0d0e9093100209847294620466e6261
:10fb8000fff795ffefe700233246616cb4f8d4002d
:10fb900017f038fda36c054683424ff000030bd0ed
:10fba0002022cde90223084a019000923220074921
:10fbb00002aaf2f797f99be71d46a36498e700bff6
:10fbc00021d40102482a0c02642a0c020c2a0c02dd
:10fbd00008b50346084619b103f15401fff755ff74
:10fbe00008bd00002de9f84f044689461746002558
:10fbf00000f11c06636bbb4228d34ff00008dff80e
:10fc000088a0dff888b0474539d9e66a26b9524658
:10fc100059460a20f1f7e4f9b268a7eb08059542c6
:10fc200028bf154671682a4609eb08009af0a2fa27
:10fc3000b3685b1bb360f3b904f12c00fff70dff51
:10fc400031462046fff7c4ffa844dce73046fff703
:10fc50000cff58b1236b3bb1186005602063636be8
:10fc6000826813446363c5e7e062f6e7636bbb42f7
:10fc7000c3d2bde8f88f73682b447360e4e7626b0e
:10fc80000120d21b6263f4e721d40102a12a0c02f5
:10fc9000f7b504461546002600f11c07636bab421e
:10fca00011d238460191fff7e0fe019958b1236b5c
:10fcb0003bb1186006602063636b82681344636322
:10fcc000ece7e062f6e7626b954228bf15464db15e
:10fcd0002a462046fff786ff20b90a20034a044936
:10fce000f1f77ef9284603b0f0bd00bf21d4010230
:10fcf000b62a0c02f7b51546d0e905329a420446f9
:10fd00000e4610d100270222806801a9adf80470c8
:10fd1000fff768fff8b1bdf804306361013bb3f54c
:10fd2000007f14d2a7616168d4e90523a068d21ac4
:10fd30001944fff7adffa36918446369a0619842b5
:10fd400009d363680020336063692b6001e06ff0c2
:10fd5000bd0003b0f0bd0120fbe7002313b56946e9
:10fd600001aa0446cde90033fff7c4ff40b9dde93d
:10fd7000001204f1280040f0e1ff18b11cf034fc3f
:10fd800002b010bd04f11c00dde90012f7f75affc4
:10fd90000028a2bf02230120c4f8c831f0e70023e5
:10fda00013b5694601aa0446cde90033fff7a2ff67
:10fdb00040b9dde9001204f1280041f043f818b120
:10fdc0001cf012fc02b010bd04f11c00dde90012b1
:10fdd000f7f738ff0028a2bf05230120c4f8c83177
:10fde000f0e70000f0b5836b04468fb0d3b9022270
:10fdf00006a9adf81830fff7f5fe00286ad0bdf867
:10fe000018502046294604f13802fff73ffc00282d
:10fe100060dba36bbdf81820db6910351a80022364
:10fe2000e5632364a36bd4e90f21dd69521a2046f0
:10fe30002944fff72dff236c1844e36b206498429c
:10fe400047d3e36c23b90a20234a2449f1f7c8f8c1
:10fe5000e66ca36baa1c9f68736d013373650693f0
:10fe6000706cb16c07ab03c308230593fb182b44dc
:10fe7000cde9032302230292cde9005330460c233f
:10fe800006aab91d46f012f918b11cf0adfb002806
:10fe900020db6988a36baa889986a36b00255a800a
:10fea0002023cde90635a36b01209a8e0c490292de
:10feb0005b8806aa01930b4b00932b46f2f712f8ce
:10fec000606822460368a16b1b689847c4e90e5519
:10fed000256400200fb0f0bd21d40102ca2a0c0213
:10fee0000c2a0c02e32a0c0238b5b0f86e308a896d
:10fef0009bb29a42044617d100f11c052846fff731
:10ff0000b4fd014618b12046fff762fef6e74ff652
:10ff1000ff73743424f8063c607354e8003f0133e7
:10ff2000c4e8e23f002af8d1002038bd70b503686c
:10ff30000546042b0c468cb027d0062b2ad0032b69
:10ff40002dd101462046fff793fa40b32023002627
:10ff5000cde904362b6802900193124b04aa00935a
:10ff6000322033461049f1f7bdff4ff6ff72b4f867
:10ff70006e309bb2934212d03146b4f86e0080b21c
:10ff80000cb0bde8704017f07dba01462046fff77f
:10ff9000abffdae701462046fff786fad5e70cb05b
:10ffa00070bd00bf1c2a0c020c2a0c020368016001
:10ffb00013b118460cf0b6bb704710b504460021cb
:10ffc0000430fff7f3ffd4e90201fff766fd0023d9
:10ffd000c4e90533e36010bd00232de9f04194b07e
:10ffe00004aa03a90646cde90333fff783fe0446be
:10fff000a0b9049a202a40f0b9805f4b06f1280886
:020000040807eb
:1000000006f5c4750590019000932946404605ab5e
:1000100041f00cf830b11cf0e7fa0446204614b069
:10002000bde8f081059f202f40f0a280404640f0bf
:1000300028fe06a8cde906440894f7f7e1fd041e62
:1000400036db06a8f7f7f5fd041e31db3a462946f4
:1000500006a8f7f7f7fd041e2adb0822474906a881
:10006000f7f7f0fd041e23db06f5d478414606a819
:10007000fff7aaf8041e1bdb06a846f034f806a812
:10008000f7f7befd041e13db06f11c07394606a870
:1000900046f056f880b900251c2229460da80c957b
:1000a0009af08ff80ca906a8fff78ef8041e08da5c
:1000b00006a846f018f8b1e71cf096fa041ef7db24
:1000c000e9e706a846f00ff809a8cde909550b9510
:1000d000fff783f8041e0bdb2022414609a846f0f7
:1000e00009f948b9264909a8fff799f8041e08da62
:1000f00009a845f0f8ffdbe71cf076fa041ef7dbf1
:10010000f0e7204909a8fff78af8041ef0db1e4932
:1001100009a8fff784f8041eeadb20220ca909a82d
:10012000fff774f8041ee3db0ca909a846f052f9a6
:10013000a8b9039c202220460ca99af00bf898b984
:1001400021463846049af7f77dfd041ed0db304681
:10015000fff733ff06230124c6f8c831c8e71cf0b7
:1001600043fa041ec4dbe4e7084cc1e7074c55e73b
:100170006ff0f90452e700bf31c50202102b0c02e8
:10018000fe290c02b36b0c02052a0c02e8feffffed
:1001900010b5d0f8c8310446013b062b05d8dfe87e
:1001a00003f0070f1215181b1e006ff0d10010bdd1
:1001b000fff7d3fd0028fada0823c4f8c831f6e7c0
:1001c000fff764fbf6e7fff7eafdf3e7fff7c8fa8e
:1001d000f0e7fff701ffede7fff7f4faeae70020a9
:1001e000e5e7000010b504460f4b40f8283b40f00f
:1001f00048fd2022002104f5c47099f0e2ff20227e
:10020000002104f5d47099f0dcff04f11c0045f0e6
:100210006aff064b20462360fff7cffe201dfff745
:10022000fdfb204610bd00bf102c0c02fc2b0c0265
:1002300010b50446fff7d6ff20464ff4e6710cf0e8
:1002400073fa204610bd036801601bb11a68184696
:100250005268104770470000f0b5002689b004ad21
:10026000074632460f2128460696cde90466cdf8aa
:100270001b600bf0f4ff002852db0e2858dd4ff412
:10028000e6702e4999f0f2f9044690b12c4bc0e982
:100290000167c0e90366c0e90566c0e90766036057
:1002a00046624ff4b0723146283099f08affc4f8a4
:1002b000c861214607f15000fff7c5ff3c6d002cd7
:1002c00039d01e494ff4007099f0d2f90146201d33
:1002d000fff76cfe63684bb30ff07bfe04f11c0666
:1002e00020613046f7f78cfc031e17db3046f7f72a
:1002f000a0fc031e12db04f12800039040f096fce2
:100300000f230622cde9005301210323039840f077
:10031000e3fc034630b11cf067f9034603eae370df
:1003200009b0f0bd0122c4f8c821f7e7054bf5e795
:100330006ff0f900f4e70348f2e700bf751d0e0205
:10034000102c0c02fcfeffff10b50a490446f420f5
:1003500099f08ef9014604f14400fff727fe636c23
:100360002bb12046fff778ff00eae07010bd02488d
:10037000fce700bf751d0e02fcfeffff034607b53c
:100380000068196048b1019045f034fe5c21019885
:1003900003b05df804eb0cf0c7b903b05df804fbe3
:1003a00070b5036d054623b90a20214a2149f0f7ab
:1003b00017fe2c6dd4f8c831072b26d104f5c47470
:1003c0005c201d4999f052f9064630b144220021c3
:1003d00099f0f7fe0023c6e9153305f14c003146cc
:1003e000fff7ccffed6c05b3284645f0dcfd80231c
:1003f00022460221284645f0dafd034660b11cf092
:10040000f3f8034603eae37070bd0a20084a0b497b
:10041000f0f7e6fd0024d3e722696a646269aa6402
:10042000a269ea64e2692a65ece70548ece700bfe7
:1004300021d40102192b0c02751d0e02312b0c0266
:10044000fcfeffff10b50368044613b9012099f0c4
:10045000a8f902790ab12d20f9e7186814f0eafd2d
:100460000123237110bd0000f0b500f1180391b015
:1004700006930023064606a88df81c30fff7e2ff1e
:10048000012306f108058df81c302846fff7cefa47
:10049000044640b1026b336f9a4204d001463046a5
:1004a000fff705fbf1e706a8fff7c8fa002c6cd0b0
:1004b000236a002b58d0236a5d6823692b80e36a86
:1004c000a28e6b606a80f36c23b90a20304a3149ee
:1004d000f0f786fdf76cd4f810c0bb6daa1c013391
:1004e000bb6543f000430893f86c396d09ab03c357
:1004f0000823059363442b44cde90323022302928e
:10050000cde9005338460c2308aa0cf1060145f04a
:1005100093fd18b11cf068f8051e2ddbb36a226a42
:10052000002b2ed01a6000231360b26220222362b7
:10053000cde90823a28e01200192174a17490092a3
:1005400008aaf1f7cffc656ab5b17369dbb19c61ac
:100550000025a56174619df81c3013b106a8fff752
:100560006dfa284611b0f0bd1021304604f120028a
:10057000fff7b6f8051e9eda21463046fff797fad8
:10058000e9e77262cfe73461e2e72546e3e700bfbf
:1005900021d40102ca2a0c02492b0c020c2a0c029b
:1005a00073b590f882300446002b58d000215030ab
:1005b000fff749fe002104f14c00fff7dffe0021a8
:1005c00004f14400fff7f2fc04f118030093002348
:1005d00068468df80430fff735ff012304f1080564
:1005e0008df804302846fff721fa014618b120465d
:1005f000fff75dfaf6e76846fff720fa04f1100509
:100600002846fff713fa014690b904f1240528465d
:10061000fff723fa014678b904f12c063046fff7bc
:100620001cfa054660b101462046fff7d1faf5e70e
:100630002046fff73cfae3e72046fff72efae6e70d
:100640002046a16bfff733fa9df80430c4e90e553c
:1006500025646563a56413b16846fff7eff902b03e
:1006600070bd000070b505468cb000f17403d3e88e
:10067000af3f026f9a4260d0b0f86e20b0f86c4085
:100680000367a0f86c20fff78bff4ff6ff72b5f8f9
:100690006c30934239d000242023cde90434574be9
:1006a00001205749009304aa2346f1f71bfc234677
:1006b00022464ff400200021cde901440094f5f7d3
:1006c000abfe2846fff740fe0446002835d0202325
:1006d000002601944ff6ff74cde90436494b3220d1
:1006e00000934749334604aaf1f7fcfbb5f86c00c8
:1006f000a04204d0314616f0c5fea5f86c4028464d
:100700000cb0bde87040fff74bbf9c4266d00024a0
:100710002023cde904343c4b01203949009304aa3d
:100720002346f1f7dffb234601224ff4002000218e
:10073000cde901440094f5f76ffe4ff6ff73b5f86d
:100740006c209a424ad0286d002849d003689b68e3
:100750009847041e16da00262023cde904362b4bd9
:10076000322000932649334604aaf1f7bbfb3346f7
:10077000cde90166009602224ff400200021f5f732
:100780004bfea4e723d12846fff70afe044620b11a
:100790000023cde901330093ede7014605f1500058
:1007a000fff751fd2023cde90434194b01201449f2
:1007b000009304aa2346f1f795fb234603224ff446
:1007c00000200021cde901440094f5f725fe2846dc
:1007d000fff786f9044600287ff479af0cb070bdae
:1007e0002846fff741fe044600287ff470af2846f4
:1007f000fff7f8fa04460028e9d068e7762b0c02e8
:100800000c2a0c02ad2b0c02802b0c028d2b0c023f
:100810009e2b0c022de9f04304460f461568dff8c5
:10082000888087b0002d3dd0d5f80c90d9f80030e5
:100830005e78022e01d02d68f4e718220021684668
:1008400099f0bffcd9f800305a78022a18d1012259
:100850005b688df800201bba019399f81030394677
:10086000204605931cf066f830b16a4641462046a2
:100870001cf0eaf90028ded1002007b0bde8f083c3
:100880000a2af9d103f108028df800600df1040c79
:100890001833664610685168083203c69a42b44657
:1008a000f7d1dae70120e8e77a0d0c0238b51468d1
:1008b000054623685bb163684bb11cf03bf838b167
:1008c000d4e900122846bde838401cf07ab901206e
:1008d00038bd00002de9f04304460f461568dff8e7
:1008e0008c8087b0002d3ed0d5f80c90d9f8003020
:1008f0005b780a2b01d02d68f4e7182200216846a6
:1009000099f05ffcd9f800305a78022a18d10122f8
:100910005b688df800201bba019399f810303946b6
:10092000204605931cf006f830b16a464146204641
:100930001cf08af90028ded1002007b0bde8f08362
:100940000a2af9d102220df1040c8df8002003f1de
:1009500008021833664610685168083203c69a4286
:10096000b446f7d1d9e70120e7e700bf7a0d0c02c2
:1009700070b50c460546f0f725fa06462046f0f716
:1009800021fa8642024607d3214628469bf04efaba
:10099000b0fa80f0400970bd0020fce710b51249a4
:1009a0000446fff7e5ffb8b920461049fff7e0ff1e
:1009b000a0b920460e49fff7dbff88b920460d4954
:1009c000fff7d6ff70b920460b49fff7d1ff00288b
:1009d00014bf1020002010bd0120fce70220fae720
:1009e0000420f8e70820f6e7842c0c02cd290d023c
:1009f00042800c02d81f0c023d2e0c022de9f04f54
:100a000005460e4600271468dff88480dff88490de
:100a10008db0002c3ad060680df10f018df80f7089
:100a200019f02dfa70bb0490adf814000df1100b05
:100a30005946606819f03ffb019018bb5846fff714
:100a4000adff8246f0b10199102208a899f0b9fbd8
:100a50005846f0f7b7f906abcde909839df80f309a
:100a6000cde906b03146284608938df82ca01bf03e
:100a700061ff38b14946284608aa1cf0e5f808b1dc
:100a80002468c6e700200db0bde8f08f0120fae72a
:100a90002d080102980d0c02002330b585b00546e3
:100aa00001a8019319f0d2f8041e0ddb019b284622
:100ab0000393074b074902aa029300f0e9f800ea02
:100ac000e074019819f0eef8204605b030bd00bf83
:100ad0007d0901023e0d0c02f0b500269fb06a466a
:100ae00047490546009600f00df9041ec0f28280c9
:100af0009df8000001a9019619f01af9041e79db8e
:100b0000019b23b90a203f4a3f49f0f769fa0026c2
:100b1000402200210ea899f054fb04af009b3946f7
:100b200001980d930496adf8146019f0c4fa041ef0
:100b300060db3846f0f746f906ab0f93334bcde94f
:100b4000067038460e93fff729ff8df84000002805
:100b500053d0019802a9029619f0aff9041e49db9f
:100b6000029b019802a9119319f016f9041e41dbaa
:100b7000029b019802a9129319f09efc041e39db16
:100b8000029b019802a91c9319f0cdfc041e31dbd5
:100b9000029b1222314608a81d9399f012fb01987e
:100ba00008a919f0b4fd041e24db9df829200df1dd
:100bb0002a01082a28bf08220df165008df864205b
:100bc00099f0d8fa019803a9039619f0cafd041efa
:100bd00010db039b0e4a149318930e4b1392284676
:100be0000d490daa179300f053f800eae07403983a
:100bf00019f09ffc20461fb0f0bd6ff06304f9e7c9
:100c0000660d0c0221d40102872c0c022d08010272
:100c10009507010255080102520d0c02002230b561
:100c200087b0054602a90a20cde90122f1f73afc76
:100c3000e0b9029c0cb1236923b90a200c4a0d4982
:100c4000f0f7cef90c23039301ab0493042305932f
:100c500001212046236903aa984738b9019b2846f9
:100c6000054903aa8df80c3000f012f807b030bd2a
:100c700021d40102af180c0288090c0208b5faf75a
:100c80001dfe002008bd08b5faf73afe002008bd99
:100c90002de9f3410024054601a80f469046019432
:100ca0001bf07cfff0b1224628460199f3f7b8f813
:100cb0000446c8b9f0f7d6fb0646f0b1d5e90312f1
:100cc0002346f0f7e3fb28b14246394630461bf095
:100cd00031ff08b96ff0630400213046f0f7c6fb1e
:100ce0003cb101e06ff06304002228461146f3f79f
:100cf00097f8204602b0bde8f081014cf4e700bf50
:100d0000fcfefffff8b5044600200e461746f0f73c
:100d1000b3fb054698b1d4e901120023f0f7ccfbf0
:100d200080b13a46314628461cf006fb0028074ca5
:100d300018bf002400212846f0f7a2fb00e0044c75
:100d40002046f8bd6ff06304f4e700bfe8feffff44
:100d5000fcfeffff70b500248ab005460c2101a8f7
:100d6000cde9014403940bf0cbf90c2825d12146a1
:100d7000182204a899f025fa01ab04a913f8012b55
:100d80000134160906f13000392888bf06f15700f2
:100d900002f00f0201f8020b02f13000392888bf7f
:100da00002f157000c2c01f8010ce7d12846044948
:100db00004aafff76dff0ab070bd6ff06300fae799
:100dc000780a0c021fb5102200210446684699f0eb
:100dd000f8f90022102168460bf0bcf9002804db6a
:100de0006a4620460249fff753ff04b010bd00bf1a
:100df000e60a0c021fb5074b6a4602930a230393c7
:100e000002ab0193044b05490093fff741ff05b086
:100e10005df804fba30f0c022d0801020e0b0c025f
:100e20002de9f0418eb0074608f058fd002846d065
:100e30000568002d43d02b6828461b6d98472b680a
:100e400028461b699847041e31db1c2200260deb47
:100e500002003146069699f0b4f92b680df1180896
:100e60002022414628461b6b9847041e1fdbadf825
:100e700002602b6828465b6b0df102019847041e47
:100e800015db4046cde903660596eff79bff01ab06
:100e900004930c4bcde901800393bdf80230384632
:100ea000094903aa0593fff7f3fe00eae0742b68f3
:100eb00028465b6d984720460eb0bde8f0816ff084
:100ec0006304f8e72d080102c80a0c02002307b5e5
:100ed000044901aa0193fff7dbfe00eae07003b0ca
:100ee0005df804fbfa0a0c0210b5044690b04022eb
:100ef0000021684699f065f96a4620460449fff7e3
:100f000001ff10b9684610f015f810b010bd00bf11
:100f1000360b0c0213b5044600208df8040010f0c7
:100f200048f804498df8040001aa2046fff7b0fef6
:100f300002b010bd220b0c02002208b511460120a0
:100f4000f8f73cf8002008bd002208b5104611460d
:100f5000f8f734f8002008bd002213b50446114606
:100f60001046f5f792fe04498df8040001aa2046c8
:100f7000fff78efe02b010bd8c0a0c026ff07700f6
:100f800070476ff07700704713b500240a4901aa33
:100f90008df80440fff7b6fe00280adb9df8041028
:100fa0002246012918bf21460420f2f7f1f800ea91
:100fb000e07002b010bd00bf680b0c02002307b543
:100fc0000c4901aaadf80430fff79cfe00280adbab
:100fd0009df80430012b09d106209df8051007f07b
:100fe0007dff00eae07003b05df804fb6ff077006e
:100ff000f9e700bf4a0b0c0237b500256a460f49d6
:1010000004468df80050fff77dfe002811db9df8a7
:1010100000308df80450012b0dd1062007f084ff1d
:1010200007498df8040001aa2046fff731fe00eac7
:10103000e07003b030bd6ff07700fae7b40a0c023d
:10104000a00a0c0238b5002281680446f2f7e8fed7
:10105000054620b9d4e90112e06899f08bf82846da
:1010600038bd6ff0770070476ff0770070476ff012
:10107000770070476ff0770070476ff07700704728
:101080006ff0770070476ff0770070472de9f047f9
:1010900013680646d3e900471823884603fb074731
:1010a000dff858a0dff8589086b0bc4223d0002368
:1010b000cde90333059325682846eff783fe01ab9e
:1010c000cde90150cde903a3636941468df81430a1
:1010d000237c30468df815301bf02cfc38b1494686
:1010e000304603aa1bf0b0fd18340028ddd10020e3
:1010f00006b0bde8f0870120fae700bf2d08010225
:10110000120c0c0270b585680446681c166899f0cc
:1011100003f8306048b10022425575602a462046e7
:101120003168bde870401bf0a5be70bd2de9f04fe1
:1011300013680546d3e900471823884603fb074791
:10114000dff884a0dff884b0dff884908bb0bc4275
:1011500038d026461822002104a899f032f856f813
:10116000043b18460193eff72dfe019b0622cde9c3
:101170000230594602ab3046cde904a398f0eaffad
:1011800040b16368cdf81930b388adf81d3006233f
:101190008df81830e36841468df81f3023692846e2
:1011a0000893636909931bf0c5fb38b1494628468b
:1011b00004aa1bf049fd18340028c8d100200bb048
:1011c000bde8f08f0120fae72d0801029e2c0c02e9
:1011d000a80c0c0210b50446086808b19af0d0f8c3
:1011e0002060204610bd10b50446006898f09cffb2
:1011f000204610bd10b5037904461bb10068036892
:101200005b6d9847204610bd10b504460068036822
:101210001b6d98470123237110bd10b504460c3097
:10122000fff7e1ff2046fff7deff204610bd034633
:10123000002010b50a461c461860096844f8041bd3
:10124000114641f8040b03c95860a180d1681846c3
:10125000d9601169526919615a6110bd38b50446e7
:101260000d46fff7b7ffd5e901016060218104f168
:101270000c0005f10c01fff7adff2b7c2046237419
:101280006b69636138bd0000f0b5002587b002ab23
:101290000193234b6a462349cde902550093fff79a
:1012a00031fd041e31db08f019fb0746002834d05d
:1012b000066896b304a804968df81450fff7a4ffaf
:1012c000336830461b699847041e1bdb2a460221ff
:1012d0000420f5f743fd336830469b6a9847041ea7
:1012e00010db2b462a4629460420f5f7c3fe384674
:1012f000029909f055f9041e0dda2a46022104204c
:10130000f5f72cfd04a8fff775ff029898f00cff85
:10131000204607b0f0bd2c46f4e76ff06304f4e715
:10132000851001024e0c0c0230b500240a46054619
:1013300004600968034645f8041b114641f8044b54
:1013400003c95860a980dc60d168d460d960117c81
:101350001846197452695a6130bd000070b586b0e4
:10136000054608f0bbfa30b3002303ae31461348fc
:10137000cde90333059308f03dfe041e09db104b55
:101380002846104901aa02960193fff781fc00ea62
:10139000e0741826dde9035306fb0356ae4204d081
:1013a0002846fff73aff1835f8e7039898f0bcfe97
:1013b000204606b070bd6ff06304f9e71919010209
:1013c0000d1001023a0c0c0230b5002585b002abbd
:1013d00001930d4b6a460d49cde902550093fff785
:1013e00091fc041e06db08f079fa48b1029808f077
:1013f0004ffe2c46029898f097fe204605b030bd6f
:101400006ff06304f6e700bf85100102940c0c0234
:1014100008b508f063fa18b108f018fe002008bdfe
:101420006ff06300fbe7000070b58eb0064608f071
:1014300055fa002843d00368002b40d00025214aec
:10144000cde906551068928804900395adf81420f4
:101450001a681846126e03a99047041e29db182249
:10146000294608a898f0adfe039c2046eff7aafc99
:1014700001ab0993144bcde901400622134904a89e
:10148000089398f067fe48b1bdf814300498adf8a1
:101490002d300623cdf829008df82830069b3046e4
:1014a0000c93079b0a4908aa0d93fff7f1fb00ea8a
:1014b000e07403a8fff797fe20460eb070bd6ff0f2
:1014c0006304f9e7cbfe0b022d0801029e2c0c02ef
:1014d000e00b0c0270b51826d0e90053044606fb59
:1014e0000356ae4204d02846fff77dfe1835f8e7d4
:1014f000206898f019fe204670bd00002de9f041eb
:101500000025a8b004ab2293ae4b06aacde9263243
:10151000ad4921aacde92355cde90455cde90655bc
:1015200025952193fff7eefb041ec0f218819df86c
:101530009430012b00f22f8108958df8243009d1c9
:10154000069808b199f01cff002308901ba81b9374
:10155000fff749fe00234ff0ff32cde90f324ff67f
:10156000ff720498cde91123cde9133308b199f046
:1015700007ff00230f901ba81b93fff734fe9df875
:101580008c30062b40f0f5809df88d509df88e40f4
:101590009df88f009df890109df891209df8923055
:1015a0008df840508df841408df842008df8431081
:1015b0008df844208df8453008f090f90546002854
:1015c00000f0e680d0f80080b8f1000f00f0e08075
:1015d00000240aa88df82c40cdf82880fff714fecf
:1015e000cde90c440e94d8f8003040465b6e774944
:1015f0000caa9847041ec0f2a680dde90c46182309
:1016000003fb0646a6421ad021461ba8fff7e2fdbf
:10161000d4e901011c90adf87410e7681b991e977e
:10162000236904981f93636918342093eff7c0fb74
:10163000002840f0a5801ba81497fff7d4fd0027d1
:101640009df82430089a8df87030129b15a81292dc
:10165000159308971b97fff7c6fd9df870301ba8e0
:101660008df84c30fff7bffd4ff0ff324ff6ff73a0
:1016700015a90498cde91623cde9187715971a977f
:1016800008f076fc0fa906461ba8fff7e7fd1ba88c
:1016900008f028fe04461ba8fff7bffdbc424fdb45
:1016a000d8f8003040461b699847041e7cdb3a4658
:1016b00039460420f5f77bfa074628b90246014669
:1016c0000420f5f725fa0746d8f800304046db69d4
:1016d0009847d8f8003040469b699847041e63db62
:1016e000d8f8003040469b6a984700220221042027
:1016f000f5f734fbd8f8003040469b699847041e44
:1017000052dbd8f8003040461b699847041e4bdb7b
:101710000023042019461a46f5f7acfc2846049924
:1017200008f03eff041e4ff0000537db2b46012278
:1017300010200021cde901550095f4f76dfe2c46ef
:1017400015a8fff76afd0ca8fff7c4fe0aa8fff76b
:1017500051fd0fa8fff761fd08a8fff744fd0698ab
:1017600098f0e2fc049898f0dffc204628b0bde831
:10177000f081ff231a46194618461c461d460fe7fe
:101780001ba8fff730fd3de70f9808f081fcd7e775
:101790006ff06304dde76ff07704e0e727b93a46be
:1017a00002210420f5f7dafa002eedd115a91ba8c5
:1017b000fff754fd1ba808f095fd1ba8fff72dfdb2
:1017c000bee700bf85100102620c0c02bd180102c9
:1017d000f0b589b0074608f081f800282dd00568db
:1017e0005db3002601a801958df80860fff70cfd98
:1017f0002b6828461b699847041e18dbcde905664f
:1018000007962b6805ae324628465b6e0c49984712
:10181000041e09db0b4b38460b4903aa04960393bd
:10182000fff736fa00eae0743046fff753fe01a8ee
:10183000fff7e0fc204609b0f0bd6ff06304f9e764
:10184000c1180102ad100102e40c0c028842f8b587
:1018500004460d46164614d9904213d2a2f118063a
:10186000751aa1f118072c44b74218d01cb13146a3
:101870002046fff7dcfc3046fff7b5fc183e183c6d
:10188000f2e70cd0b5420ad01cb129462046fff73a
:10189000cefc2846fff7a7fc18351834f2e7f8bd50
:1018a0002de9f0410c468cb001466846fff7bffcbd
:1018b000694606a86668fff7bafcd4e901739f423f
:1018c00016db0137002f35dd4ff0180808fb07f84d
:1018d000404698f021fc0546f8b12168a8f11802ad
:1018e0000a44fff7b3ff206898f01efc2560a7604c
:1018f00018222368616802fb063602fb013206f1fa
:1019000018003146fff7a2ff1eb1304606a9fff7c7
:101910008efc012563680133636006a8fff763fc52
:101920006846fff760fc002d034818bf00200cb08c
:10193000bde8f0810025d6e7fcfefffffff7b0bf52
:10194000fff7aebf8842f8b504460d46164614d9d7
:10195000904213d2a2f11806751aa1f118072c446f
:10196000b74218d01cb131462046fff7ddfc3046a7
:10197000fff753fc183e183cf2e70cd0b5420ad0f2
:101980001cb129462046fff7cffc2846fff745fc4f
:1019900018351834f2e7f8bd2de9f0410c468cb04b
:1019a00001466846fff7c0fc694606a86668fff76f
:1019b000bbfcd4e901739f4216db0137002f35ddf4
:1019c0004ff0180808fb07f8404698f0a5fb0546bd
:1019d000f8b12168a8f118020a44fff7b3ff2068a4
:1019e00098f0a2fb2560a76018222368616802fbbb
:1019f000063602fb013206f118003146fff7a2ff5e
:101a00001eb1304606a9fff78ffc0125636801333c
:101a1000636006a8fff701fc6846fff7fefb002d98
:101a2000034818bf00200cb0bde8f0810025d6e7c0
:101a3000fcfeffff2de9ff4700248246274615687c
:101a40000e46dff85c90dff85c802b7c697c6a8a4c
:101a5000023bdbb2062b02d819f803302bb9e4b9ec
:101a600001242b7d697dea8af2e7cde90212504616
:101a70003146adf805708df807708df804301af016
:101a800059ff30b14146504601aa1bf0ddf800284d
:101a9000e5d1002004b0bde8f0872046fae700bf9a
:101aa000172d0c02c4090c02134682681ab11b6878
:101ab0004168c3e9001200211bf0dcb92de9f04fa9
:101ac00006460f460025d2f80080dff89c90dff82c
:101ad0009cb089b0b8f80830ab4241d97823d8f827
:101ae000044003fb0544a17b002933d194f8223044
:101af000023bdbb2062b2dd819f803a0baf1000f78
:101b000028d01c2201a898f05cfb94f823303946b9
:101b10000293e38b30460393d4e905239b1ab4f870
:101b20007020049382f00203c3f34003520758bfae
:101b300043f0020305930b4b14348df804a0079473
:101b400006931af0f7fe38b15946304601aa1bf049
:101b50007bf808b10135bde7002009b0bde8f08f82
:101b60000120fae7b5190102172d0c02ec090c024d
:101b70000022044b18681a6010b11c210af0d4bd71
:101b8000704700bfb8d0001000b50f4b8bb018687d
:101b9000b0b100220121f1f769fc00280bda202204
:101ba0000023cde90223094a01900092322008491e
:101bb00002aaf0f797f90bb05df804ebfff7d8bf76
:101bc0000bb05df804fb00bfb8d00010a42c0c02d1
:101bd00018100c0200b50f4b8bb01868b0b1002282
:101be0001146f1f743fc00280bda20220023cde94f
:101bf0000223094a019000922820084902aaf0f71e
